:020000040000FA
:040000006FD00400B9
:101000006F00907E00000000000000009020002093
:10101000AA220020A9BDF9F56C23002000000000E1
:10102000000000006C230020902000200000000041
:101030000000000090200020000000009020002010
:101040000000000090200020902000209020002030
:101050009020002090200020582F00209424002071
:101060000000000090200020902000201E2400207E
:1010700090200020D22300209020002090200020EB
:101080009020002090200020902000209020002020
:101090009020002001A04111B7170040985F3AC688
:1010A000945F3247E39CE6FE3245410182800111A4
:1010B00013078008F337078093F787083EC20100C3
:1010C0000100B7170040930570052380B70413068D
:1010D00080FA2380C7040100010083C6B70493F699
:1010E000F60DA385D704238007049246F3A6068055
:1010F0000100010093760502D5CEF336078093F602
:10110000860836C4010001002380B7042380C70489
:1011100001000100B70614007D89558D88C70100C4
:1011200001000100010023800704A246F3A6068007
:101130000100010073370780137787083AC6010062
:1011400001002380B7042380C704010001000100CF
:1011500001003727004093061005A303D7802380A2
:101160000704B247F3A70780010001009307800836
:10117000F3B7078093F787083ECE01000100B71749
:101180000040130770052380E704130780FA2380CB
:10119000E7040100010003C7B70413670708A3852C
:1011A000E70423800704F247F3A70780010001004A
:1011B0000561828093760504BDC6F336078093F6F9
:1011C000860836C8010001002380B7042380C704C5
:1011D00001000100B7061400938606047D89558D31
:1011E00088C7010001000100010023800704C246F6
:1011F000F3A6068001000100733707801377870884
:101200003ACA010001002380B7042380C70401000B
:1012100001003727004093062005A303D7802380D1
:101220000704D24781B773370780137787083ACC12
:10123000010001002380B7042380C70401000100DE
:1012400098471367070C98C723800704E24719BF24
:101250000111814601468145114506CE97000000E7
:10126000E780605893078008F3B7078093F78708F3
:101270003EC601000100B717004013077005238028
:10128000E704130780FA2380E7040100010003C785
:101290006704136717002383E70423800704B2471A
:1012A000F3A7078001000100F2400561828041112F
:1012B000814601468145114597000000E780A05214
:1012C00013078008F337078093F787083EC40100AF
:1012D0000100B7170040130670052380C70493066A
:1012E00080FA2380D70401000100FD552396B70240
:1012F00023800704A245F3A5058001000100733790
:101300000780137787083AC6010001002380C704CD
:101310002380D7040100010003C767041367170087
:101320002383E70423800704B247F3A70780010063
:10133000010001A0BD473305F50201007D1575FDD3
:101340008280411122C426C206C6AA8401446317C2
:101350009400B24022449244410182800504130566
:10136000803E420497000000E78000FD4180C5B741
:101370009305000273A04580824573901534924016
:101380002242B2424243D2436244F2440255925551
:101390002256B2564257D2576258F25806499649D9
:1013A000264AB64A464BD64B664CF64C065D965DD1
:1013B000265EB65E465FD65F09617300203041113C
:1013C000B7170040985F3AC6945F3247E39CE6FE49
:1013D000324541018280B71700401307000323887C
:1013E000E702854717170000232EF74673002030C9
:1013F000411122C42D6426C24AC006C637190040D6
:101400001304A4AAB704002023208900976000E0F9
:10141000E780C0299C408297976000E0E780002920
:10142000E5B737370040834747009146BD8B639E41
:10143000D702B73600401306F00F973500009385AA
:10144000651E9737000083D7E72D03C7A6001377E3
:10145000F70F1DE3B7E70400BC4F09468945171590
:1014600000000345A5F7829731A099466394D70001
:10147000834757007300203003C786001377F70FA8
:10148000E365F6FC13851700AE9717380000231BA1
:10149000A8282380E70075B7B787004003C7670017
:1014A000098B6309071003C77700930600031377BE
:1014B0000703630DD70817380000034878761736FE
:1014C00000001306E6720547B30606012380E60016
:1014D00083C577001737000013078773429793F58A
:1014E000F50F2300B70003C58700973500009385EB
:1014F0002571C2951375F50F2380A50003470700DA
:1015000089451377F703630CB70C63E7E50A6306B5
:10151000071A8545630CB7129737000083C75770C9
:101520003307F600034707001377F70F19CB85073A
:1015300093F7F70F3D476363F71A17370000A301CE
:10154000F76EB787004009472383E700B78700405D
:1015500083C77700E207E18763DE0704973700005F
:1015600083C7176C17370000130787683E978546B7
:101570002300D70017370000130787693E979306AB
:1015800000032300D70017370000130767673E9753
:10159000A14685072300D70093F7F70F3D47636403
:1015A000F71417370000A30DF766B7870040094707
:1015B0002383E70073002030930610026300D70EE8
:1015C000930620026305D70693060002E316D7F4BC
:1015D00003C727021377C70F13672700D5A803C7D0
:1015E00067001377070465CB03C7A702173800000D
:1015F00013088841173500001305C538134707083D
:101600002385E70203C7A7021377370F1367870005
:101610002385E702814713070004B305F5008C41D9
:10162000B306F80091078CC2E399E7FEF5B503C74E
:10163000A702134707042385E70203C7A70213770E
:10164000C70F136727002385E702F9B503C76700B3
:101650001377070449C303C767021738000013084C
:10166000682E173500001305A525134707082383A7
:10167000E70203C767021377370F136787002383D7
:10168000E702814713070004B305F5008C41B30658
:10169000F80091078CC2E399E7FEBDBD03C767025E
:1016A000134707042383E70203C767021377C70FB3
:1016B000136727002383E70285B503C76700137705
:1016C000070411CB03C727021377370F136787006F
:1016D0002381E70291B5238006003DBD97370000C6
:1016E000A3800754B9BD97370000A38B075275BD7F
:1016F0002303048015472303E48001002302A48010
:10170000828083076480E3CE07FE23030480828007
:1017100083076480E3CE07FE03454480828083070D
:101720006480E3CE07FE2302A4808280411126C498
:101730004AC24EC006C61377F50BAD47AA892E895B
:101740009544630CF700194597000000E78080FA84
:1017500097000000E78020FB8D444E859700000035
:10176000E78040F9FD59FD1463983401B240A2446A
:101770001249824941018280135509011375F50F01
:1017800097000000E780E0F92209F1BF011126CCA3
:1017900006CEB704080097000000E780C0F61545A4
:1017A00097000000E78000F597000000E78080F6D2
:1017B00097000000E78000F62AC697000000E78047
:1017C00080F432459377150089EB13651500137586
:1017D000F50FF240E24405618280FD14E9F0014515
:1017E000CDBF397126DC4ADA4ED852D656D45AD2F9
:1017F0005ED006DE62CE66CCB7E700E07D5783AAF6
:10180000070022C603AA470023A0E71823A2E7186F
:10181000B7170040130770052380E704130780FA09
:101820002380E70483C74704930B75FFB684E20760
:1018300093FBFB0F8546AA892E8B32893724004003
:10184000E187015763FA76016308D50089461307DB
:1018500000026313D5000157D98F93F7F70FB71C18
:1018600000402382FC0411472303E4801305F00F9A
:1018700097000000E78000E8094C97000000E7802F
:1018800080E863657C15B7050700DA9537870700A0
:10189000795563FEE504B3879500636AF704370B57
:1018A0000800A94733EB65016395F90881E8814495
:1018B00097000000E78020E5268515A8DA85094510
:1018C00097000000E780C0E605090345F9FFFD1415
:1018D000050B97000000E780C0E481C49377FB0FFD
:1018E000E5F797000000E780A0EA69F17D55B7179A
:1018F0000040130770052380E704130780FA238054
:10190000E70403C74704418B2382E704F250B7E79B
:1019100000E023A0571123A24711E2543244525948
:10192000C259325AA25A125B825B724CE24C21615C
:101930008280A547639BF90685691309F00FB306FA
:101940009900B3742B01B6941349F9FFB37499004D
:10195000856B33796901416B9387F9FFB3F72701F1
:1019600099E363FC340193D94900C147E3E637FFAB
:101970003DBF0569C1697D19D9B71305800D63881D
:101980006901130500026384790113051008CA85F3
:1019900097000000E780C0D997000000E78040DF93
:1019A00031D54E99B38434416DBFDA852D4597000A
:1019B0000000E780E0D7CA94E30B99EE0509970091
:1019C0000000E78020D5A30FA9FEFDB79387F9FF9C
:1019D00093F7F70F636DFC0C83C71C0413073008E3
:1019E0006315F706370708006361EB06B3079B0032
:1019F000B706100063FBD704334BEB0089476399AC
:101A0000F9068980D549E38404EADA850945970017
:101A10000000E780E0D111090327C9FF9147232087
:101A2000E48003076480E34E07FE23033481FD173F
:101A3000EDFBFD14110B81C49377FB0FE9FF9700B9
:101A40000000E780E0D461F155B5B717004003C747
:101A50005704B70708001377070219E3B787070091
:101A60007955E376FBE833079B00E3F9E7F841B5E6
:101A70008547E380F9F0DA852D4597000000E7807F
:101A800020CB9389F4FFE38404E297000000E78011
:101A900060C893F7390091EB83260480032709007F
:101AA00093074900E396E6E03E89CE84D9BFB54767
:101AB0006399F9001305900B97000000E78080C33D
:101AC000FDB3B1471305B00AE388F9FE9947639760
:101AD000F904B7050800B365BB002D459700000069
:101AE000E78000C581448D4BA14997000000E78045
:101AF00060C263967401832704802320F900850463
:101B0000E39534FF8327048013172B0163550700E7
:101B10002312F90069BB2322F90051BB9D47639F43
:101B2000F90281451305B00497000000E78040C02A
:101B3000BD442320090023220900FD59970000001D
:101B4000E78040BD93F77400CA9703C70700FD14F0
:101B5000398D2380A700E39334FF91BBA14763979E
:101B6000F90697000000E780A0C28144630D0B00D6
:101B70008D479304C0036308FB00930400056304CE
:101B80008B01930440041375C507E30295D21945F0
:101B900097000000E78000B697000000E780A0B63D
:101BA000054597000000E780E0B426859700000017
:101BB000E78020B7094597000000E78080B69700CE
:101BC0000000E780E0BCE31405CE0DB39147639FAE
:101BD000F9001305600697000000E780A0B19700A8
:101BE0000000E78040B213059009F9B5E38109CC04
:101BF000F1547DB9BD660147173600001306862EE5
:101C0000938606A685458347060093F7F70F91C391
:101C100082800507E3F9E6FE973700002384B72C9E
:101C2000DDB77D166206618693178601E18763D46E
:101C3000070001458280931726003307F500AE9711
:101C400018439C4363E7E7007D16E37FF7FC7D556F
:101C5000828005458280FD15E205E18513978501A7
:101C6000618793F7F50F63480700FD15139725006B
:101C70002A97584365D713851700620561858280CE
:101C80003308B5021C4283A80600B335B502C297DB
:101C900033B50701AE98469585486367B5006394F0
:101CA000A50063E3070181480C43C6950CC388C2B5
:101CB0001CC2828081471397870161876343B70005
:101CC0008280139727002A97232007008507E5B70E
:101CD0008147014793968701E18663C5B6001335B6
:101CE0001700828093962700AA9694428507558F05
:101CF000D5B793D755408A07AA979C430545331516
:101D0000B5007D8D828017F3FFDFE702833D2A84D3
:101D100097000000E78060F405C5931725003E9406
:101D20000327C4FF814711EB7D1516053E9542053B
:101D3000418517F3FFDF6700033D05838507E5B79E
:101D40000145C5BF81471397870161876343C7007A
:101D5000828013972700B386E50094422A9785076F
:101D600014C3D5B77D1662066186014793178601B5
:101D7000E18763D50700133517008280931726008B
:101D8000B306F500AE9794429C437D16B58F5D8FE8
:101D9000F1BF8A05AA9501476363B500828083A6D7
:101DA000C5FFF11593D71600D98F9CC11397F60183
:101DB000E5B72A830148014701456343D700828084
:101DC000B387050183A80700B30706019C43C697A4
:101DD000AA976384F80033B517010507B308030118
:101DE000620723A0F80061871108C1BF2A83014759
:101DF0008147014563C3D70082803388E50083288B
:101E00000800330EE600032E0E003388A840330886
:101E1000C8416384080133B508018507B308E300AE
:101E2000E20723A00801E1871107E9B717F3FFDFF5
:101E3000E702232B0111B286B2842E86AA850A8579
:101E400097000000E780C0FA2A84A6850A859700DB
:101E50000000E78020E833348000060413351500C5
:101E6000018D056117F3FFDF6700E32917F3FFDF3B
:101E7000E702A3244111AA89AE8A328BB68402C23A
:101E800002C402C60144131C8401135C8C416349E3
:101E90009C02939B1400FD1B0549138CF4FFF15C1D
:101EA00033048901620461846340740792478E049D
:101EB000CE9423AEF4FE410117F3FFDF67006323E6
:101EC00013192400B30B2B01014A93172A00D6974C
:101ED00083A50B0088437800340050009700000071
:101EE000E78040DA050A93178A01E187F11BE35E78
:101EF000FCFC92474E9905042320F900A2473EC2FC
:101F0000B24702C63EC441B7131A8901135A8A4127
:101F1000131D240093178A01E18763CF970092472E
:101F20000A044E941CC0A24705091379F90F3EC25A
:101F3000B24702C63EC4ADB7B3079A0313152A00D1
:101F400056950841780034005000050AEA97DA9760
:101F50008C4397000000E780E0D26DBF197106C284
:101F600012C416C61AC81ECA22CC26CE2AD02ED219
:101F700032D436D63AD83EDA42DC46DECAC0CEC2C9
:101F8000D2C4D6C6DAC8DECAE2CCE6CEEAD0EED2F9
:101F9000F2D4F6D6FAD8FEDA971500009385058CB0
:101FA0008841E700050092402242B2424243D243B8
:101FB0006244F244025592552256B2564257D257C5
:101FC0006258F25806499649264AB64A464BD64BBD
:101FD000664CF64C065D965D265EB65E465FD65F45
:101FE0000961730020300000972100209381810156
:101FF000175100201301018117F5FFFF1305C500DC
:102000009705002093850500171600201306C6FDCE
:1020100063FAC5008322050023A055001105910530
:10202000E3EAC5FE17050200130585DB97150020BE
:102030009385C5FB171600201306C66563FAC50015
:102040008322050023A0550011059105E3EAC5FE92
:1020500017150020130505649745002093858534E6
:102060006377B500232005001105E36DB5FEFD4241
:10207000739002BC8D4273904280B722000093821D
:10208000828873900230970200209382A2F793E235
:10209000320073905230974200009382627A7390BC
:1020A00012346FB0F47573002030397101436EC67D
:1020B00019A0397141536AC866CA62CC5ECE19A0B4
:1020C000397101535AD056D252D44ED64AD826DA54
:1020D00022DC06DE33016140828241114AC026C201
:1020E00022C406C68282B24D4101024D924C224C5E
:1020F000B24B4101024B924A224AB2494101024984
:1021000092442244B240410182803D432A87637356
:10211000C3029377F700BDEFADE5937606FF3D8AE6
:10212000BA960CC34CC30CC74CC74107E36BD7FE30
:1021300011E28280B306C3408A0697020000969699
:102140006780A6002307B700A306B7002306B700E1
:10215000A305B7002305B700A304B7002304B70005
:10216000A303B7002303B700A302B7002302B700FD
:10217000A301B7002301B700A300B7002300B700F5
:10218000828093F5F50F93968500D58D9396050182
:10219000D58D61B7939627009702000096968682A8
:1021A000E78086FA9680C1171D8F3E96E374C3F8C8
:1021B000A5B73367B500FD530D8B79E7B7877F7FF0
:1021C0009387F7F710419441B372F6003363F6003A
:1021D000BE92B3E262006397720C6318D606504158
:1021E000D441B372F6003363F600BE92B3E26200EC
:1021F0006398720A631BD60410459445B372F600C7
:102200003363F600BE92B3E262006391720A631E0A
:10221000D6025045D445B372F6003363F600BE9241
:10222000B3E26200639A72086311D60210499449BE
:10223000B372F6003363F600BE92B3E262006393BA
:1022400072085105D105E30FD6F6131706019397CF
:102250000601631CF7001357060193D706013305E7
:10226000F7409375F50F91E982804183C18333056F
:10227000F7409375F50F91E182801377F70F93F78D
:10228000F70F3305F74082800346050083C605003B
:10229000050585056313D60065FA3305D6408280AF
:1022A00011059105E312D6FE014582802105A105A5
:1022B000E31CD6FC014582803105B105E316D6FC4E
:1022C000014582804105C105E310D6FC01458280AD
:1022D000B717004003C777051377E70FA38BE70411
:1022E000130700F8A38DE7043D47238CE704130789
:1022F0005003A38CE70403C7A7051377D70F238DDB
:10230000E7048280B717004003C7E7020D89411137
:102310001377C70F498F93068008F3B6068093F6AC
:10232000860836C601000100930670052380D70495
:10233000930680FA2380D704010001002387E70277
:1023400023800704B247F3A7078001000100410181
:10235000828041112A83014E930E407E130F001993
:10236000930F400663E56E129308001913034006AD
:10237000B3781503854E0D4FA14F337365020D8958
:102380001335150063EFBE121308F6FF79467298F5
:102390004208135808013307C70213D61700BE07B7
:1023A00032976146B3F6C60213068070B386C60242
:1023B0003697A166F58F42075D8FB716004083C739
:1023C000F60293F70708A303F1000346710083C7E1
:1023D000F60293F70708E394C7FE83477100B71628
:1023E000004093F7F70F6388071293078008F3B74D
:1023F000078093F787083EC401000100B71700402B
:10240000930670052380D704930680FA2380D704AF
:102410000100010023AA070383C6170393E60608F9
:10242000A388D70223800704A247F3A707800100EF
:1024300001001166B71700407D16D45BC85F938515
:102440004703A98EF18EF5FA93068008F3B606804D
:1024500093F6860836C601000100930670052380B6
:10246000D704930680FA2380D7040100010098C1A5
:1024700003C7170313670704A388E7022380070431
:10248000B247F3A7078001000100410182807D135C
:102490003368E3039308E016630E08003368F30320
:1024A0009308D016630808009378330093B8180097
:1024B0009388D81633081E01131E0801135E0E01FF
:1024C00055B56393E5030548638608000148630337
:1024D00003002A8871087298FD15131E0801C205B1
:1024E000135E0E01C18179BD13F8150063F4BF00BE
:1024F0007908D5B713381800E5BF83C7F60293F7FC
:102500000708A303F1000346710083C7F60293F79F
:102510000708E394C7FE8347710093F7F70FF1DFD5
:10252000E9B531714AD966CB06DF22DD26DB4ED70D
:1025300052D556D35AD15ECF62CD6AC96EC7AA8C26
:1025400002D897100000E78020B12A8993078008FD
:10255000F3B7078093F787083EDA01000100B71749
:102560000040130770052380E704130780FA2380D7
:10257000E7040100010003C7F7021377770FA38771
:10258000E70203C7F70213678700A387E7022380E8
:102590000704D257F3A70780010001000545970003
:1025A0000000E78060D6130780C13347E902116A53
:1025B00093070AE893065002BD69930BA004814A71
:1025C000014B13048008930470057D1AB347F90288
:1025D0003307D7023EC0FD873ECC938709A69309F7
:1025E000803E3347F7023AC27D873AC43347390306
:1025F0008549B399990193D93940B306D702B30BF2
:102600007703B3C6F602B3CBFB0236C6FD8636C8E7
:1026100093D6FB4136CEB7460F0093860624334946
:10262000D9028566938606FAB3969601B389E902C4
:10263000130760553309D90293060010B389E902E4
:102640003349D902B3C9F9029316390036CA37198A
:102650000040FD8636D0930D090493D7F9413ED250
:10266000F336048093F6860836DC010001009307F8
:1026700070052380FD00930680FA2380DD000100B1
:1026800001008346390593F6860FA309D9048346D2
:10269000390593E61600A309D90423800D00E256FC
:1026A000F3A6068001000100130C80FA116DF336C9
:1026B000048093F6860836DE01000100930770055A
:1026C0002380FD0023808D01010001008346390530
:1026D000216693E60602A309D90483560905B3E6E9
:1026E000A6012318D90483560905D18E2318D904CD
:1026F00023800D00F256F3A60680010001008346F8
:10270000390593F606026381061A03463905218AC4
:102710006DDE081897100000E7800098733604807B
:1027200013768608B2C20100010023809D00238039
:102730008D0101000100B717004003C6370513766D
:10274000F60DA389C70403C6370513660602A389DD
:10275000C704835609052166B3E6A6012318D904E8
:1027600083560905D18E2318D90423800D0096467F
:10277000F3A60680010001008346390593F60602A0
:10278000638B061483463905A18AEDFE970000206D
:10279000E7806090AA8636D497000020E780A08F5B
:1027A000A256E30AD5FE835609054255B3E6A601B3
:1027B0002318D90497100000E780C08F834639059D
:1027C000A18AEDDE03560905834629058247337643
:1027D000CA00B306DA0293D5F641B296B388F64042
:1027E000E24733B8C6002E983308F840A247B3B684
:1027F00016013308D84063C70701631DF8009247EC
:1028000063FA1701C247634FF80E63950701B24799
:1028100063EAF80E894663E9660FF24693151800DD
:1028200013D3F8015E8613951800B365B30042D642
:1028300046D497C00100E78080C83258050B137B4F
:10284000FB0F63470001631A0838A25863870838F2
:1028500013081500B336A800B69513D6F5013298C3
:10286000B336C800AE9613581800FE06B3E606014C
:102870007336048013768608B2C6010001002380F7
:102880009D0023808D01010001000356C902B2960C
:10289000C206C1822316D90223800D00B646F3A6D4
:1028A00006800100010021B5F336048093F6860806
:1028B000B6C00100010023809D0023808D0101002E
:1028C00001008346390593E60602A309D904238053
:1028D0000D0086460DB5F336048093F68608B6C41F
:1028E0000100010023809D0023808D010100010073
:1028F0008346390593E60602A309D90423800D0017
:10290000A646BDB5E30B0BF0F336048093F68608BC
:10291000B6C801000100930680FA23809D00238041
:10292000DD00010001008346390593F5FC0F93F6A5
:10293000860FA309D90483463905CD8EA309D9048E
:1029400023800D00C646F3A6068001000100130592
:1029500080FA03463905930639051D8A631C9629BA
:102960007336048013768608B2CC0100010013068A
:1029700080FA23809D002380CD000100010003C662
:1029800006001376F60D2380C60003C60600136604
:1029900006022380C600835609051166D18E2318CE
:1029A000D904835609052166D18E2318D9042380C2
:1029B0000D00E646F3A6068001000100130680FA2A
:1029C0008346390593F60602638006268346390559
:1029D000130C3905A18AFDDA081897000000E7807A
:1029E000A06BF336048093F68608B6D00100010090
:1029F000930680FA23809D002380DD000100010002
:102A000083460C00116693F6F60D2300DC00834626
:102A10000C0093E606022300DC0083560905D18EE4
:102A20002318D904835609052166D18E2318D904A9
:102A300023800D008656F3A60680010001001306D0
:102A400080FA8346390593F60602638A0620834698
:102A50003905A18AEDFE97F0FF1FE780C0632A8C3D
:102A600097F0FF1FE7802063E30C85FF835609057D
:102A700011664255D18E2318D90497000000E780D3
:102A800060638346390513063905A18AFDDAF336FA
:102A9000048093F68608B6D401000100930680FAFC
:102AA00023809D002380DD00010001008346060095
:102AB00093F6F60D2300D60023800D00A656F3A64C
:102AC0000680010001008356090503462905D24707
:102AD000B376DA003306CA021305800C9355F6412B
:102AE0003696330DF6408257333CD6002E9C333653
:102AF000A601330CFC40330CCC40330885039256BE
:102B00004E86B335A5033305A503C29597C00100D2
:102B1000E780E09A63468001631E0C16630C0D1675
:102B2000130615003335A6002E959356F5013696FB
:102B3000B335D600AA959396F50105828585D18E89
:102B40006346B000639D051A638B061A0356C902DB
:102B500015823305D6003336C500B2956348B00000
:102B6000639105241306F00F637DA622894663F363
:102B7000561593078008F3B7078093F78708BED6EA
:102B80000100010037170040930770052300F70488
:102B9000930780FA2300F704010001008356C7025F
:102BA00089678117D58FC207C1832316F7022300D7
:102BB0000704B657F3A7078001000100FA506A54D2
:102BC000DA544A59BA592A5A9A5A0A5BFA4B6A4C49
:102BD000DA4C4A4DBA4D296182801308F5FF33352E
:102BE000A800FD152E951356F5013298B336C8008E
:102BF000AA9695B9F336048093F68608B6CA010002
:102C0000010023809D002380AD0001000100834668
:102C10003905CD8EA309D90423800D00D646F3A62D
:102C200006800100010035B3F336048093F6860870
:102C3000B6CE0100010023809D002380CD0001005D
:102C400001008346390593E60602A309D9042380CF
:102C50000D00F646F3A606800100010095B3F33699
:102C6000048093F68608B6D20100010023809D00FF
:102C70002380CD00010001008346390593E606025A
:102C8000A309D90423800D009656F3A606800100FF
:102C9000010045BB9306F5FF33B5A600FD152E9543
:102CA0009355F501AE96B3B5B600AA951396F50106
:102CB000858269B5F336048093F68608B6D801009C
:102CC0000100930680FA23809D002380DD0001002F
:102CD00001008356C9020566011693F6F60FD18EE0
:102CE000C206C1822316D90223800D00C656F3A660
:102CF000068001000100850A93FAFA0F95B233E6C7
:102D0000B60045C20356C9023305D0403338A0008F
:102D1000B305B040B385054115826345B000D1E1EC
:102D20006371A608894663F0560593078008F3B7D8
:102D3000078093F78708BEDA01000100B71700404B
:102D4000130770052380E704130780FA2380E70444
:102D50000100010003D7C7027D8B2396E702238081
:102D60000704D65781BDF336048093F68608B6DC97
:102D700001000100930680FA23809D002380DD007E
:102D8000010001008356C9020566011693F6F60F8D
:102D9000D18EC206C1822316D90223800D00E656C9
:102DA000B9B793078008F3B7078093F78708BEDEAB
:102DB0000100010037170040930770052300F70456
:102DC000930780FA2300F704010001000356C702AD
:102DD00093975600B297C207C1832316F7022300C8
:102DE0000704F657C1BB914763EEB70217D701003E
:102DF0001307070B8A05BA959C41BA978287B717C4
:102E0000004003A7470B1345F5FF698F23AAE70A84
:102E100003A7070B698F23A8E70A03A7070A798D81
:102E200023A0A70A8280B717004083A6470B134749
:102E3000F5FFF98E23AAD70A83A6070B558D23A881
:102E4000A70A83A6070A758F23A0E70A8280B7170F
:102E5000004003A7470B498F23AAE70A03A7070BE4
:102E60001345F5FF45BFB717004083A6470B13472F
:102E7000F5FF758F23AAE70A03A7070A598D4DB7F7
:102E8000B717004003A7470B498FEDB7914763EE93
:102E9000B70217D701001307E7018A05BA959C41CD
:102EA000BA978287B717004003A7470D1345F5FF70
:102EB000698F23AAE70C03A7070D698F23A8E70CE6
:102EC00003A7070C798D23A0A70C8280B7170040B9
:102ED00083A6470D1347F5FFF98E23AAD70C83A6C7
:102EE000070D558D23A8A70C83A6070C758F23A06B
:102EF000E70C8280B717004003A7470D498F23AA2C
:102F0000E70C03A7070D1345F5FF45BFB7170040B2
:102F100083A6470D1347F5FF758F23AAE70C03A778
:102F2000070C598D4DB7B717004003A7470D498FC0
:102F3000EDB7797122D43714004026D24AD0035914
:102F400024028354040206D64209C2044ECE52CC57
:102F500056CA13590901C1802DE11379F9F793F489
:102F6000F49F4209C20413590901C18093078008E4
:102F7000F3B7078093F787083EC401000100930769
:102F800070052300F404930780FA2300F404010081
:102F90000100231124032310940223000404A247F8
:102FA000F3A7078001000100B25022549254025945
:102FB000F249624AD24A45618280B7F507008146EC
:102FC0003000B105194597000020E7808081A247B5
:102FD00013972701E34A07FC1369090893E40440A7
:102FE00093098008F3B7098093F787083EC0010072
:102FF0000100930A700523005405130A80FA230088
:10300000440501000100231124032310940223002E
:1030100004048247F3A7078001000100294597F0C7
:10302000FF1FE7802031F3B9098093F989084EC268
:1030300001000100230054052300440501000100A4
:103040008357040293E707202310F40223000404AB
:103050009247B9B7B7170040884742054181937737
:10306000050491EB9377F5013755E80113050580C9
:103070003345F50282809377050C130700046397AC
:10308000E7009377F50137459C1CCDB72165130503
:1030900005D0828037E700E01C435443A183E20659
:1030A000D58F1CC1FD572320F7182322F7188280E3
:1030B00013178500B7E700E023A0E710618123A282
:1030C000A7108280B7F700E08847CC47828081470D
:1030D00037370040A14663C4C7003285828003456C
:1030E000B740E38EA6FE3385F5000345050085074E
:1030F0002304A740CDB797070020938727EF9C4371
:10310000173700201307072A3E95636EE50017372F
:1031100000201307273F6368A70017070020232715
:10312000A7EC3E858280FD57EDBF8280411122C40D
:1031300006C62A8497000000E78000F22947B307FB
:10314000E502B2408D83B3D7870222449507B3D7F7
:10315000E70237370040C207C1832316F700410159
:103160008280411137150E0006C697000000E780E7
:1031700020FCB7370040130770F82381E7000D47A4
:10318000A381E70013070004A380E7000547238716
:10319000E700B24041018280373700408347270073
:1031A0001A0593F7F703C98F93F7F70F2301F70079
:1031B0008280B737004003C7170019C9D98DA38093
:1031C000B70003C70700136787002380E7008280EA
:1031D00093C5F5FFF98DA380B7008280AE872A875B
:1031E000B736004021463738004089E71703000012
:1031F0006700E3F383C8B600E30916FF05078348B9
:10320000F7FFFD17C20723041801C183F9BF41115D
:1032100022C406C62A8497000000E780E0E329471D
:10322000B307E502B2408D83B3D7870222449507E6
:10323000B3D7E70237370040C207C1832316F740F0
:1032400041018280716541111305052006C6970072
:103250000000E78000FCB7370040130770F82381B7
:10326000E7400D47A381E74013070004A380E74030
:1032700005472387E740B24041018280CC4141119C
:1032800006C6328503C6150083C5050022064D8E8D
:1032900042068D654186138875A2630C0611634B47
:1032A000C804138845A26300060D634AC8009385CD
:1032B00035A26301B6082390060029464DA0138865
:1032C00055A26305060D938565A2E316B6FE8D45EE
:1032D0001D4663E6E5081146198E63F3C7003E8676
:1032E000B7E704002390C600FC4797D501009385FB
:1032F000A5BE9DA0138895A263030611634E060D1B
:103300001388A5A263000613938505A5E315B6FAF5
:1033100099451D4663E5E504198E63F3C7003E86B3
:10332000B7E704002390C600FC479705002093856B
:1033300025D61DA09D451D4663E3E5022146198E55
:1033400063F3C7003E86B7E70400FC472390C6003E
:103350009705002093858534BA9582970146B2403F
:10336000328541018280AD451D46E3EAE5FE3146E6
:10337000198E63F3C7003E86B7E704002390C600AA
:10338000FC4797D501009385A5B7F9B7B1451D4610
:10339000E3E7E5FC3546198E63F3C7003E86B7E7E1
:1033A00004002390C600FC4797D50100938545B6DD
:1033B00065B78D451D46E3E4E5FA1146198E63F3C2
:1033C000C7003E86B7E704002390C600FC4797D5A8
:1033D0000100938525B149B78D451D46E3E1E5F828
:1033E0001146198E63F3C7003E86B7E704002390A9
:1033F000C600FC4797D50100938545B3B1BFA545ED
:103400001D46E3EEE5F42946198E63F3C7003E86B8
:10341000B7E704002390C600FC4797D501009385C9
:1034200025AD1DBFB5451D46E3EBE5F23946198EC6
:1034300063F3C7003E86B7E704002390C600FC474D
:1034400097D50100938545A801BFB7E7040003A302
:103450000713970600209386A6C24146A545170587
:1034600000201305E5B802832D455DE703C505007F
:103470000947631FE50803A84500411106C6034735
:10348000180032850346080022074168518F9308CF
:1034900028FE6307170563E9E800051863030703BF
:1034A00023900600294591A8130648FE630AC70425
:1034B0001518E31707FF15463E87637BF60015478F
:1034C00001A8130600023E876374F600130700028A
:1034D000B7E704002390E600FC471316070111A884
:1034E0003E8691C30546B7E70400FC472390C6001B
:1034F0004206CC45418282970145B240410182801B
:10350000130600083E87E375F6FC13070008C9B7E9
:103510002390060005458280828041677917630405
:10352000E504411122C406C685472A84639FF5003D
:10353000B7E7040022852244B24003A3871397050E
:1035400000209385E52F4101028389476399F500A7
:10355000B7E7040083A7070B8545829771D9B2406E
:103560002244410182808280797126D252CCAE847D
:103570002A8A97D501009385659D17D5010013050B
:10358000659F06D63AC622D44AD0368432894ECEBA
:1035900097B00100E780E03DA28517D50100130533
:1035A000659E97B00100E780C03C294597B00100B7
:1035B000E780004183C7840093F70702F9E383C9DA
:1035C00004008947054532476396F908D44083C70C
:1035D000160083C60600A207D58FC166138616FEA5
:1035E000638CC7028D16638FD7068D6693862690EF
:1035F00029456391D706B7E70400A286225403A3A6
:103600004714B250F2494A86A6850259925452850F
:10361000624A8547456102832D450DEF93070002FD
:10362000354563E98702B7E70400FC47C844130641
:103630000002CA8582978149970700209387072156
:103640009C43014581CB9C4391C74E852286CA8508
:1036500082970145B250225492540259F249624A6B
:10366000456182802D457DF79307700F3545E3E373
:1036700087FEB7E70400FC47C8442286CA858297C4
:1036800065BF2145C1BF411122C437E4040083272F
:10369000841326C2AA84416506C697050020938537
:1036A000251A7D1582978327C40A17050000130584
:1036B00005E78588829795C0032304132244B2400E
:1036C000924497060020938626AE4146C5451705CD
:1036D00000201305659C41010283B24022449244BC
:1036E00001454101828019C59707002023A0A71634
:1036F00001458280454582801147636AA70A97D6B3
:103700000100938666830A0536951841411106C665
:103710003697AE87B2850287130700026145639D25
:10372000E700B7E70400FC47130600021705002076
:10373000130545F782970145B24041018280054754
:103740006145E39BE7FEB7E70400FC470546170524
:103750000020130525F7F9BF1307700F6145E39D9E
:10376000E7FCB7E70400FC471306700F17050020BD
:10377000130585F5C1B7130700086145E39EE7FA15
:10378000B7E70400FC4713060008170500201305DF
:1037900025034DB715476145E390E7FAB7E7040005
:1037A000FC471546170500201305C50961B70945F3
:1037B0008280411126C2B7E4040083A7C41322C447
:1037C0004AC006C62E8497050020938565072A897E
:1037D0008297058905C5970700209387E78B83D7D4
:1037E000A70BA28503A3440D2310F4002244B2408A
:1037F00092444A850249014641010283B240224473
:103800009244024949454101828097070020238163
:1038100007049707002023AF0702B717004003A74C
:10382000070CB706C0FFFD16758F23A0E70C03A792
:10383000070DB7064000558F23A8E70C03A7070C18
:103840003D9B23A0E70C03A7070D1367070123A8DF
:10385000E70C8280B717004003A5470C83A7470CED
:10386000598113451500C18B058999E3136525001E
:103870009707002083C7C7FD6380A7029707002032
:103880002388A7FC11C9970700209387A7FC03A3EF
:1038900007006303030002838280114517F3FFFFD3
:1038A000670063C8011122CC06CE3714004026CA37
:1038B0004AC84EC652C483447405034AB4058349BA
:1038C00084050349940597F0FFFFE780A0A0834794
:1038D000A40593F4F40F137AFA0F93E71700230D5E
:1038E000F40493F9F90F1379F90FB717004003C7E0
:1038F000A705058B6DFF03D5C705A38D4705238C51
:103900003705A38C2705A38B9704F2406244D24469
:103910004249B249224A05618280411193970501CB
:1039200022C406C626C2C1872E8463DC0700B7E422
:103930000400FC54829719C1BC5482972165218DE3
:1039400015A893F7150013C515008DE793F725000B
:103950009DC797000000E78020F0B7E70400BC4F48
:103960001306000A894517050020034525EF8297B5
:1039700013452400B240224492444101828093972F
:10398000250163D80702B7E4040083A7C41E829709
:1039900097000000E780A0F0BC4C375607001306E4
:1039A0000630896517050020034545EB82970965B8
:1039B00079B7939715010145E3DE07FA17C50100B2
:1039C0001305456497B00100E7808012B7E7040053
:1039D000BC4F13060064916517050020034505E8F8
:1039E00082971165A9BF1D71A2CC37E404005C5C0D
:1039F000485886CE494697C501009385255C829735
:103A000011E917C501001305A55C97B00100E78017
:103A1000200E01A0B7F600E0795798CAFD57DCCA1E
:103A20000567B7E700E023A0E7101306F00290C295
:103A300023A0E718010001003707002018471306EC
:103A4000000481459706002023A8E6E04157A38A99
:103A5000E7403C4408088297970700209387077C3B
:103A60003EC8856713870740938757D1231AE10023
:103A70002312F1021307B00F97F7FFFF9387C76474
:103A80002310E1023ED81547970700009387C7E14E
:103A9000B7F50700A30FE1003EDC054797070000DC
:103AA0009387E7DF81463000E10519452301E102F4
:103AB0003EDE97F0FF1FE780C0D218088147994685
:103AC00030003E960346060085070507A30BC70096
:103AD000E398D7FEC24791C70357410185676373D7
:103AE000F70001A0B7E7040083A7470A08088297F8
:103AF000AA8511C917C501001305C54E97B001006D
:103B0000E78020E701A0F6406644256182804111EC
:103B100026C2B7E4040083A7040806C622C417051A
:103B200000001305C5DF829717040020130404D397
:103B30002300A40097000000E780800297000000A7
:103B4000E780E0CC03450400224403A38405B2408F
:103B5000924413060032896541010283797106D6C9
:103B600022D413078008F337078093F787083EC2F3
:103B700001000100B7170040930570052380B704CA
:103B8000130680FA2380C7040100010083C6F702F0
:103B900093F6A60FA387D702238007049246F3A6C5
:103BA00006800100010073370780137787083AC445
:103BB000010001002380B7042380C7040100010035
:103BC00003C7F70213672700A387E70223800704D0
:103BD000A247F3A7078001000100054597E0FFFF1A
:103BE000E780807297000000E78060CB0147814644
:103BF0008147054685451305407E97E0FFFFE78036
:103C0000807537E404003C44680051468145829742
:103C1000B707C0A83EC8B787E803938707D03ECA56
:103C200097E7FF1F9387A7793EC67C586800829765
:103C3000B250225445618280411197D5010093858D
:103C4000A59E17C501001305E53206C697B0010011
:103C5000E78020D217D501001305C5B497B0010045
:103C6000E78020D1B2402945410117B30100670028
:103C700023D5411197D501009385459C17C50100B7
:103C80001305452F06C697B00100E78080CE17D5F3
:103C900001001305E5AF97B00100E78080CDB24089
:103CA0002945410117B30100670083D1411122C4A6
:103CB00006C6834705002A849DC797D501009385D2
:103CC000A59D17C501001305E52A97B00100E780FF
:103CD00040CA4C4017D50100130505C297B001003A
:103CE000E78020C93DA058410DEF97D5010093858D
:103CF000A59A17C501001305E52797B00100E780D5
:103D000040C717D501001305A5C097B00100E78093
:103D100040C62244B2402945410117B30100670063
:103D200023CAA1679386D7036313D70297D50100EF
:103D30009385859617C501001305C52397B001002B
:103D4000E78020C317D50100130585BD7DBFED07B2
:103D500097D501009385459417C50100130585216A
:103D6000631BF70097B00100E780A0C017D50100E2
:103D7000130545BC59BF97B00100E78080BF4C4098
:103D800017D50100130505BD91BF411197D501005D
:103D90009385058C17C501001305C51D06C697B090
:103DA0000100E78000BDB2402945410117B3010081
:103DB000670003C1797122D426D24AD02E842A8981
:103DC000B28481457146480006D697E0FFFFE78040
:103DD000003497F7FF1F9387275EDC4783D70700E0
:103DE000231421012313F10097500000E78020D510
:103DF0008547A305F1009307401F2305A1003EC698
:103E00002686FD57A2854800230AF100975000003E
:103E1000E780C0D5B2502254925402594561828045
:103E2000411197270020239E078E97170020238794
:103E3000077E06C6170700200347C72E9307F00A20
:103E40006315F7029307F0F889451705002013055D
:103E5000652D170700202307F72C97070020A38361
:103E6000072C97600000E780C08E97600000E78015
:103E700020BA97600000E78060BB814537050400E9
:103E80009707002023A607289707002023810728EB
:103E9000970700202390072097070020239E071CE8
:103EA00097070020239307269707002023940726CF
:103EB00097300000E7808020014597600000E78090
:103EC0004092D147170700202312F724B7E70400D8
:103ED000BC4F13060014894517050020034585983B
:103EE000829797C501009385257917C501001305B1
:103EF000650897B00100E780C0A79705002083D52B
:103F0000E52017D50100130525AB97B00100E78028
:103F100040A6B2402945410117B30100670043AAFA
:103F20004111814617F6FF1F1306464685451705C2
:103F300000200355251406C697C00000E780201511
:103F400015C997C501009385E57317C501001305D1
:103F5000650297B00100E780C0A117D501001305E5
:103F6000A59597B00100E780C0A0294597B0010052
:103F7000E78000A597C501009385C57017C50100AE
:103F8000130545FF97B00100E780A09E17D50100FB
:103F90001305C59397B00100E780A09D294597B010
:103FA0000100E780E0A197F7FF1F9387E740DC4718
:103FB000054797C501009385E56C2390E70017C579
:103FC0000100130525FB97B00100E780809A17D503
:103FD00001001305E59097B00100E7808099B24099
:103FE0002945410117B301006700839D011122CCCF
:103FF00006CE26CA4AC84EC693F715002E84B5CB06
:1040000097000000E78000F2930710F817070020E0
:10401000230AF7109707002083D78705170700208A
:10402000A302F7109145A183170500201305850F02
:10403000170700202309F70E97070020A385070E16
:1040400097500000E780E070B7E70400BC4F13060C
:10405000001493050010170500200345A5808297E2
:1040600013451400F2406244D2444249B24905610A
:10407000828093F70510B1C3054597500000E78093
:104080004076171500200355C56997500000E7805A
:10409000C04197200000E780E0229707002083C7F7
:1040A000B71789E797600000E78080969760000067
:1040B000E780C0971345041075B793F72500E9CF43
:1040C000170700200357870469C7AD64B71900407C
:1040D0009384A4AA23A09900970600209386460300
:1040E000944297D701009387E78E17060020034676
:1040F0000602814517D501001305C58E9770000093
:10410000E780A01423A0990097F7FF1F239AA71A0E
:104110002A8941C197C501009385855D17C50100B6
:10412000130545E597B00100E780A084CA8517C54F
:1041300001001305E5FB97B00100E7808083294566
:1041400097B00100E780C08797070020239007FC05
:10415000930710F8170700202306F7FC97070020A5
:1041600083D707F117070020A30EF7FAA1831707DB
:104170000020230AF7FA91458D4717050020130503
:1041800065FA17070020A300F7FA97500000E780B0
:10419000405C13452400F9B593F74500D1C397C59A
:1041A00001009385E55417C501001305A5DC97A010
:1041B0000100E780007C17C50100130525F597A0D5
:1041C0000100E780007B294597A00100E780407F40
:1041D000930720F8170700202306F7F4970700201D
:1041E00083D747EB17070020A30EF7F2A183170729
:1041F0000020230AF7F2854717070020A305F7F2EE
:1042000097500000E780A0AA17050020130585F14C
:10421000914597500000E780C0531345440099B57D
:1042200093F78500A9C797C501009385654C17C50D
:104230000100130525D497A00100E780807317C5FE
:1042400001001305E5ED97A00100E7808072294584
:1042500097A00100E780C07697070020239807EA1F
:1042600097700000E780400E13458400E5BB93F78C
:104270000501D1C38545170500200355A5E19760C9
:104280000100E78000C497C501009385654617C506
:104290000100130525CE97A00100E780806D17C5AA
:1042A0000100130525E997A00100E780806C2945EE
:1042B00097A00100E780C070930730F8170700202F
:1042C0002302F7E69707002083D7C7DC17070020F3
:1042D000A30AF7E4170500201305C5E4A1838D4563
:1042E000170700202301F7E497500000E78060469D
:1042F0001345040185BB93F70502D1C797C501009B
:104300009385053F17C501001305C5C697A0010099
:10431000E780206617C50100130505E497A001009A
:10432000E7802065294597A00100E7806069930731
:1043300040F8170700202307F7DE9707002083D7F0
:10434000A7D317070020A30FF7DCA18317070020CE
:10435000230BF7DC854717070020A306F7DC970738
:104360000020239B07D097500000E780409417055A
:104370000020130525DB914597500000E780603D44
:1043800013450402C5B193F70504FDC397C50100A9
:104390009385053617C501001305C5BD97A001001B
:1043A000E780205D17C50100130585DC97A001009B
:1043B000E780205C294597A00100E78060609707AF
:1043C000002083C727D61307700A6386E706130702
:1043D000800A638CE7081307600A6393E704930776
:1043E00060F817070020230FF7D29707002083D724
:1043F000C7D117070020A307F7D2A1831707002012
:104400002303F7D2854717070020A302F7D2B1454F
:1044100017050020130505D197500000E780603391
:1044200097500000E780A0881345040497070020F8
:10443000239D07CC05B9930770F8170700202303C5
:10444000F7CE9707002083D747CC17070020A30B90
:10445000F7CCA183170700202307F7CC8547170760
:104460000020A303F7CC994565B7930780F8F1B70F
:1044700093F705080145E38707BE97C501009385BB
:10448000252717C501001305E5AE97A00100E780B9
:10449000404E17C50100130525CF97A00100E78006
:1044A000404D294597A00100E78080519307A0F86F
:1044B000170700202308F7C69707002083D787C572
:1044C00017070020A300F7C6A18317070020230CBD
:1044D000F7C4854717070020A307F7C497070020F4
:1044E000239A07C297400000E780607C17050020F0
:1044F000130545C3914597500000E780802513457B
:1045000004088DB6411122C497C501009385051A90
:104510002A8417C501001305E5A506C697A001006A
:10452000E78020454C4017C501001305653697A06C
:104530000100E7800044294597A00100E78040483A
:10454000034704009307F00F631FF70297C50100AC
:104550009385C51517C501001305C5A197A00100D6
:10456000E78020414C4017C501001305653397A033
:104570000100E78000402244B2402945410117A3D1
:1045800001006700E343B2402244410182804111AF
:1045900022C426C22A84AE8417C501001305859D56
:1045A00097C501009385450C06C697A00100E780DA
:1045B000403C17C501001305A53E97A00100E78008
:1045C000403B294597A00100E780803F97C5010047
:1045D0009385850997070020239E87A817C50100AA
:1045E00013054599054497070020239397A897073B
:1045F0000020239087A8971700202394971297A054
:104600000100E78000379715002083D5851117C575
:1046100001001305653997A00100E7808035294521
:1046200097A00100E780C03997170020238887FEF4
:1046300097F7FF1F938747D8DC4717F5FF1F034500
:10464000652203D70700C167FD17631EF700B7E7B0
:10465000040003A387051306000A85452244B240DF
:10466000924441010283B7E7040003A387051306C0
:10467000001493050010DDB7B1C1411122C417C564
:1046800001001305258F2E8497C50100938505FD34
:1046900006C697A00100E780C02DA28517C50100BE
:1046A0001305452F97A00100E780A02C2244B240BB
:1046B0002945410117A30100670083308280011161
:1046C00022CC37E404005C5C06CE26CA354697C58A
:1046D00001009385650E17D50100130525D6829735
:1046E00011E917C501001305A58E97A00100E78009
:1046F000204001A097F7FF1F938787173EC4B7F5A7
:104700000700856793870780814617F6FF1F13060A
:10471000A615E10519453EC697E0FF1FE780600C2E
:104720007C44194697F5FF1F938505141705002053
:10473000130585968297340017F6FF1F1306C612DD
:1047400097C501009385455217C5010013054553D0
:1047500097700000E7806084AA8421C197C501009A
:10476000938505F817C501001305C58097A00100C2
:10477000E7802020A68517C501001305E50497A052
:104780000100E780001F294597A00100E780402332
:10479000F2406244D2440561828097E00000E780E5
:1047A00040EA17C50100130525F997500000E7807E
:1047B000807897A00000E780803E97600100E78046
:1047C00000A317F5FF1F1305A5BB97600100E78045
:1047D000A08B17C50100130525F797600100E7803E
:1047E00080A3AA8497600000E780C0DE97000100E4
:1047F000E780E07A97800100E7800014977000005E
:10480000E780A03A97600000E780C054973001002D
:10481000E780403C97C50100938585EC17B5010002
:104820001305457599C897A00100E7808014A685F7
:1048300017C50100130585FB99B797A00100E78014
:10484000401317C501001305A5FC97A00100E780E0
:104850004012294597A00100E7808016973001009B
:10486000E780201897F00000E780E0366DC58545A9
:104870003705040097300000E780408497C50100A9
:10488000938505E617B501001305C56E97A00100D5
:10489000E780200E17C50100130505F997A0010058
:1048A000E780200D294597A00100E780601197F768
:1048B000FF1F9387E79F83D7070017170020231256
:1048C000F7E6854717170020230AF7D497F7FF1F4D
:1048D000938787AEDC4703D70700C167FD176316D0
:1048E000F70097F0FFFFE780E06397700000E78034
:1048F000E0B58567938707E33E9597700000E780F2
:10490000A0B597200000E780E09B17150020035515
:1049100045E197500000E78040B9054597500000F9
:10492000E78020EC97500000E780401097C5010019
:10493000938505DB17B501001305C56397A001003A
:10494000E780200317C50100130545F397A0010078
:10495000E78020020DBDD14797C50100938545D85A
:1049600017B501001305056117F7FF1F2310F77A2C
:1049700097A00100E780E0FF17C60100130606EDCF
:1049800097F5FF1F83D5857817C50100130545EC02
:1049900097A00100E780E0FD294597A00100E7808E
:1049A00020023C4C1306000A894517F5FF1F0345FA
:1049B00065EB8297014597500000E78080E2BDB724
:1049C000411122C437E404008327041A06C68297E3
:1049D00097500000E78020B18327040817F5FFFFF8
:1049E00013050561829797F7FF1F238DA7E617F53B
:1049F000FF1F1305659C97400000E780006222447A
:104A0000B2404101170300006700A3CBB7E70400E1
:104A1000FC471171A2DDCAD986DFA6DBCED72E8472
:104A200032892E86AA8517F5FF1F1305A56F829779
:104A300017F7FF1F1307076F8347070093068002CE
:104A40009387E70793F7F70FE3ECF610BA898A0725
:104A500017B701001307475BBA979C43BA97828741
:104A60008D4797C501009385E5C917B5010013056A
:104A70006550630FF40097A00100E78080EF17C531
:104A800001001305E58697A00100E78080EEBDA434
:104A900097A00100E780E0ED17C501001305C5866A
:104AA00097A00100E780E0EC294597A00100E7808E
:104AB00020F1930720F8114697F5FF1F938585662F
:104AC0004A8517F7FF1F230FF76497F7FF1FA38C83
:104AD000076497F0FFFFE780202E2A841DC997C541
:104AE0000100938525C217B501001305A54897A0BD
:104AF0000100E78000E8A28517C501001305858441
:104B000097A00100E780E0E6294597A00100E78033
:104B100020EB97C501009385E5BE17B5010013058D
:104B2000654597A00100E780C0E417C501001305A3
:104B3000A58297A00100E780C0E3294597A0010066
:104B4000E78000E84165930730FA054697F5FF1FB7
:104B50009385455D7D1517F7FF1F2305F75C97F0DB
:104B6000FFFFE78060252A841DC997C50100938552
:104B700065B917B501001305E53F97A00100E7806F
:104B800040DFA28517B501001305C57B97A0010082
:104B9000E78020DE294597A00100E78060E2B7E7C3
:104BA0000400BC4F0566130606C8A14517F5FF1F94
:104BB000034545CB8297FE506E54DE544E59BE5984
:104BC0001161828091476303F40297C501009385C8
:104BD00065B317B501001305E53997A00100E7801B
:104BE00040D917B501001305657A71BDB7E7040018
:104BF000FC4F914517F5FF1F0345C5C6829797C522
:104C00000100938525B017B501001305A53697A0BF
:104C10000100E78000D617B501001305E57897A0DD
:104C20000100E78000D5294597A00100E78040D921
:104C300097400000E780A007914535A485476303AE
:104C4000F40297C501009385E5AB17B50100130584
:104C5000653297A00100E780C0D117B501001305A8
:104C6000257615B597F7FF1F23962743B7E704006E
:104C70000566BC4F130606C8C1450DBF8D476303CB
:104C8000F40297C501009385E5A717B50100130548
:104C9000652E97A00100E780C0CD17B50100130570
:104CA000E573D5B3930740F8114697F5FF1F938539
:104CB00065474A8517F7FF1F2306F74697F7FF1F3B
:104CC000A383074697F0FFFFE780000F2A84E304E1
:104CD00005EE97C501009385E5A217B50100130500
:104CE000652997A00100E780C0C8A28517B501001B
:104CF0001305456597A00100E780A0C7294597A047
:104D00000100E780E0CB45BD9147E31CF4F6B7E72F
:104D10000400FC4F9305000217F5FF1F034585B4FF
:104D2000829797C501009385E59D17B5010013058E
:104D3000652497A00100E780C0C317B501001305E3
:104D4000656BF1BD894763E3870297C501009385D1
:104D5000659B17B501001305E52197A00100E780C9
:104D600040C117B501001305256A31BB97F4FF1F39
:104D700083C4643B97F7FF1F83C7D73A97C50100E9
:104D800093854598A20417B501001305A51EDD8C77
:104D900097A00100E780E0BDA28517B501001305CB
:104DA000E56797A00100E780C0BCC204294597A031
:104DB0000100E780E0C0C1849305D4FF939604010D
:104DC000C1824A8693F5F50F17F5FF1F1305B53518
:104DD00097200000E7804032E35F90DC930750F8B3
:104DE00017F7FF1F2300F73483C73900228697F592
:104DF000FF1F9385253385074A8517F7FF1FA304F7
:104E0000F73297F0FFFFE78020FB2A84E30505DAFD
:104E100097C501009385058F17B50100130585150A
:104E200097A00100E780E0B4A28517C50100130533
:104E300065B5C9B5894763E3870297C501009385C6
:104E4000658C17B501001305E51297A00100E780F6
:104E500040B217B501001305255E35B1974000003B
:104E6000E780E0E4A28517F5FF1F1305A52B9750F7
:104E70000000E780008E81B38D476303F40297C57D
:104E800001009385258817B501001305A50E97A08D
:104E90000100E78000AE17B501001305A55BE5B67C
:104EA000B76602000146B7750200054597E0FF1F8F
:104EB000E7802093930760F817F7FF1F2304F72676
:104EC00097F7FF1FA38107269307000617F7FF1F19
:104ED000230CF724894717F7FF1FA307F72497F739
:104EE000FF1F2384072497F7FF1FA3800724C147D0
:104EF00017F7FF1F230CF722930720F917F7FF1F5F
:104F0000A306F722314697F7FF1FA382A72297F542
:104F1000FF1F938525214A8597F7FF1F23890720C7
:104F200097F0FFFFE78040E92A84E30605C897B5BC
:104F300001009385257D17B501001305A50397A0F2
:104F40000100E78000A3A28517B5010013050552F3
:104F500055B3B1476303F40297B501009385857A91
:104F600017B501001305050197A00100E78060A0B7
:104F700017B501001305455139B6B7E70400FC4FDA
:104F80009305000417F5FF1F0345C58D82979740D1
:104F90000000E780C0D1B145F9B5914763E38702CE
:104FA00097B501009385057617B50100130585FCBB
:104FB00097A00100E780E09B17B501001305854E1F
:104FC000D9B497F4FF1F83C4241697F7FF1F83C734
:104FD0009715A204DD8C8E04B77702006D14BE9481
:104FE0002286A68517B501001305054D97A001007F
:104FF000E7802098B7E70400FC47228697F5FF1F5B
:10500000938595122800829793160401C18230007F
:10501000A685094597D0FF1FE780A07C2A8409C98F
:1050200017B501001305054B97A00100E78040ACC0
:10503000930770F8194697F5FF1F9385A50E4A85CB
:1050400017F7FF1F2300F70E97F7FF1FA38E870C9C
:1050500097F0FFFFE78040D62A84E30E05B497B5AA
:1050600001009385256A17B501001305A5F097A0E7
:105070000100E7800090A28517B501001305854661
:1050800095B99947630BF41297B50100938585672D
:1050900017B50100130505EE97A00100E780608DAC
:1050A00017B5010013058545F9BA914763E38702F7
:1050B00097B501009385056517B50100130585EBCC
:1050C00097A00100E780E08A17B501001305854429
:1050D0005DBA97F4FF1F83C4240597F7FF1F83C7AA
:1050E0009704A204DD8C8E04B77702006D14BE9481
:1050F0002286A68517B501001305054397A0010078
:10510000E7802087B7E70400FC47228697F5FF1F5A
:10511000938595012800829793160401C18230007F
:10512000A6850D4597D0FF1FE780A06B2A8409C98B
:1051300017B501001305054197A00100E780409BCA
:10514000930780F8194697F5FF1F9385A5FD4A85BB
:1051500017F7FF1F2308F7FC97F7FF1FA38687FCAD
:1051600097F0FFFFE78040C52A84E30605A497B5C2
:1051700001009385255917B501001305A5DF979008
:105180000100E780007FA28517B501001305C53C2B
:1051900095B699476303F40297B501009385855648
:1051A00017B50100130505DD97900100E780607CCD
:1051B00017B501001305C53BF9B0B7E70400FC4F74
:1051C0009305000417E5FF1F0345C56982979740C3
:1051D0000000E780C0AD994579B18D476303F402C3
:1051E00097B501009385055217B50100130585D8C1
:1051F00097900100E780E07717B501001305C538E7
:1052000059B017B501001305253997A00100E780B3
:10521000208E1305C01297D0FF1FE7808012014532
:1052200097E0FFFFE78040E70D4597100000E7801B
:10523000A09E294597D0FF1FE780A01097D0FF1FA1
:10524000E78000018DBA99476303F40297B5010026
:105250009385454B17B501001305C5D19790010003
:10526000E780207117B501001305C53329B817F77A
:10527000FF1F034777EB97F7FF1F83C7E7EA220774
:105280005D8F9166BA96C2061166C1821306F6EF6B
:105290008D476365D60297E7FF1F9387E7119C4B05
:1052A00017F6FF1F034636E89386C7002DC203D6C4
:1052B000070069CA8907E39CD7FE89471307A0F84E
:1052C000114697F5FF1F9385E5E54A8597F6FF1F81
:1052D000238AE6E417F7FF1FA307F7E497F0FFFF21
:1052E000E78080AD2A84E308058C97B5010093859B
:1052F000654117B501001305E5C797900100E780E8
:105300004067A28517B501001305052BE5B203D64A
:105310000700630EE60A8907E39BF6FE8D4779BF17
:1053200091476304F40297B501009385A53D17B535
:105330000100130525C497900100E780806317B52D
:1053400001001305E5286FF00FF4B7E70400FC4FE8
:105350009305000817E5FF1F0345C5508297C9B89C
:1053600097B501009385053A17B50100130585C06F
:1053700097900100E780E05F17B501001305C5268F
:105380006FF06FF02390E70017E5FF1F1305C502CC
:1053900097300100E780608A97B5010093858536D4
:1053A00017B50100130505BD97900100E780605C0B
:1053B00017B501001305452497900100E780605B55
:1053C000294597900100E780A05F8147C5BD2390E4
:1053D000070017E5FF1F130525FE97300100E78042
:1053E000C08597B501009385E53117B50100130518
:1053F00065B897900100E780C05717B50100130505
:1054000025215DBF011122CC06CE26CA4AC883479A
:1054100005002A849DC797B501009385652A17B5B5
:105420000100130525B597900100E78080544C409A
:1054300017B501001305055C97900100E7806053E4
:10544000D1A05841B707CF009387777D631BF7063C
:105450000359C500854704450356E50063FA270351
:1054600083C7040003C71400A207D98FC20771774E
:10547000C1871307C755639DE7006244F240CA85A0
:1054800026854249D2440561171300006700A373C3
:105490009707002083D7E728638AC700CA85268537
:1054A00032C697E0FFFFE780A0D332466244F24065
:1054B000CA8526854249D244056117F3FFFF67007C
:1054C0002355B707CC009387777D6317F70497B50B
:1054D00001009385E51E17B501001305A5A9979056
:1054E0000100E78000491C448356E4008355C40052
:1054F00003C6070017B50100130545519790010039
:10550000E78020476244F240D24442492945056180
:10551000179301006700C34AB707CE009387777DD2
:105520006304F70297B501009385851917B501004B
:10553000130545A497900100E780A0434C4017B5A0
:10554000010013052541CDBDF2406244D2444249D9
:1055500005618280B7E70400FC4741112E8606C62C
:1055600022C426C24AC02E842A89AA8517F5FF1FA5
:10557000130545BB829797B501009385651A17B54A
:1055800001001305259F97900100E780803E97F565
:10559000FF1F83C525B917B50100130565C0979096
:1055A0000100E780003D294597900100E7804041D8
:1055B00097F4FF1F938404B783C704004147938780
:1055C000070693F7F70F6369F75A17B70100130738
:1055D000E7AD8A07BA979C43BA9782879D476307CE
:1055E000F40297B501009385A51317B501001305C3
:1055F000659897900100E780C03717B50100130543
:10560000A5BA97900100E780C036A1AC97F7FF1FBD
:1056100083C757B1DDCB17F7FF1F0347D7B097F705
:10562000FF1F83C747B022075D8F97F7FF1F83C710
:10563000A7AFC2075D8F97F7FF1F83C7F7AEE207DB
:10564000D98F17F7FF1F2325F7AC83C7640097B5E1
:1056500001009385E50C17B501001305A59117F717
:10566000FF1F2306F7AA97900100E780803097F785
:10567000FF1F9387E7A98C4317F6FF1F034626A950
:1056800017B50100130505B497900100E780602E5F
:10569000294597900100E780A03297F7FF1FA38369
:1056A00007A82244B24092440249930700F817F732
:1056B000FF1F2309F7A69D4517F5FF1F130585A6B4
:1056C0004101174300006700C30897600000E780AE
:1056D00020D797F7FF1F2388A7A49357850017F7B4
:1056E000FF1FA302F7A4935705012A8417F7FF1F92
:1056F000230CF7A293578501014517F7FF1FA30558
:10570000F7A297600000E78000D897F7FF1F238E6D
:10571000A7A097B501009385A50017B50100130553
:10572000658597900100E780C02417F6FF1F0346A8
:10573000C69FA28517B50100130545AAB1B7CD478D
:105740006303F40297B50100938585FD17B5010049
:105750001305458297900100E780A02117B501004D
:10576000130545A979BD97F7FF1F83C7C79CA207FB
:1057700017F7FF1F0347179CD98FC207C1876357CD
:10578000F00217F7FF1F2313F798B7E7040003A3EE
:1057900087051306000A89452244B2409244024913
:1057A00017E5FF1F0345050C41010283D147D1BF17
:1057B0008D476303F40297B50100938565F617A53D
:1057C00001001305257B97900100E780801A17B52B
:1057D00001001305E5B135B517F4FF1F0344A49488
:1057E00097F7FF1F83C7179497B50100938545F37B
:1057F000220417A501001305E5775D8C9790010041
:10580000E7802017A28517B50100130525A0979002
:105810000100E7800016294597900100E780401AB3
:105820000D4697F5FF1F9385E58F228597E0FFFFD3
:10583000E7808058AA8421C197B50100938545EE81
:1058400017A501001305057397900100E78060120A
:10585000A68517B501001305A59C97900100E78068
:1058600040112244B2409244024929454101179314
:1058700001006700E31497F7FF1F239D8780B7E7B8
:105880000400116603A38705130606E8914529B7AE
:105890008D476303F40297B50100938565E817A56A
:1058A00001001305256D97900100E780800C17B566
:1058B00001001305A5B2B1B317F4FF1F0344A4867A
:1058C00097F7FF1F83C7178697B50100938545E5B6
:1058D000220417A501001305E5695D8C979001006E
:1058E000E7802009A28517B501001305A5949790BC
:1058F0000100E7800008294597900100E780400CEF
:105900000D4697F5FF1F9385E581228597E0FFFF00
:10591000E780804AAA841DC197B50100938545E0C0
:1059200017A501001305056597900100E780600445
:10593000A68517B501001305259105B797E7FF1F49
:10594000239C8772B7E70400116603A3870513063B
:1059500006E89305000289B5894763E3870297B596
:1059600001009385E5DB17A501001305A56097905D
:105970000100E780000017B501001305E5A851B14B
:1059800097E4FF1F83C4247A97E7FF1F83C79779A3
:1059900097B501009385C5D8A20417A5010013058A
:1059A000655DDD8C97900100E780A0FCA68517B5AA
:1059B00001001305E58A97900100E78080FB2945E7
:1059C00097900100E780C0FF228697E5FF1F93852F
:1059D0006575268597E0FFFFE780003E2A84630E09
:1059E000051A97B501009385A5D317A501001305E6
:1059F000655897900100E780C0F7A28517B50100B0
:105A00001305458799BD854763F9871883451900B4
:105A10002244B24092440249B335B00097E7FF1FD9
:105A20002384B76817B50100130505864101179354
:105A30000100670003F4A2852244B24092444A85E3
:105A4000024941011703000067004323994763039C
:105A5000F40297B501009385A5CC17A501001305A5
:105A6000655197900100E780C0F017B5010013055C
:105A700065B341BE17E4FF1F0344E46A97E7FF1FC5
:105A800083C7576A97B50100938585C9220417A576
:105A900001001305254E5D8C97900100E78060EDB5
:105AA000A28517A501001305A57F97900100E78047
:105AB00040EC294597900100E78080F0194697E572
:105AC000FF1F93852566228597E0FFFFE780C02EA4
:105AD000AA841DC197B50100938585C417A501004F
:105AE0001305454997900100E780A0E8A68517A512
:105AF00001001305E57B95B397E7FF1F239C8760A3
:105B0000B7E70400116603A38705130606E89305AB
:105B1000000859B1854797B50100938565C017A561
:105B2000010013052545630BF40097900100E78001
:105B300040E417A501001305E578E1B49790010052
:105B4000E78020E317A50100130545799790010030
:105B5000E78020E2294597900100E78060E6224433
:105B6000B2409244024997E7FF1F2391075A41012F
:105B7000175300006700437D97B50100938545BA30
:105B800017A501001305053F97900100E78060DE2F
:105B900017B50100130545A5ADB4B24022449244A7
:105BA000024941018280411106C622C426C239C180
:105BB0002A8497E00000E7800002AA8411EDB7E78D
:105BC0000400BC474146814522858297B240224469
:105BD000268592444101828041657D1597E0000051
:105BE000E7804000B7E7040001E9BC474146814532
:105BF000228582978144D9BF0347E501FC4793057D
:105C0000900819E393050003AA95414622858297DF
:105C100085446DBF411122C491462A8417E6FF1FB7
:105C20001306465E9D652D4506C697D0FF1FE7808B
:105C300040BBB7F7070003C70701A5476313F70089
:105C400001A09306001001469D65254597D0FF1FD2
:105C5000E78020B997E7FF1F2386875A2244B24086
:105C6000914617E6FF1F1306E6599D652945410138
:105C700017D3FF1F6700E3B61171CED7B7E9040051
:105C800083A7C904CAD917E9FF1F1309A949A2DDCF
:105C90002E8686DFA6DB2E84AA854A85829797E723
:105CA000FF1F83C727481307700A6385E710636DDA
:105CB000F7001307600A6385E704FE506E54DE5454
:105CC0004E59BE59116182801307800A6385E71619
:105CD0001307900AE393E7FE8D476306F41C97B51C
:105CE0000100938525DE17A501001305A5289790CF
:105CF0000100E78000C817B501001305E5D925A00C
:105D00008D47630CF40297B501009385A5DB17A5B9
:105D100001001305252697900100E78080C517B57F
:105D200001001305A5D097900100E78080C42945A4
:105D300097900100E780C0C849B7854717B50100B3
:105D4000130585D017E7FF1F2300F7369790010052
:105D5000E78000DAB7750200B76602000146054524
:105D600097D0FF1FE780E0A7930760F817E7FF1FB2
:105D7000230AF73A97E7FF1FA387073A93070026FE
:105D800017E7FF1F2322F73AE5779387072117E7E5
:105D9000FF1F231DF738B14597E7FF1F23890738F9
:105DA00097E7FF1FA385A7384A8597000000E78083
:105DB000E01621B7914763E3870297B50100938509
:105DC00065D017A501001305E51A97900100E7803B
:105DD00040BA17B50100130525C9B1B797E4FF1FF5
:105DE00083C4843497E7FF1F83C7F733A204DD8C95
:105DF00083A7C9046D14228697E5FF1F9385D532CA
:105E0000280082978E0493160401B7750200C182A0
:105E10003000A695094597D0FF1FE780809C930727
:105E200070F817E7FF1F230FF72E994597E7FF1F1D
:105E3000A38CA72E95BF914763E3870297B5010016
:105E4000938545C817A501001305C5129790010059
:105E5000E78020B217B50100130585C2E9B597E4C4
:105E6000FF1F83C4642C97E7FF1F83C7D72BA204AF
:105E7000DD8C83A7C9046D14228697E5FF1F9385E7
:105E8000B52A280082978E0493160401B775020084
:105E9000C1823000A6950D4597D0FF1FE780609422
:105EA000930780F8BDBF17B50100130525C0979073
:105EB0000100E780E0C3930790F82304F1008347D3
:105EC00019008D452800A304F1008347290023050C
:105ED000F10097000000E78060041305C01297C02E
:105EE000FF1FE7800046014597D0FFFFE780C01AFB
:105EF0000D4597000000E78020D2294597C0FF1F7D
:105F0000E780204497C0FF1FE78080347DB397E788
:105F1000FF1F23A1A730828097E7FF1F9387872F5A
:105F200003A3070063030300028317430000670015
:105F3000438241114AC097F6FF1F83D6867E32897D
:105F400017D6FF1F0356664922C426C206C62A84F6
:105F5000AE8497000000E780204C29C921C89947EA
:105F600063F697048347140003470400A207D98F00
:105F700013978700A183D98FC2073167C1831307A5
:105F8000C7556395E70297D7FF1F83D70745A3013E
:105F9000F400A1832302F40097F7FF1F83D76778EB
:105FA00091C7A302F400A1832303F400630D090247
:105FB00097F7FF1F83C787669DE797E7FF1F83C794
:105FC000A72595C38DC097E7FF1F83C7E70D81EF16
:105FD00022852244B2400249A685924441011733EA
:105FE000000067000377B240224492440249410115
:105FF0008280834755008345450017B5010013058E
:1060000025AFA207DD8D179301006700839617B5B2
:1060100001001305E5AC17930100670063AD8D47E0
:1060200063F6B708011126CA06CE22CC0344350018
:1060300097E4FF1F83C4541E97B50100938585AC78
:10604000B337800017E7FF1FA308F71C09C497B5F3
:1060500001009385E5AB17B501001305E5AB9790FB
:106060000100E780009197E7FF1F83C7F71A638657
:10607000970097000000E780002997400000E78024
:10608000E09A9967938757EE2316F10068008547D9
:106090009145A30781002307F10097000000E780E6
:1060A000E0E7F2406244D244056182808280894701
:1060B00063F7B708011122CC06CE26CA8344250017
:1060C00085472A84639DF404914763F5B70403452B
:1060D00045008347340022055D8D97D7FF1F239E1F
:1060E000A72E97000000E780003C9967938767EE32
:1060F0002314F1008347340023059100A305F10028
:1061000083474400954528002306F10097000000CE
:10611000E780C0E0F2406244D24405618280FDF82D
:106120009967938767EE2314F10097D7FF1F83D7F2
:10613000C72AA305F10023050100A183E1B78280EE
:106140000111996722CCD51717F4FF1F1304044DD2
:106150002314F1008347040026CA97F4FF1F938499
:10616000445C2305F10083D7040028009545A3056E
:10617000F100A18306CE2306F10097000000E7801E
:10618000E0D903D604008345040017B501001305C8
:10619000A59997800100E780C07DF2406244D24417
:1061A000056182809D677971D9172316F10097F7F1
:1061B000FF1F9387A74683C707001305F10006D684
:1061C0002307F10097000000E780209E09E9B7E768
:1061D0000400BC47414681451305F10082976800E1
:1061E000CD4597000000E78060D397F5FF1F83C57A
:1061F000E54217B501001305259697800100E78059
:106200004077B250456182805DC9411122C426C2E7
:1062100006C6930750FA2300F5009307A005A300D4
:10622000F50089472301F5009147A301F500930785
:106230002004A302F50097F7FF1F9387273E83C72B
:1062400007009304C5002A842303F50097E7FF1F86
:10625000938797FC83C7070023020500A303F5007B
:1062600097F7FF1F83D7E74B2304F500A183A3040F
:10627000F50097D7FF1F83D747162305F500A183A5
:10628000A305F500268597000000E780009201E94C
:10629000B7E70400BC4741468145268582972285A1
:1062A000F14597000000E7802013230EA400218110
:1062B000A30EA400B2402244924441018280828015
:1062C0005D710A8586C6A2C497000000E78000F4CD
:1062D00037E404007C448A850810794682973C4460
:1062E0001305E103094681458297101093050002CA
:1062F000014597D0FFFFE7806040B64026446161CA
:1063000082800111B7C7A55A22CC9387C73317E4FF
:10631000FF1F130474F03EC48347040085660146E2
:106320009965254506CE3EC697C0FF1FE780604BA6
:106330003000A1469965294597C0FF1FE780604A54
:106340008345040017B501001305858B9780010074
:10635000E7802062F2406244056182800111A1461B
:10636000300099652D4522CC06CE97C0FF1FE780EF
:106370004047A24737C4A55A1304C4336395870224
:10638000B24517A501001305657FB335B00097E747
:10639000FF1FA383B7E897800100E780805DF2408C
:1063A0006244056182809165A1463000938505F0C5
:1063B0002D4597C0FF1FE780C042A247E38287FCBC
:1063C00097E7FF1FA38A07E4814517A5010013057E
:1063D000257DD1B7C16769768146FD1705061397FC
:1063E000060141836364B7003E8582803307D50090
:1063F00003470700B98F214713F81700858363050A
:106400000800B18FC207C1837D171377F70F6DF7AF
:106410008506F1B741C5A547054763F2B70883472D
:106420001500034705003168A207D98F139787002D
:10643000A183D98FC207C1831308C855054763904C
:106440000707411106C622C426C20344250091470E
:1064500063F087049307540063ECF502A301C500C1
:1064600021822302C5009304340091C6A302D50003
:10647000A1822303D5002A84A68597000000E78027
:10648000A0F526942300A4002181A300A4000147C5
:10649000B240224492443A854101828005473A85C0
:1064A00082800111B7C7A55A22CC9387E7342A848A
:1064B0002AC6856601469565254506CE3EC497C029
:1064C000FF1FE78000323000A1469565294597C03F
:1064D000FF1FE7800031A28517A501001305457451
:1064E00097800100E780E04897000000E78080DDAA
:1064F000F2406244056182800111A1463000956539
:106500002D4522CC06CE97C0FF1FE780802DA247E5
:1065100037C4A55A1304E43463958702B24517A51E
:1065200001001305E56997D7FF1F2398B7EAC20555
:10653000C18197800100E780C043F2406244056159
:1065400082809165A1463000938505EE2D4597C068
:10655000FF1FE7800029A247E38287FCD14717D7B6
:10656000FF1F231CF7E6D14517A50100130545675A
:10657000C9B721C1411126C206C622C4AE848DC549
:106580002A8497000000E780006497E7FF1F83C715
:10659000A7C899CB22852244B240A68592444101E6
:1065A000173300006700E31AB240224492444101CD
:1065B0008280828001114EC606CE22CC26CA4AC8ED
:1065C00093F71500AE899DCBAD67371700409387D1
:1065D000A7AA1CC3B7E70400BC4F130600198545E2
:1065E00017D5FF1F034545DF829713C51900F240F9
:1065F0006244D2444249B2490561828093F7250042
:106600000145F5D717F7FF1F03578711954763F922
:10661000E70C014417F6FF1F1306860093063005AA
:1066200013055004130810049308B00413039005D5
:10663000930764006374F7043A847D5997F4FF1F4D
:1066400083C404FE97F7FF1F83C797FDA204DD8C68
:10665000AD679387B755638BF41463E3970AA96713
:106660009387A755638EF414A28517F5FF1F1305B2
:1066700025FB97000000E78000F0E9A0B307860043
:1066800083C50700639AD50483C517006396A504E4
:1066900083C527006392050583C53700639ED50235
:1066A00083C54700639A150383C757006396670243
:1066B00022890DE897F5FF1F83D58506B38525410F
:1066C000C20517F5FF1F1305A5F5C1814A9597006F
:1066D0000000E78040EAE1A005044204418089BF50
:1066E0003A847D598547E3EB87F45DC4854517F50A
:1066F000FF1F1305E5F297000000E780C0E769A8D7
:10670000B1679387C7556389F404B5679387D755F5
:10671000E39CF4F4A28517F5FF1F130565F097308D
:106720000000E78000038947630EF4009305E4FF4F
:10673000C205C18117F5FF1F1305A5EE97000000E4
:10674000E7806048A68517A501001305254F9780AF
:106750000100E780002289A097200000E780C0F4B4
:1067600097000000E780804511C9A28517F5FF1F3B
:10677000130505EB97000000E780E0440546A2857D
:1067800017F5FF1F1305C5E997F0FFFFE780A07A13
:1067900097200000E78040F1FD57E31DF9F097F7DF
:1067A000FF1F239F07F613C5290091B5A28517F592
:1067B000FF1F1305E5E697000000E780C08359B787
:1067C000A28517F5FF1F1305A5E597000000E780D8
:1067D00040848DBF411122C437E404005C5C06C6CE
:1067E000354697A50100938525FD17B501001305D2
:1067F000E5C4829711E917A5010013056545978047
:106800000100E780E02E01A08327041C82972A84E0
:10681000054597C00000E78020E297600100E7800F
:10682000406797600100E780403C97B00000E78038
:10683000A0F32285B24022444101828041110545E6
:1068400006C622C426C297C0FFFFE780C06E1305AC
:10685000A00497C0FF1FE7808085757585457D156D
:1068600097C0FFFFE78060587D7585451305F536B5
:1068700097C0FFFFE780C061371400408327840A78
:106880008D451305002093E707202324F40A97C0C1
:10689000FFFFE7808055B7E4040097D0FFFFE78053
:1068A000A09AC85897800100E780802417B501009E
:1068B0001305C5B897800100E78080238327840CE7
:1068C0008545414593E707082324F40C97C0FFFF53
:1068D000E780005C8D451305000897C0FFFFE78047
:1068E000205B97D0FFFFE780008837A507001305DE
:1068F000051297D0FFFFE780A083014597D0FFFFE7
:10690000E780C08995450545894717F7FF1F230B89
:10691000F7E097D0FFFFE780008AB7E700E01307B2
:106920000006238DE7403707000423A0E71097D027
:10693000FFFFE780800B97D0FFFFE780801D970067
:106940000000E78060E997000000E78060A1970001
:106950000000E780A0BA97E0FFFFE780A00697005D
:106960000000E780802797000000E780801083A761
:10697000040817050000130525C4829797D7FF1F49
:10698000238CA7A4BC4C130600648545829797C04E
:10699000FF1FE780E0A501458280AD673717004003
:1069A0009387A7AA1CC3B7E700E03707400023A0DE
:1069B000E71801000100B7F7070003C70701A54763
:1069C0006316F7009397450191C301A04111AE866C
:1069D0000146AA85254506C697C0FF1FE78060E0EF
:1069E000B240B7E700E03707400023A0E7104101BD
:1069F00082804111B2862E86AA852D4506C697C093
:106A0000FF1FE78000DEB24001454101828093070D
:106A1000000463ECC7041D71A2CC2A840808A6CA2E
:106A2000CAC886CE32C697800100E78020E9AD67EC
:106A3000371700409387A7AA1CC3B7E400E03709C3
:106A4000400023A0241901000100B2461008A285CD
:106A5000294597C0FF1FE780C0D8F640664423A0B1
:106A60002411D644464925618280395582804111DE
:106A70000D658D4506C697C0FFFFE7800037B71745
:106A800000408D6623A6D70A17F5FF1F1305C5C959
:106A90001387C70A9387870A1CC15CC58566896707
:106AA0005CC958C114C518C9B7E70400B24003A3B4
:106AB000871E410102838145B307B5008387070024
:106AC00089E7172300006700C3C48505C205C1819B
:106AD000E5B797A70100938727321357C5003E9764
:106AE00003470700011106CE2304E1001357850078
:106AF0003D8B3E970347070023060100A304E100F6
:106B0000135745003D8B3D893E97AA9703470700E1
:106B100083C7070028002305E100A305F1009700C3
:106B20000000E78080F9F24005618280411126C2B1
:106B3000E97797F4FF1F9384A4CF22C49387A755C6
:106B40002E842381B4002E86AA8517F5FF1F130516
:106B500065CE06C62390F400A3810400978001004F
:106B6000E780C0D593052400C205C18117F5FF1F3A
:106B7000130525CC97000000E7800086B3878400CA
:106B80002382A7002181A382A700930564002244E9
:106B9000B24026859244C205C181410117230000FD
:106BA000670023B709C99307800263E6B70017039C
:106BB00000006700E3F7828017F5FF1F034545B823
:106BC000828097F7FF1F83C767C689E717230000F6
:106BD000670023B4828097F7FF1F83C747C899EFE8
:106BE000411106C697200000E78080AAB240854781
:106BF00017F7FF1F2305F7C6410182808280630CCF
:106C0000054A638A054A5D71CAC04EDE86C6A2C4C3
:106C1000A6C252DC56DA5AD85ED662D466D26AD0A0
:106C2000B9472A89AE8963F9B706394697A50100A5
:106C30009385C50997800100E780E0C531ED834762
:106C4000E900130710036394E702854717F7FF1F56
:106C5000230EF7BC17A501001305450897F7FF1F82
:106C6000239507BC97000000E78020E571A013077B
:106C7000000317A5010013056509E395E7FE97F7E3
:106C8000FF1F238507BA97F7FF1F239007BA17A5A1
:106C9000010013052506F9B797F7FF1F83C707B94A
:106CA00063870722BD6AB96B938CFA55014A17FBBB
:106CB000FF1F130B2BA9138CEB65938AFA6605A8AB
:106CC000B307490183C6070097F7FF1F83D7E7B5CE
:106CD000B1E39307A005639BF600854717F7FF1FF5
:106CE0002315F7B497F7FF1F238ED7A4050A931730
:106CF0000A01C183E3E637FDB640264496440649BF
:106D0000F259625AD25A425BB25B225C925C025DDB
:106D100061618280054D639BA7039307500A639EC0
:106D2000F600894717F7FF1F2311F7B0930750FAB2
:106D300017F7FF1FA308F7A055BF9307A005E38728
:106D4000F6FA97F7FF1F239207AE4DB71387170088
:106D50004207DA9741832380D70017F6FF1F2316D7
:106D6000E6AC8D47E3F4E7F817F4FF1F0344B49D46
:106D700097F7FF1F83C7279D22045D8C9307F4FFBD
:106D8000C207C1839306F00DE3EDF6FA93076400A2
:106D9000C207C183E31CF7F493052400C205C18137
:106DA00017F5FF1F1305259A97F0FFFFE780C062D4
:106DB00033078B008347570003474700A207D98F4B
:106DC00017F7FF1F231307A66318F50E8144630C02
:106DD000A40197F4FF1F83C42497A20497F7FF1F11
:106DE00083C79796DD8C170500001305E5DB97F048
:106DF000FFFFE780001263878407636D9C0293871F
:106E0000EB556382F40497F7FF1F83C7E7930547A9
:106E10006389E70681CB1387A7051377F70F8D46A4
:106E200063F2E6081307F0072300E100A300F10076
:106E300089459DA063829405E39754FD97F0FFFF79
:106E4000E780803611A8A28517F5FF1F1305C58FAF
:106E500097F0FFFFE780E01C014597F0FFFFE78018
:106E6000400B69B5A28517F5FF1F1305E58D97F057
:106E7000FFFFE7800024CDB797F0FFFFE780802C6D
:106E8000E1BF930710F8130511002300F10097F0FC
:106E9000FFFFE780A037FD450A8597000000E780E7
:106EA00020C95DBFA28517F5FF1F1305E58997F07F
:106EB000FFFFE780A0DC4DB79307F00789450A85FF
:106EC0002310F10097000000E78080C605B5BD479C
:106ED00063FD3717414697A50100938565E54A850F
:106EE00097800100E780209B6311051617A501001C
:106EF000130545E597000000E78020BC17F5FF1F4C
:106F00000355258297000000E780E0BC97E7FF1F4C
:106F100083C7C77017A50100130545DA89E717A5D0
:106F20000100130525DA97000000E78000B917A5D6
:106F300001001305A5E297000000E78000B817A53F
:106F40000100130525E297000000E78000B717C590
:106F5000FF1F0355254697000000E780C0B717A51F
:106F60000100130565E097000000E78000B517C534
:106F7000FF1F0355854697000000E780C0B517A5A1
:106F800001001305E5DE97000000E78000B317D588
:106F9000FF1F0355C51197000000E780C0B317A578
:106FA0000100130565DD97000000E78000B117D5EB
:106FB000FF1F0355850F97000000E780C0B117A59C
:106FC00001001305E5DB97000000E78000AF17D54F
:106FD000FF1F0355A50D97000000E780C0AF17A560
:106FE0000100130525DA97000000E78000AD17C502
:106FF000FF1F0355E52C97000000E780C0AD17A5E3
:1070000001001305A5D897000000E78000AB0A85B2
:1070100097F0FFFFE78060B9834701000345110047
:10702000A2075D8D97000000E780E0AA834721005A
:1070300003453100A2075D8D97000000E780A0A9FD
:10704000179501001305C54F31B9C14763FE3705D8
:10705000414697A501009385A5D34A8597800100F5
:10706000E780608331E18347090113071003639CC4
:10707000E700854717E7FF1F2304F76C17A50100FA
:10708000130545D2C5B61307000317A50100130564
:1070900065D4E399E7BC97E7FF1F2383076A17A529
:1070A00001001305A5D17DBECE854A8597C0FFFF9F
:1070B000E780001391B18280411126C2AE848D45D4
:1070C00022C406C62A8497C0FFFFE78060DCB7179A
:1070D000004099C803A5C70C418D23A6A70CB24058
:1070E000224492444101828003A5870C418D23A450
:1070F000A70CF5B78347050003471500A207D98FF2
:10710000C2076177C18713072720639AE700834589
:1071100025003705040017030000670023FA82806A
:1071200017E6FF1F130606748147B2861303F00F9C
:10713000A9483308F6000348080013F7F70F630760
:10714000A80C630668008507E39517FF2947B387F6
:10715000E6002380A70097E7FF1F938767715DA86C
:10716000411113D765001347170006C693F6350083
:10717000058B954791CA054699476387C60009461E
:107180009D476383C600A14713F645003336C00010
:1071900093F68503050685C2A145638BB604E145D8
:1071A000638AB604930580026388B604930580035E
:1071B0006393B600914697F5FF1F2380F59297F5EC
:1071C000FF1F238BC59097F5FF1FA387D590BE8522
:1071D00017A50100130545C697700100E780607987
:1071E000B240854717F7FF1FA309F78E4101828040
:1071F0008546D1B78946C1B78D4675BF17A5010031
:10720000130505C6177301006700A37617E7FF1F74
:1072100013070766BA972380B700E147E302F5F446
:1072200093077002E30CF5FC82802A872380050017
:10723000814717E5FF1F1305E5621308F00F294684
:10724000B306F50083C606006396E60297E6FF1FC5
:1072500093860662B69783C7070005452380F5002D
:107260009947636EF7029D4763FDE700E147630DB1
:10727000F7008280638506018507E393C7FC01451B
:10728000C5B7238005008280B737004003C73700A9
:1072900083C7050093F70704D98F2380F500828008
:1072A0005D7152DC56DA5ED6716A97FBFF1F938BD5
:1072B000EB938D6AA6C24EDE62D486C6A2C4CAC053
:1072C0005AD866D26AD06ECEC1495E8C97E4FF1F51
:1072D0009384C45A130A0A20938A7ADC17F9FF1F91
:1072E0000349C993B3872B0183C7070093F7F70FAF
:1072F000C9EFB787004003C76700058BE310077C21
:1073000003C76700118BE30D077E83C75700918B7E
:1073100099E36F10200317F7FF1F03474790854736
:107320006304F7006F10400197E7FF1FA387E77A18
:1073300097E7FF1F2384076097E7FF1F2382076CEF
:1073400097E7FF1F2380077897E7FF1F238D0776B6
:1073500097E7FF1FA384075E97E7FF1FA382076AD3
:1073600097E7FF1FA380077697E7FF1FA38D07749A
:1073700097E7FF1FA384077697F7FF1FA381078A6C
:10738000B787004011476F0070779307190093F794
:10739000F70F3D476364F70617F7FF1F2300F788D1
:1073A00097F7FF1F93878786CA9783C7070013073E
:1073B000100293F7F703638EE71E6366F704054434
:1073C0006385871CE38C07620947638EE710130708
:1073D0000002E384E74EB7E700E03707400023A050
:1073E000E71801000100629923000900FD1923A09C
:1073F000E71093F9F90FE39309EEE5BD97F7FF1F47
:10740000238E078071BF130730026388E70C63E89F
:10741000E71613074002638CE70A13070003E39C97
:10742000E7FA97E7FF1F9387677DCA9703C70700AF
:10743000A1471377F70FE31BF71483C7640097E6A0
:10744000FF1F2383F66897E7FF1F83C7974391C702
:10745000FD5797E6FF1F2389F66697E5FF1F83C553
:10746000F54197E7FF1FA381B76697E7FF1F83C723
:10747000E74013FB07089306000493F70706639F92
:10748000D74C9307A009638DF51663EAB7129307EB
:10749000F0056386F54A930750096384F52A014491
:1074A00097E7FF1F83C757621547E392E736B7E7B1
:1074B00000E03707400023A0E71801000100B7866D
:1074C000004023808602130680FC6F00500EFD579B
:1074D00017E7FF1F2309F75EFDBDFD5717E7FF1FE5
:1074E0002302F75ECDBD17A501001305E5A897702F
:1074F0000100E780E05F97E7FF1F93872770CA9737
:1075000003C40700014B97ECFF1F938CAC4F13741F
:10751000F40F17AD0100130DADA663478B04294589
:1075200097700100E780C049854717E7FF1FA3094F
:10753000F74C17E7FF1F2306874C17E7FF1F230FA2
:10754000F75837E700E0B70640002320D7180100BE
:107550000100378600408347A60293F7370F2305C3
:10756000F6022320D71085BDB3876C0183C50700C1
:107570006A85050B97700100E780A03F79BF8547BA
:1075800017E7FF1F230EF746B9B517E7FF1F1307CD
:10759000E7664A970347070097E6FF1FA380F63A7E
:1075A00097E6FF1F238DE63817E7FF1F2308F752E2
:1075B0001DB5854717E7FF1F2302F73829BD93073D
:1075C000400A6389F5349307200B6384F5369307EB
:1075D000100AE396F5EC838724000144E3D207EC1C
:1075E00097E7FF1F83C7B72993F63700638A061A08
:1075F0000546638AC62209466395C61A1D4755A2E9
:1076000017E5FF1F0345A527C94797ECFF1F83CC4C
:107610001C2797E5FF1F83C5A52617E4FF1F03441A
:1076200034266315F510CD476392FC10930770085C
:10763000639CF5021307300FB7170E006308E400D0
:107640001307900DB7B704006314E40817E7FF1F92
:107650002322F748BE8517A501001305E592977010
:107660000100E780003125BD93078008639DF50088
:10767000B307804013F4F70FB7774600938787CDA1
:10768000B3D78702E1B793079008639AF500B30771
:10769000804013F4F70F91679387C766D5B79307B8
:1076A000A008639BF500B307804013F4F70FB717EA
:1076B0003D0093870790E9B79307B008639AF500F8
:1076C000B307804013F4F70F9167938797D04DBFAE
:1076D00093F5F5078D47639BF500B307804013F4DE
:1076E000F70FB7975B00938707D859BF8947639B0C
:1076F000F500B307804013F4F70FB7770B009387BB
:10770000071BBDBF8547639AF500B307804013F49C
:10771000F70FDD67938767E3A5B7D28785F9B307CE
:10772000804093F7F70FB3D7FA020DB79700000028
:10773000E780409FA285668597000000E780809ED5
:10774000B9BB9305610017E5FF1F0345451317E417
:10775000FF1F0344D41297000000E78040AD93055B
:107760007100228597000000E78060AC3C0017E7BD
:10777000FF1F232BF746834761002304F100834753
:107780007100A304F100894717E7FF1F230EF732AA
:107790008357810017E7FF1F2312F70E094409B32F
:1077A000154793F64700B336D00093F78703850655
:1077B00085C32146638BC7066146638AC7061306E5
:1077C00080026388C706130680036393C70091474E
:1077D00017E6FF1F2302D63097E6FF1FA38EF62E73
:1077E00097E7FF1F238BE72E17E7FF1F0347470984
:1077F0009376070497E7FF1F83C797088DEE1377EB
:10780000770C93067008630CD7021377F7078D4641
:107810006312D70CB307F040B7955B0093F7F70FEF
:10782000938505D849A81947ADBF854755B78947FE
:1078300045B78D4771BF930670086311D7021307D0
:10784000300FB7150E006389E7021307900DB7B527
:1078500004006383E7021307700845BF9306800C9A
:107860006311D702B307F040B775460013F7F70F5F
:10787000938785CDB3D5E70297E7FF1F23ACB724E5
:10788000D9BB9306900C631CD700B307F04093F567
:10789000F70F91679387C766B3D5B702F1BF930619
:1078A000A00C631DD700B307F040B7153D0093F758
:1078B000F70F93850590B3D5F5027DBF9306B00C05
:1078C000E315D7F4B307F04093F5F70F916793876B
:1078D00097D0D9B78946631BD700B307F040B77577
:1078E0000B0093F7F70F9385051BF1B78546631AD5
:1078F000D700B307F040DD6593F7F70F938565E395
:107900005DBFD28535FBB305F04093F5F50FB3D5D8
:10791000BA029DB783C72400C18B99C7854717E773
:10792000FF1F2306F71AA5BE97E7FF1F2381071A3B
:10793000BDB6854717E7FF1FA301F71A8DB63C00B8
:1079400017E7FF1F2322F72A094793070003231491
:10795000F10097E6FF1F2389E6162DBD63940756B5
:10796000A94763E5B742179701001307274A8A051D
:10797000BA959C41BA97828717E4FF1F034434F0FD
:10798000894C6306940D63E68C0685476303F4080F
:107990009307F00F17E7FF1F0347071363F6E7008E
:1079A00017E7FF1F2302F71297ECFF1F83CCCC11C0
:1079B0009307000413F4FC0F63F49701130400040D
:1079C00097E7FF1F9387472203AD0700228626858E
:1079D000EA85B38C8C40229D97700100E78000EE11
:1079E00097E7FF1F2382970F97E7FF1F23AEA71F7D
:1079F00045BC8D47630CF40A9947E31BF4F897974D
:107A000001009387274717E7FF1F232FF71CA9477C
:107A100051B717E7FF1F0347872097E7FF1F93879B
:107A2000A70C4946979501009385C54D63068700CD
:107A300097950100938505493E8597700100E78081
:107A4000E0E717E7FF1F2321A71AC947A1B797E669
:107A5000FF1F83C6C61C054797E7FF1F9387C7080C
:107A60006394E6023E8513067002979501009385A4
:107A7000E54697700100E78060E417E7FF1F2325C4
:107A8000A7169307700239B73E8513063004979501
:107A900001009385E53E97700100E78020E217E73B
:107AA000FF1F2323A71493073004EDB597E5FF1FAD
:107AB00083C5E5DC179501001305454E977001005D
:107AC000E78020EB054D97EDFF1F83CD4D1597E522
:107AD000FF1F83C5C5DA179501001305254C639870
:107AE000AD0B97700100E780C0E897E7FF1F83C7E1
:107AF00007D9B5CBE36EF4E8179401001304C4442E
:107B0000638CB701179401001304844463869701C2
:107B10001794010013044445228597700100E78003
:107B200060FE1375F50F93071500860717E7FF1F13
:107B3000230CF7FA8D4717E7FF1FA307F7FA97E71C
:107B4000FF1F938767FA0147BE861376F70F8907F1
:107B50006365A60297E7FF1F23A8D70897E7FF1FD3
:107B600083C787F805BD979701009387E73617E726
:107B7000FF1F232BF706914731BD3306E400034670
:107B80000600A380070005072380C7007DBF97700C
:107B90000100E78000DE97E7FF1F83C747CEE1D7EC
:107BA000E368F4DE1794010013040437638CA70123
:107BB000179401001304C4366386970117940100DB
:107BC00013048437228597700100E780A0F31375B2
:107BD000F50F93071500860717E7FF1F2306F7F039
:107BE0008D4717E7FF1FA301F7F097E7FF1F938764
:107BF000A7EF0147BE861376F70F8907E37CA6F44B
:107C00003306E40003460600A3800700050723802F
:107C1000C700D5B797E5FF1F83C565C61795010057
:107C20001305853897700100E780A0D497E7FF1F00
:107C300083C757EB93E7470017E7FF1FA304F7EA53
:107C400083C7240017E7FF1FA30CF7E889B817952F
:107C500001001305A53697700100E78060E997E7FA
:107C6000FF1F9387E7E783C7070017E7FF1F230777
:107C7000F7C017E4FF1F034424E5333480000DB040
:107C8000179501001305C53497700100E78040E6A1
:107C900097E7FF1F83C717E593E7070117E7FF1F64
:107CA000A302F7E483C7240017E7FF1F230AF7E2C4
:107CB0006FF0EFFE179501001305C53297700100B4
:107CC000E78000E303C704007D8B51EFB7870040D6
:107CD00003C767021377C70B136727002383E702E5
:107CE00003C7A7021377C70B136727002385E70293
:107CF00003C7E7021377C70B136727002387E70241
:107D000003C727031377C70B136727002389E702ED
:107D1000854717E7FF1F2303F7C217E7FF1F23015C
:107D2000F7CE17E7FF1F230FF7D817E7FF1F230C26
:107D3000F7D897E7FF1FA38307C097E7FF1FA3812B
:107D400007CC97E7FF1FA38F07D697E7FF1FA38CEA
:107D500007D697E7FF1FA38307D897E7FF1FA380E6
:107D600007EC6FF0CFF389476312F70297E7FF1F25
:107D700083C707B19146638CD70863E0F604638E2E
:107D8000E70C6369F70A05476380E70EFD5717E7BD
:107D9000FF1FA30BF7D237074000B7E700E023A08F
:107DA000E71801000100B78600401306F0FC2381AC
:107DB000C60223A0E7106FF00FE2130720086382CA
:107DC000E7086362F70213071008E391E7FC3787BF
:107DD00000408347670293F7C70B93E7270023030D
:107DE000F7026FF0CFEB130730086389E702130740
:107DF0004008E39DE7F8378700408347270393F760
:107E0000C70B93E727002309F7026FF04FE9378785
:107E100000408347270393F73707F5B737870040BC
:107E20008347E70293F7C70B93E727002307F7027F
:107E30006FF0EFE6378700408347E70293F7370795
:107E4000F5B7378700408347A70293F7C70B93E73F
:107E500027002305F7026FF08FE437870040834740
:107E6000A70293F73707F5B73787004083476702C4
:107E700093F73707ADB7179501001305A51797704E
:107E80000100E780E0C697E7FF1F2389079ED5B36F
:107E9000179501001305051797700100E78040C58D
:107EA00097E7FF1F239C079C97E7FF1F9387C7C196
:107EB00003C40700894763F3870009441374F40F70
:107EC0006FF00FDE13070002E392E7EC631B0B0A6F
:107ED000638FF500930720026383F508179501006F
:107EE0001305C51597700100E780A0A845B5179543
:107EF00001001305E51197700100E78060BF0144A0
:107F0000179D0100130D0D12A14CB387840083C58A
:107F100007006A85050497700100E78080A5E316D5
:107F200094FF178501001305A56797700100E7808E
:107F300020BC17E4FF1F0344A49401E897E7FF1F48
:107F400023800792014B6FF0AFD58947E310F4E42B
:107F5000854717E7FF1F2305F7906FF04FD417E60B
:107F6000FF1F0346D69197E5FF1F83C545911795DF
:107F700001001305A50B97700100E780809F6FF04B
:107F80000FD26380F50693071002E399F5F497E5A5
:107F9000FF1F83C5E58E179501001305250B97700C
:107FA0000100E780009D97E7FF1F23AF97C297E787
:107FB000FF1F938727B2944383D7470017E7FF1F1C
:107FC0000347A7B117E6FF1F232AD68A1D4497E669
:107FD000FF1F2397F68A97E7FF1F2384E78A6FF036
:107FE0002FCC97E5FF1F83C5A589179501001305C1
:107FF000650797700100E780C09797E7FF1F23810F
:10800000078697E7FF1F239B07866FF02FF9254709
:10801000638FE7C89946378700406394D7022300EF
:108020008702B7E700E0B706400023A0D718010099
:108030000100130600FC2301C70223A0D7106FF034
:108040008FB99306100A639FD70023008702B7E712
:1080500000E0B706400023A0D71801000100130676
:1080600080FCD1BF9306A009E381D7FE9306400AA6
:10807000E38DD7FC93062002639DD700B7E700E0AD
:10808000B706400023A0D718010001002300870293
:10809000F9B78546E384D7FE93070008E300FBFEAB
:1080A000B7E700E0B706400023A0D71801000100A1
:1080B000130620FC23008702BDBF17E7FF1F0347FD
:1080C000B7A06302F71E63E7E70295476300F71066
:1080D0009947630AF704B786004023800602B7E792
:1080E00000E03707400023A0E71801000100130655
:1080F000A0FC75B99307F005630AF70093075009D0
:108100006306F70093071002E317F7FCB7E700E0F8
:108110003707400023A0E71801000100B7860040A0
:10812000130620FC69B117EBFF1F034BEB99930774
:1081300000045A8D63F46701130D000497E7FF1FD5
:10814000938787AA83AC07001374FD0F2286E68508
:10815000268597600100E7806076B3078B406694C0
:1081600017E7FF1F2302F79697E7FF1F23AE87A6A7
:10817000B7870040630C0B022380A703B7E600E03B
:108180003706400023A0C6180100010003C72702DC
:10819000134707042381E70203C727021377C70F9A
:1081A0002381E70223A0C6106FF0EFA2238007020D
:1081B00037E700E0B70640002320D7180100010090
:1081C000130620FC2381C7026FF0AFB93787004048
:1081D0008347370097E6FF1F83C6969093F70708FB
:1081E000D58FA301F700B7064000B7E700E023A052
:1081F000D718010001001306A0FC35BD97E7FF1F4B
:108200009387C79FCA9783C7070093F7F70FC1CF1C
:1082100097E7FF1F83C7A7A0D9E717E7FF1F03470B
:10822000B78A930700026310F70883AD040017DDD7
:10823000FF1F034DED6497DCFF1F83CC7C6417DBCD
:10824000FF1F034B0B64E6876A87DA866E8697D535
:10825000FF1F83C5E56017950100130525E29760B0
:108260000100E780007197E7FF1F23A5B78797E715
:10827000FF1F2383A78797E7FF1FA38F978597E7A4
:10828000FF1F238C678597D7FF1FA38A875CB7E7FB
:1082900000E03707400023A0E71801000100B7867F
:1082A00000406FF04FA2B7E700E03707400023A07F
:1082B000E71801000100B786004015BD97E6FF1FD3
:1082C00083C6E6950547639CE60429472381E702B8
:1082D00009472383E7022385E70297D7FF1FA38F70
:1082E000077E97E7FF1FA38C0792B7870040A38103
:1082F000070017D7FF1FA305077E05472383E70065
:10830000B640264496440649F259625AD25A425B14
:10831000B25B225C925C025DF24D61618280294712
:108320002381E70209472383E7022385E7022387A6
:10833000E7022389E70255B717D7FF1FA301F752BA
:108340006FE01FFF854717D7FF1F2309F75E17D779
:10835000FF1F2307F76A17D7FF1F2305F77617D7E5
:10836000FF1F2302F7766FE0BFFE854717D7FF1F79
:108370002306F75C17D7FF1F2304F76817D7FF1FE3
:108380002302F77417D7FF1F230FF77217D7FF1FAA
:10839000A306075A17D7FF1FA304076617D7FF1FA7
:1083A000A302077297D7FF1FA38F07708280411126
:1083B00006C697000000E78080FBB7870040238057
:1083C0000700130740FC2386E7001307C004A386B9
:1083D000E70017D7FF1F1307674A2398E70017D74F
:1083E000FF1F1307A74D239AE70017D7FF1F130797
:1083F0002759239CE70017D7FF1F1307A764239E65
:10840000E70029472381E70209472383E702238501
:10841000E7022387E7022389E702A3810700930687
:1084200000F8A380D700930690022380D700FD5662
:108430002383D7002381E7009306000537E700E098
:10844000230BD740B70640002320D71003C71700DF
:1084500013671700A380E700B24097D7FF1F23914F
:10846000076841018280411106C697000000E7803D
:1084700000F0B787004023800700130700FC238625
:10848000E7003147A386E70017D7FF1F1307073F11
:108490002398E70017D7FF1F13074742239AE700E7
:1084A00017D7FF1F1307C74D239CE70029472381D8
:1084B000E70209472383E7022385E702A381070038
:1084C000930600F8A380D700930690022380D7007C
:1084D000FD562383D7002381E7009306000537E785
:1084E00000E0230BD740B70640002320D71003C776
:1084F000170013671700A380E700B24097D7FF1F4C
:108500002390075E41018280F1679387072017D788
:10851000FF1F2321F75C854717D7FF1F231EF75A3C
:10852000A14717D7FF1F230AF75A97D7FF1FA38624
:10853000075A97D7FF1F2383075A97D7FF1F238117
:10854000073297D7FF1FA38C0730814717D5FF1F2E
:1085500013054531FD5517D6FF1F13066631294710
:10856000B306F5002380B600B306F60023800600AC
:108570008507E397E7FE97D7FF1FA388075497D790
:10858000FF1FA386075497D7FF1F2381075497D750
:10859000FF1F238C075297D7FF1F238B075297D7B4
:1085A000FF1FA385075297D7FF1F238207528147DA
:1085B00017D6FF1F130686634147B306F6002380D4
:1085C00006008507E39BE7FE828017D7FF1F03475E
:1085D000076585476316F700170300006700E3E8A7
:1085E000170300006700E3DC411122C406C617D759
:1085F000FF1F0347C76285472E8613F4F50FAA8530
:108600006317F70417D5FF1F1305853B976001001B
:10861000E780C02A97D7FF1F2384073EB787004013
:1086200023848702B7E600E03706400023A0C6187F
:108630000100010003C7A7021377C70F2385E702D4
:10864000B240224423A0C61001454101828017D5C3
:10865000FF1F1305A52A97600100E780202697D702
:10866000FF1F238D072CB787004023828702B7E6C0
:1086700000E03706400023A0C6180100010003C730
:1086800067021377C70F2383E7025DBF411106C658
:1086900097000000E78080E7B24041011703000027
:1086A0006700E3F2411106C697F0FFFFE78080BF45
:1086B00097D7FF1F83C79728A1CB97D5FF1F83C5E7
:1086C000052889C917D5FF1F1305852797E0FFFFE8
:1086D000E780205397D7FF1FA382072697D7FF1F56
:1086E000238E073E37E700E0B70640002320D71867
:1086F00001000100378600408347660293F7370F79
:108700002303F6022320D710B2404101828041C9E1
:10871000D9C597D7FF1F83C7A73CD1C3011122CC6E
:108720004AC84EC656C25AC006CE26CA52C42E8960
:10873000AA890144930A0004371B030063772403CA
:10874000B3078940C207C183BE8463F4FA0093046F
:108750000004C204C180130A1BD497D7FF1F83C72C
:10876000E71D9DE37D1A631C0A00F2406244D24477
:108770004249B249224A924A024B0561828097F0EF
:10878000FFFFE78020B2D1BF338589002694A685FC
:10879000420497000000E78060E5418045B7828091
:1087A00097D7FF1F9387075A18429C4383D64500EB
:1087B0000345070083C5C700035646006396A5001E
:1087C00083D5E700638DD502011106CE2386A7006D
:1087D0002397D700B705CF00DC4B9385757D050740
:1087E0007D162EC2230001003AC42316C1002317B0
:1087F000D10099C30A858297F24005618280828008
:10880000411122C417B4FF1F130484BF5C4C06C679
:1088100091CBC84B01C9B7E70400BC5782975C4CA9
:1088200023AA0700B240224441018280DC4DDC4B88
:1088300081CFB7E70400904503A38705914517D57D
:10884000FF1F0345655002838280B7E7040003A33E
:108850000705A14517D5FF1F0345054F02836D711D
:108860003C083EC6B707E500232291103EC8AA8403
:108870003C083285232611103ECA23248110232070
:1088800021112E8997300000E78000592A8497959E
:10889000010093852582177501001305A56D97606A
:1088A0000100E780000DA285179501001305458D95
:1088B00097600100E780E00B294597600100E780A1
:1088C0002010B705CB009385757D680097100000D8
:1088D000E780805EA285680097300000E780204630
:1088E000014781467000CA85268597200000E780F1
:1088F000008205CD2A84978501009385A57B177595
:1089000001001305256797600100E7808006A285B6
:10891000179501001305858797600100E7806005C2
:10892000294597600100E780A0098320C110032436
:10893000811083244110032901105161828097D74F
:10894000FF1F9387274018429C43797122D406D693
:108950000348070083C807012A8483D645000355CE
:1089600046006396080183D82701638DD8022388C7
:10897000070105072399D7003708CC00DC4B130803
:10898000787D3ACC1307F5FF42CA23080100231E65
:10899000E100231FD10099C7080832C62EC4829770
:1089A0003246A245228597000000E78080EBB25056
:1089B0002254456182807971314697750100938513
:1089C000254C280006D697600100E78020EF97B776
:1089D000FF1F83D7E7A2231B0100231C0100231DD7
:1089E0000100231E0100231F010099E3C167FD1749
:1089F000231AF10097B7FF1F83D7A7A091EB97D752
:108A0000FF1F938727349C439C43DC4783D7070091
:108A100097B6FF1F9386C69E231BF100D84E83D7BF
:108A20004600231CF1005C4B91CB97B7FF1F83C717
:108A3000979D81EB97000000E780C0DCB250456154
:108A40008280FD1717B6FF1FA30FF69A0356070182
:108A500083C706014C472800230FF1009730000020
:108A6000E780002B97D7FF1F9387C72D9C430147B3
:108A7000978601009386866D884330004C089710D6
:108A80000000E780C0685DD975B799C9B7E70400F1
:108A900003A30705A14517D5FF1F0345E52A028358
:108AA00082805C4EDC4BB9CFB1CD411122C4177529
:108AB00001001305254C2E84978501009385C5641C
:108AC00006C697600100E780C0EAA285178501000D
:108AD0001305C56597600100E780A0E92945976007
:108AE0000100E780E0EDB7E704002244B24003A3B1
:108AF000870517D5FF1F0345252513064006914519
:108B0000410102838280411122C417B4FF1F130464
:108B1000E48C1C4C06C689C7DC4399C34C48829739
:108B2000584CB7E70400BC57484B82975C4CB240A6
:108B3000224423AA07004101828017B7FF1F1307B1
:108B4000E78B834707009306F00B850793F7F70F32
:108B500063E9F60097B6FF1F2382F68A03450700F4
:108B60008280930700F8FDB78357450099E37D5550
:108B70008280011122CC17B4FF1F130464885C4C5F
:108B80004AC84EC6DC4B52C406CE26CA56C2B2896B
:108B90002E8A2A898DC7B7E70400FC5F829797D792
:108BA000FF1F938727189C431307301FB307F54017
:108BB00071556375F70697000000E780A0C493071E
:108BC000D00D7D5563EC3705B7E404009387890029
:108BD000B858832AC401139507014181029723AA3B
:108BE000AA00484C584921E7978501009385C54F55
:108BF000177501001305053897600100E78060D7FD
:108C0000178501001305455B97600100E78060D67A
:108C1000294597600100E780A0DA5D55F240624483
:108C2000D2444249B249224A924A0561828013875E
:108C30004900B705CF002319E5009385757D3105FF
:108C400097100000E7804027484C834569003105B4
:108C500097300000E780A00E484C4E86D285310543
:108C600097300000E780C00A7146CA8517A5FF1F2C
:108C70001305057997600100E78040C4FC5C82978A
:108C80000326C90097D7FF1F23AEA70811CABC4C03
:108C9000854517D5FF1F0345250B82970145BDBFAD
:108CA00097000000E78060D1D5BF411106C622C4FD
:108CB00026C217D4FF1F1304240997000000E78081
:108CC00060B4B7E40400FC4C03450400854582977A
:108CD00003450400224403A3C405B2409244A145C5
:108CE00041010283411126C297D4FF1F938484055A
:108CF0009C4006C622C44AC0D5C3DC43C5C35CC180
:108D00002300B5002A8497850100938525391775BE
:108D100001001305252697600100E78080C52945DD
:108D200097600100E780C0C99C4023A4070023A2EC
:108D3000070097A7FF1F9387676ADC4FDC4B91C73B
:108D4000295597000000E78040DC97A7FF1F938715
:108D5000276BDC4FDC4B89C797000000E78020F5CC
:108D600037E904008327C905894517D5FF1F034547
:108D7000A5FD82978327C905914517D5FF1F034598
:108D8000A5FC82979C4003A3470163090300228549
:108D90002244B2409244024941010283B24022443B
:108DA00092440249410182800111328506CE22CCD3
:108DB00026CA2E8497300000E7800006AA84978593
:108DC00001009385E530177501001305A51A97601A
:108DD0000100E78000BA030784000356640083554E
:108DE0004400A686178501001305C536976001006B
:108DF000E78020B8294597600100E78060BC97A70D
:108E0000FF1F83C7075E639D970001459700000021
:108E1000E780A0CF81450A8597000000E780C0EC7D
:108E2000F2406244D244056182806D712324811036
:108E3000232611102322911093F745002E84638777
:108E400007143C083EC0B707E5003EC23C083EC4DC
:108E5000231701002318010023190100231A010020
:108E6000231B010097A7FF1F83D7475799E3C167CB
:108E7000FD172316F10097A7FF1F83D7475691EBE5
:108E800097D7FF1F938707EC9C439C43DC4783D70E
:108E9000070017A7FF1F130767542317F100544F4C
:108EA000835747002318F100DC4AA1E797850100AA
:108EB00093854526177501001305C50B97600100C2
:108EC000E78020AB17850100130585359760010009
:108ED000E78020AA294597600100E78060AE13452E
:108EE00044008320C1100324811083244110516168
:108EF000828097A7FF1F83C7D74E2555D9C3FD177B
:108F000017A6FF1FA30FF64C03D6060183470701E0
:108F1000CC460A85230BF10097300000E78040DF44
:108F200097D7FF1F938707E29C4317A7FF1F1307DD
:108F3000E74A978601009386E61E88430A866C00FE
:108F400097100000E780A01CAA8451D997850100E2
:108F50009385451C177501001305C5019760010035
:108F6000E78020A1A685178501001305252C9760B1
:108F70000100E78000A0294597600100E78040A438
:108F8000268597000000E78040B891BF93F7250041
:108F90009DC7B7E70400BC47414681452808829732
:108FA000255597000000E78040B628089305F00F8C
:108FB00097000000E78040D3134524001DB793F7C6
:108FC000150081CB97000000E780209F1345140017
:108FD00009BF93F78500014589D717A7FF1F0347EE
:108FE000974297A7FF1F9387A7410DC3D84F584BB0
:108FF00011CF37E70400384F9047854517D5FF1F3D
:10900000034585D4029713458400E1BD97F0FFFF27
:10901000E780407FCDBF5C4D411106C688C317D79E
:10902000FF1F2321F7D2B7E7040083A7070817051E
:1090300000001305C5DF8297B24097D7FF1F238535
:10904000A7D001454101828001113335A000A3075B
:10905000A100B7E7040083A7471706CE1306F10067
:109060008545130550308297F240056182808280E9
:10907000411122C406C697B7FF1F83C7F7190544DD
:1090800089EF97C7FF1F83C76759014499E717B452
:10909000FF1F034464181344140022859700000046
:1090A000E780C0FA178501001305051F09E417853D
:1090B00001001305651F2244B240410117630100FE
:1090C0006700238B797122D4A30F010037E40400D9
:1090D0008327841726D24AD006D6AA842E89130560
:1090E00050309305F10132C6829732468347F10131
:1090F00093150601C18185CB01452EC6970000005E
:10910000E780C0F483274417B2454A8626858297B4
:10911000054597000000E78060F3B2502254925456
:10912000025945618280832744174A8626858297A3
:10913000EDB741119397050122C406C626C2C18727
:109140002E8463D40702B7E40400FC5417A5FF1F64
:109150000345052E829719C1BC5482972165218D44
:10916000B240224492444101828093F715008DC79A
:10917000B7E7040083A7471A17A6FF1F1306462A5E
:1091800097D5FF1F938505BD17A5FF1F0345452AEA
:10919000829713451400E9B793F725000145E9D3F9
:1091A00097D7FF1F83C787BC85E7B7E7040003A8ED
:1091B000871A1307401F97A7FF1F83C7672781469A
:1091C00013064006994517D5FF1F0355A5B9029808
:1091D0001345240071B797D7FF1F83D7A7B86398AB
:1091E000A70217D7FF1F2310B7B817D7FF1F231DDC
:1091F000C7B617D7FF1F231AD7B62E8617850100CB
:1092000013050511BE851753010067008376178586
:10921000010013056511176301006700638D035793
:10922000450097D7FF1F83D7E7B36318F702C167DD
:10923000F91717D7FF1F2327F7B297D7FF1F23A5CB
:1092400007B297D7FF1F238D07B097D7FF1F238F34
:1092500007B0170300006700E3E11785010013055D
:10926000A50C176301006700A3887D15954763E28D
:10927000A71C178701001307A7000A053A951C4190
:10928000011122CC06CEBA972E8482871785010061
:109290001305050A97600100E7808085A1A203C736
:1092A000250099476311F7022E8597000000E7809B
:1092B00040F7834564001785010013056508975042
:1092C0000100E780006B97B7FF1F238707F417851E
:1092D00001001305A5087DBF03C725009547631945
:1092E000F702C16717D7FF1F0357C7A7F91703D5A1
:1092F000A5006309F702B7E7040083A7C7178297A1
:10930000178501001305850697500100E780407E10
:10931000854717B7FF1F2301F7F0178501001305D5
:1093200065078DBF97D7FF1F239EA7A283D7E500B0
:1093300097D6FF1F2399F6A283D7050197D6FF1F63
:109340002394F6A283D7250197D6FF1F239FF6A06B
:1093500097D7FF1F238607A0631BE502B7E704002A
:10936000BC4F096613060690894517A5FF1F0345E4
:10937000250C82970356E4008355A400178501004D
:109380001305050097500100E780A05E51B79307D1
:10939000700F2316F100B7E7040083A7870D17A607
:1093A000FF1F0346E6086C0082974DF9854717D7E3
:1093B000FF1F2307F79A5DB717850100130545FEC8
:1093C000D1BD83C5250091476392F5021785010041
:1093D000130585FE97500100E7808071970000001B
:1093E000E78040C9F24062440561828099476392F8
:1093F000F502228597000000E780A0E28345640023
:10940000178501001305C5F397500100E7806056EA
:10941000D1BF9547639AF50083471400E1F31785A0
:1094200001001305A5FBBDB517850100130585FBDC
:10943000E1BF82803757315F97A7FF1F938787006F
:10944000130777D598C39356C500178701001307F4
:10945000E7E8BA9683C5060093568500BD8ABA969A
:1094600003C6060093564500BD8A3D89BA962A97E1
:1094700083C6060003470700238407002383D70021
:10948000A383E7002382B700A382C70097A7FF1F2B
:10949000938747FC2383B700A383C7002384D700A7
:1094A000A384E7008280411106C697000000E78090
:1094B000A0F8B7E7040083A7871417A6FF1F1306B9
:1094C00066F8D54501458297B2404D4697A5FF1FE6
:1094D000938545F8130570304101170300006700BC
:1094E000A3BE61712324811A37E404008327040892
:1094F0002326111A2322911A2320211B232E3119EE
:1095000017050000130525C3829717A9FF1F13092C
:1095100029F2994785442300A900231CF10097856F
:1095200001009385A5DA930740061775010013051E
:1095300065A4231CF1082308910097C9FF1F938994
:10954000491E97500100E780C04283D50900178566
:1095500001001305A5D697500100E78080412945F9
:1095600097500100E780C04503D50900970000002F
:10957000E78080EC83274417100885451305503099
:1095800082978327441717A6FF1F1306A6ECCD4525
:109590001305703082978327441717A6FF1F130601
:1095A00066E9B54513056030829783274417300874
:1095B000894513051031829783274417300989455F
:1095C000130520318297832744159305000A0D4522
:1095D0008297832744159305000A11458297A305B6
:1095E00091002306910002CD23080100230C010005
:1095F000832784163009914513057040829783278D
:1096000084161306B1008545130500408297832711
:1096100084167000854513051040829783278416B1
:10962000300885451305204082978327841610084B
:109630008545130550408297832704157D558297F1
:10964000832744137D5582977D5597A0FFFFE780C0
:10965000C0038327440C829797A0FFFFE78020DF99
:109660008327841417A6FF1F1306C6DDD5450145C1
:10967000829789471306700F814528092306F10058
:109680009790FFFFE780A0A88D471306000881454B
:109690002808230CF1089790FFFFE78040A7914727
:1096A000230CF100976701009387477E984383C797
:1096B00047003AC8230AF10097D0FFFFE78080C037
:1096C00070008545054597A0FFFFE780200330091E
:1096D0009305700F094597A0FFFFE780200230082F
:1096E000930500080D4597A0FFFFE78020011008B3
:1096F0009545114597A0FFFFE7804000C16717C758
:10970000FF1F13072766F9171CC32322070017A59D
:10971000FF1F1305A5D197A0FFFFE78000FD83275A
:10972000C41D17C5FF1F1305656282973C4803459A
:109730000900854582978320C11A0324811A832456
:10974000411A0329011A8329C1195D618280C16709
:1097500017C8FF1F03580861F9176301F8083DCDCA
:10976000B5CD011126CAB7E4040083A7841222CC28
:109770002E862315B10006CE2A8401478146ED4589
:10978000428582972AC611ED17850100130545B65B
:1097900097500100E780C035F2406244D244056131
:1097A0008280FC440356A100A28582972C0017C535
:1097B000FF1F0355255B97A0FFFFE780C0FF69DD12
:1097C00017850100130505B497500100E78040326A
:1097D00083A7C412ED45280082977DBF82800DC506
:1097E000854717A7FF1FA30CF7C497A7FF1F23895F
:1097F00007C4354697A5FF1F9385C5C31305603081
:10980000170300006700438C97A7FF1FA38907C2B7
:10981000E9BF97C7FF1F83C76755A9EFC16717C780
:10982000FF1F03572754F9176306F70441118547B3
:1098300022C417C7FF1F230BF75237E404007C4CE8
:1098400006C6894517A5FF1F034585BE82970323DA
:10985000841A2244B24097A7FF1F83C767BD17C56C
:10986000FF1F035525501307401F81463146994578
:109870004101028382806D712324811023261110FF
:1098800023229110328401CD8947630AF502832097
:10989000C1100324811083244110516182801785F7
:1098A00001001305E5B4AE8497500100E780402421
:1098B000A285268597C0FFFFE78000CAC9BFB7E72A
:1098C0000400FC472800829717850100130505B3A3
:1098D00097500100E780C0218347810039C41307F6
:1098E000000B6380E7021387A7051377F70F8D46F8
:1098F00063EDE602A285280097C0FFFFE7800038ED
:1099000079B78547E3F587F883459100177501001E
:1099100013058597B335B00097A7FF1F2386B77847
:1099200097500100E780E0049DB703479100A2072C
:10993000D98F35671307D7556385E7086368F70242
:109940002D671307B7556387E70631671307C755B8
:10995000638AE70429671307A7556394E702A28582
:10996000280097C0FFFFE780C06A15B739679306E4
:10997000E7656381D70863E9F6001307E755638459
:10998000E706A28528003DB73D679306F755638A31
:10999000D7061307F766E396E7FE97D0FFFFE78049
:1099A000A080F5B50146A285280097C0FFFFE7809B
:1099B0008058F1BDA285280097C0FFFFE780A06313
:1099C000F9B58947E3F587EC97000000E780A0E44C
:1099D0009305E4FFC205C1811305A10097A0FFFF15
:1099E000E78000806DB5A285280097C0FFFFE78063
:1099F000406371BDA285280097C0FFFFE780606BC0
:109A000079B597C0FFFFE780E07351B5C16717C50F
:109A1000FF1F03552535F9176307F500B7E7040065
:109A200003A3C7170283828017F3FFFF67008364D5
:109A30001783FFFFE70203692A8408452E89B2894C
:109A400019C900C1971500009385A5866105973057
:109A50000100E780200581447D5A97100000E780CF
:109A6000E03963C7A404814497100000E780003AFE
:109A700063C8A40497C7FF1F9387872F9C43DC47C5
:109A8000B307F94091872302F40063830904832715
:109A9000C900B307F4409587A302F4001C4C89C7A2
:109AA0009C4799C3228582971783FFFF6700C36491
:109AB0005C44139714008504BA972390470171BF43
:109AC0001C48139714008504BA972390070069BFB8
:109AD000832789000547B307F4409587A302F40064
:109AE00083570400638EE7028DC309476384E7044C
:109AF0000D47E395E7FA978701009387E7E21CCCCF
:109B000097870100938747E311A897870100938700
:109B100027A91CCC97870100938787A95CC8BDBF84
:109B2000978701009387C7941CCC97870100938780
:109B30002795EDB7978701009387C7E31CCC9787DC
:109B40000100938727E4D9BF95E51783FFFFE7025C
:109B50000359004618448347940075839D8B63170F
:109B6000F70097100000E78060B448C41783FFFF38
:109B70006700235982801783FFFFE702A3541389EC
:109B80003500C16442094111AA890144F1141359F5
:109B90000901054A2EC697100000E7802026B2452D
:109BA0006348A400014541011783FFFF6700C354C8
:109BB00083A7090013171400BA9783D70700638897
:109BC000B7006394970063742A010504E1B7054563
:109BD000D9BF1783FFFFE702034EAA892E89328B74
:109BE000B6843A8ABE8A97A00000E780C0FE71C999
:109BF000268597200000E780C00C8D4763E7A7000B
:109C00007D551783FFFF6700834E83DB4400971069
:109C10000000E780A0242A8497100000E7804025F8
:109C20009307740031443305850263CDA702971072
:109C30000000E780A02297100000E78020222A84FD
:109C400097100000E780C022930774003144330569
:109C5000850263C3A70497100000E78020209307C4
:109C6000450029A897100000E78080203305850271
:109C70001307F0179307C017E35FA7FA2D55E3C248
:109C800077F963040B02D6865286A6854A8597200B
:109C90000100E780C0BDB5B797100000E780401D08
:109CA000330585029307C5FFD1BF8327490013857C
:109CB000C90083D5270097000000E78000EC61F51C
:109CC00081B769553DBF97C7FF1F2395A70A97C75F
:109CD000FF1F9387E709904381470C463307F50040
:109CE000420741836393B70082805446139847002C
:109CF0008507C2962390E600D5B797C7FF1F9387C5
:109D000027079C4303C58700828017C5FF1F0355A3
:109D1000650682801783FFFFE702633CC1671387F4
:109D2000D7FF630BE502636AA700F1176300F50232
:109D300001451783FFFF6700C33C1387E7FF6302FA
:109D4000E502FD171D8D13351500E5B7975000008E
:109D5000E780602A7D15C5BF97500000E780E0FED0
:109D6000D5BF97500000E78000FDEDB71783FFFFD8
:109D7000E702E3364111AA8401442EC69710000081
:109D8000E780C008B2456348A4000145410117833C
:109D9000FFFF670003379C48131514003E95835757
:109DA0000500E385B7FE0504C9BF03485500814699
:109DB00093F7F60F63E5070181473E85828058459A
:109DC00093975600BA9703D727006316B70003D7B7
:109DD0000700E304C7FE8506E1BF8346450001474F
:109DE0009377F70F63E4D700814711A81C4513163A
:109DF00057000507B29703D60700E313B6FE3E856A
:109E000082801783FFFFE702E32B93170501C187C9
:109E100097CAFF1F938ACAF5635BF00883A70A00FD
:109E2000C0479C4703570400198D42054181636870
:109E3000F500014422851783FFFF6700E32B12051D
:109E40002A94CDBFDC4713944900014A3E948347CE
:109E500044006341FA02014A834754006349FA020D
:109E60008509C20993D9090183A70A009847E3EB42
:109E7000E9FCC1B71C4413195A00A6853E994A85CE
:109E800097000000E780C0EE05E1050AC9B75C4411
:109E900013195A00A6853E994A8597000000E7806D
:109EA00020ED19E1050A4DBFE30C09FA61B7AA8458
:109EB00081495DBF1783FFFFE70263221C452A84A7
:109EC00081E79307C5001CC51C44231204001CC075
:109ED0009307F00F63EDB70093F5F50F22859720F8
:109EE0000000E780C0E51783FFFF6700832193949C
:109EF0000501C167C18063F9F500A6852285972019
:109F00000000E780E0E8C5B7C18193F5F50F228531
:109F100097200000E780A0E2A68522859720000018
:109F2000E780E0E3C9B797C7FF1F938767E48843DB
:109F300082801C4599C797C7FF1F23ABA7E2014545
:109F400082807D55828097C7FF1F938767E2984381
:109F500083474500484792073E9582801783FFFF5D
:109F6000E702E317617100451C183EC6B707800180
:109F70003EC81C183ECA8357440002CE02D002CC11
:109F8000231EF100834784002A8902D22301F102B3
:109F90003C083ED402D697000000E78000FB8357C0
:109FA00005002316F10297500000E78000C8230740
:109FB000A1025C4003556400F18313F71700834747
:109FC000F10252055181F99BD98FA307F102971035
:109FD0000100E780207939CDAA840355050097A0B8
:109FE0000000E78020C083D704002AD26800231C29
:109FF000F10083D72400231DF1001C4803D647003D
:10A000008C4397200000E780A0D08347B400CA8625
:10A01000177601001306463F8117A305F4006C0074
:10A02000481097200100E78080845D611783FFFF5F
:10A030006700230D2155D5BF1C45B1CF03C5A7002F
:10A04000894613576500630BD7028D46630ED7020E
:10A0500085466300D702130740063305E50203C7B0
:10A06000B700418B15CB83C7B700BD8B3355F54087
:10A0700082801375F5031307803EC5B70967137512
:10A08000F50313070771D1BF372709001375F503CF
:10A090001307077CD9B7014582801783FFFFE702CA
:10A0A000030403A98500630C09048347B900AE8447
:10A0B00093F7070E85C303459900930520030D818F
:10A0C0000505B305B5028844610597300100E780B6
:10A0D00080AD35A02E8597000000E78020F62A8409
:10A0E00019CD97000000E780605C8325C900B307A5
:10A0F000B54063FA87002E94B305A440E9F51783B1
:10A10000FFFF6700030085457DBF1783FFFFE70260
:10A1100003FD2A8403D50500011132C636C43AC2B4
:10A120002EC002CA02CC02CE97A00000E78080AB0E
:10A1300082452ACA22852ECC97000000E780E0E005
:10A1400003570500231EE10097500000E780E0ADB3
:10A15000A24632469247230FA10036874C08B286AA
:10A160002285014697000000E780E0A6056117837D
:10A17000FFFF670003F91783FFFFE70243F66171F2
:10A180001C183EC6B70780013EC81C183ECA3C08D2
:10A1900000453ED4AA8402CC02CE02D002D202D61E
:10A1A00097000000E78060DA8357050035592316D1
:10A1B000F10297500000E78040A72307A10209C4DD
:10A1C0008357440081EB21594A855D611783FFFF66
:10A1D000670023F303556400520551819710010075
:10A1E000E78040582A8965D18347B40093F7070E6A
:10A1F00099C71305840197300100E780009D8357BC
:10A200004400231EF100834784002301F1025C40D7
:10A2100003550900D98313F7070883471102231C4C
:10A22000A10093F7F707D98FA300F1028357290004
:10A23000231DF1005C40F18313F717008347F102FF
:10A24000F99BD98FA307F10297A00000E7808099BE
:10A250002AD235D983479400680013975700834763
:10A26000B400FD8BD98FA305F4001C4803D647002A
:10A270008C4397200000E780A0A9A68717770100EC
:10A2800013078718740005464C10268597000000B8
:10A29000E78060942A890DD98347B400A685FD8B99
:10A2A000A305F40097000000E78060DF31BF17834B
:10A2B000FFFFE702C3E2832485FE2A84411126853D
:10A2C00097000000E78080D7834734FF93F7070E9D
:10A2D0008DCB2AC6268597000000E78060C809CD8F
:10A2E000834734FFB245FD8BA309F4FE91C5228557
:10A2F00097300100E780208B41011783FFFF670043
:10A3000043E07DD98327C4FF2685829775F583476F
:10A3100034FF93F7070E91C7228597300100E7803D
:10A32000C08A032584FE97000000E78000E5E9B7B6
:10A330001783FFFFE702A3D79C4141112A8903C776
:10A34000070089472E84935667006380F6040D4604
:10A350006388C6049307F0076304F7022E859720ED
:10A360000000E78060ABAA848149C16B130C4900EF
:10A3700097C7FF1F9387C79F9C43984763E4E904EF
:10A3800041011783FFFF670043D603D74500854788
:10A39000E3F8E7FE2E8597200000E78040ADE1B7A7
:10A3A00003D74500E3FEE7FC2E8597200000E780F9
:10A3B000A0A6AA84228597200000E78000A8C204F6
:10A3C000C98C5DB7DC470355A900139A49003E9A32
:10A3D00093170501C187635DF00083570A006397F7
:10A3E000A70263E774038327CA00034D5A002DA018
:10A3F000A1672167A98F1307F7EFE374F7FE63974F
:10A40000090097000000E780209161FD85098DB764
:10A4100083278A00034D4A00835DA9000357690022
:10A42000216A138BC7003AC6814A33CA4D01631EA5
:10A430005D0197C7FF1F938727949C43E1DBA286AA
:10A440006286814526858297D1B7A1679387F7EF0A
:10A45000930C4BFF63F24703B2455A8597F0FFFF19
:10A46000E780A0710DC103278B00104709CE104370
:10A470006382C4023107D5BFEE8566859700000070
:10A48000E780008F71F993861A0093FAF60F130B89
:10A490000B0271BF835644005C43E3E9F6F6228564
:10A4A0003AC697200000E7802081A1679387D704F0
:10A4B0002A8A035D4400324763E897008347D90046
:10A4C00093E707F8A306F9001C4766852286E28514
:10A4D0008297C1670844FD17337AFA00529508C085
:10A4E0002312A40125B797C7FF1F93876788984356
:10A4F000814715C31447814763FFD50093974500F3
:10A500004C47BE9519C903C7550081476375E600DE
:10A51000DC451606B2973E85828003C74500814719
:10A52000E37BE6FE16069C45F5B71783FFFFE702BF
:10A5300063B9AA892E8A814497CAFF1F938A4A83E6
:10A5400083A70A00984763E6E4001783FFFF6700CC
:10A55000A3BADC471394440001493E9413BB140092
:10A5600083474400634BF900014913BB1400834740
:10A570005400634FF9008504E1B70844931759006C
:10A580005287DA860146A2853E9582990509C9BFA0
:10A590004844931759005287DA860546A2853E95AE
:10A5A00082990509E9B71783FFFFE70243B38145A5
:10A5B00017F5FFFF1305054897B7FF1F239C077A80
:10A5C00097000000E780A0F61783FFFF670063B3E2
:10A5D00097B7FF1F9387C7799C4395C31783FFFFE6
:10A5E000E702E3AF814517F5FFFF1305A544970088
:10A5F0000000E780C0F31783FFFF670083B082800D
:10A600001783FFFFE70203AC37E4040083278412BB
:10A6100041112315E100AE893289368A3A86814696
:10A620000147ED45AA8482972AC621C90356A10095
:10A63000D28597400100E78060288327C413CE8528
:10A6400026858297058905C98327440D2314210196
:10A6500001462C00268582972A8401C9B7E70400A9
:10A6600083A7C712ED4528008297228541011783F1
:10A67000FFFF670063A84944D5B76554FDB75C4147
:10A68000FD175CC182801783FFFFE70243A5B7E790
:10A690000400FC5F829795473305F50281450D81E3
:10A6A0001783FFFF6700E3A51783FFFFE70223A3DC
:10A6B000B7E70400FC5F829795473305F5020D81EB
:10A6C0001783FFFF6700E3A31783FFFFE70223A1C0
:10A6D000B7E7040083A7870B03550500829717830C
:10A6E000FFFF670003A21783FFFFE702439F0355A5
:10A6F00005003287AE861796FF1F0356C6DB97B557
:10A70000FF1F9385A56797000000E780A0EF1783E0
:10A71000FFFF6700039F1783FFFFE702439CB7E734
:10A72000040083A7C71782971783FFFF6700639D05
:10A730001783FFFFE702A39AB7E7040083A78713F5
:10A7400097B5FF1F93858563829701451783FFFFA8
:10A750006700239B1783FFFFE7026398B7E70400B6
:10A7600083A7C71F81451795FF1F0355C5D0829743
:10A770001783FFFF6700E3981783FFFFE702239625
:10A78000B7E7040083A7871397B5FF1F938505607C
:10A79000829701451783FFFF6700A3961783FFFF8A
:10A7A000E702E393B7E7040083A7C71F8145179526
:10A7B000FF1F035545D282971783FFFF67006394FD
:10A7C0001783FFFFE702A3912E8597800000E780A3
:10A7D00080B397800000E78080F01783FFFF670059
:10A7E00043921783FFFFE702838F97800000E78083
:10A7F00080FA1783FFFF6700C3905C49E1175CC9CB
:10A800005CC583572501A1072319F500835705016E
:10A81000A1072318F5008280F1473305F50297B7A9
:10A82000FF1F9387A7589C433E9582808D476315F1
:10A83000F60803D74600854763F0E7081783FFFF54
:10A84000E702E389368536842E8997100000E78079
:10A85000A05C29C98357440093140501C18063E3B8
:10A860009704228597100000E780005BFD142312F7
:10A8700094009307A0026300F5029307B0026307F8
:10A88000F50293079002631FF500228597000100EF
:10A89000E780608901A80146CA85228597A000004B
:10A8A000E78000B41783FFFF6700A3852285971018
:10A8B0000000E7806007FDB7828097B6FF1F938690
:10A8C000264F9C42014599CF9843D44217B6FF1FAB
:10A8D0002320E64E6396D70097B6FF1F23ACE64CC5
:10A8E0001385C7FE82801773FFFFE702437F97003F
:10A8F0000000E780A04B7144330585029145979095
:10A900000000E780C0EC11E565551773FFFF670095
:10A91000437F97B7FF1F23A9A74897000000E78050
:10A92000E04833058502914597900000E78020EAD2
:10A9300061DD97B7FF1F23ABA74697000000E780B4
:10A94000E04697B7FF1F239BA74497000000E780CE
:10A95000E04597B7FF1F2394A7449777010093879B
:10A96000E7AF17B7FF1F232FF74297070000938722
:10A9700007E917B7FF1F2325F742014579B717737A
:10A98000FFFFE702C375AA8517B5FF1F1305054131
:10A9900097100000E780605F1773FFFF6700637622
:10A9A0001773FFFFE702A37397000000E78060FDC5
:10A9B00097100000E780E05E97B7FF1F9387473F3F
:10A9C0009C4391CF1387C7FE19CB83D5C7FF17B51B
:10A9D000FF1F1305653E97200100E780C01C177319
:10A9E000FFFF670003721773FFFFE702436F9700D3
:10A9F0000000E780C0EC09CD834785002A8493F7E7
:10AA0000070499EB0355E50097000000E78080F903
:10AA10001773FFFF6700E36E8347C500930445018A
:10AA200017B9FF1F1309C93885E3832709005CC9DB
:10AA300097B7FF1F23AE973683274900F1FB97B7DF
:10AA4000FF1F23A99736E9B7FD172306F500610517
:10AA500097800000E78060DA8307840063CB0704F7
:10AA60008347840093E707F82304F400B7E7040062
:10AA70009C5F82974205A94741813375F502834760
:10AA8000840093F707FCC98F2304F4008347D400A4
:10AA90003E951C402318A40089CF984319CB8347C7
:10AAA000C4005040814585073305F50242054181C8
:10AAB0000297832709005CC897B7FF1F23AA972E28
:10AAC0008327490089E797B7FF1F23A5972E834760
:10AAD000C4009DDF8355040117B5FF1F1305C52D65
:10AAE00097200100E780200C25B71773FFFFE702CE
:10AAF000035F97B7FF1F938767519C470144858386
:10AB0000858B85E3AE84B2853A8697100000E78096
:10AB1000204F2A8419C597100000E7806045829471
:10AB200008CC22851773FFFF6700A35D1773FFFF33
:10AB3000E702435941112E8932C6AA8997000000C5
:10AB4000E780C031324713060502CA869705000028
:10AB50009385C5CC17B5FF1F13054524970000004A
:10AB6000E780E0F82A8425C99304C5009700000017
:10AB7000E780E0411946AA85268597100000E78006
:10AB800020198545268597100000E7800015177568
:10AB900001001305658A4E958345050026859710AB
:10ABA0000000E780C0195C4831468145A1075CC8B8
:10ABB0005CC483572401E1172319F400835704016F
:10ABC000E1172318F4001C4C3E859770FFFFE780C7
:10ABD0000054A3042501228541011773FFFF67007C
:10ABE000A3511773FFFFE702834F4111AA842EC6BA
:10ABF00032C497100000E780003A004DB24522466B
:10AC0000834784000CC050C093F7F70393E7070411
:10AC10002304F40023180400268597100000E78021
:10AC2000203583479400A9462317A40013D7370083
:10AC300005073307D7029D8B85072306F400A3067B
:10AC4000E40083C70401D8488507230FF7FE17B730
:10AC5000FF1F1307E7155843232A040093074401F5
:10AC600029E317B7FF1F2327F71417B7FF1F232167
:10AC7000F71417B4FF1F1304241422859720010032
:10AC8000E780A0E41C44858B5D8D19E58145228514
:10AC900097200100E78020F141011773FFFF670053
:10ACA00043461CC317B7FF1F2326F710D9B71773E6
:10ACB000FFFFE702C34297050000938565B7014592
:10ACC00097000000E78000B001451773FFFF6700A1
:10ACD00043431773FFFFE702834097000000E780BC
:10ACE00080B01773FFFF6700C3418347C500A5E32A
:10ACF0001773FFFFE702A33E2A840355E500970080
:10AD00000000E78000C821C18347840093F7F7FB68
:10AD10002304F4001C4091C7DC4381C74C4001452B
:10AD2000829797000000E78080B917B5FF1F1305D1
:10AD3000A50897200100E78040E90355E40097004B
:10AD40000000E78020C61773FFFF6700833B828007
:10AD50001773FFFFE702A33897B7FF1F93874705D5
:10AD600097050000938565C817B5FF1F1305C50437
:10AD700023A0070023A2070097200100E78080D2CC
:10AD80001773FFFF6700E3371C4D91CFDC4381CF82
:10AD90001773FFFFE702A3348345070082971773F9
:10ADA000FFFF67000336828097B7FF1F9387070373
:10ADB0009C4303C50700828097B7FF1F9387070254
:10ADC0009C4303C51700828097B7FF1F9387070135
:10ADD0009C4303C52700828097B7FF1F9387070016
:10ADE0009C4303C54700828097B7FF1F938707FFE7
:10ADF0009C4303C53700828097B7FF1F938707FEE8
:10AE00009C4303C55700828097B7FF1F938707FDB8
:10AE10009C4303C56700828097B7FF1F938707FC99
:10AE20009C4303C57700828097B7FF1F938707FB7A
:10AE30009C4303C58700828097B7FF1F938707FA5B
:10AE40009C4303C59700828097B7FF1F938707F93C
:10AE50009C4303C5A700828097B7FF1F938707F81D
:10AE60009C4303C5B70011E11D45828097B7FF1FC2
:10AE70009387C7F69C4303C5C700828097B7FF1F1F
:10AE80009387C7F59C4303C5D700828097B7FF1F00
:10AE90009387C7F49C4303C5E700828097B7FF1FE1
:10AEA0009387C7F39C4303D50701828097B7FF1FA1
:10AEB0009387C7F29C4303C52701828097B7FF1F82
:10AEC0009387C7F19C4303D54701828097B7FF1F43
:10AED0009387C7F09C4303D56701828097B7FF1F14
:10AEE0009387C7EF9C4303D58701828097B7FF1FE5
:10AEF0009387C7EE9C4303C5A701828097B7FF1FC6
:10AF00009387C7ED9C4303C5B701828097B7FF1FA6
:10AF10009387C7EC9C4303C5C701828097B7FF1F87
:10AF20009387C7EB9C4303C5D701828097B7FF1F68
:10AF30009387C7EA9C438857828097B7FF1F938700
:10AF4000E7E99C4303D5C702828097B7FF1F938729
:10AF5000E7E89C4303D5E70219E11305800C8280E2
:10AF600097B7FF1F938787E79C4303C5070382803A
:10AF700097B7FF1F938787E69C43C85B828097B78C
:10AF8000FF1F938727E58843828097B7FF1F93872A
:10AF9000A7E48843828019E17D558280F5DE9842DE
:10AFA00065DFFDD917B7FF1F130747061847AA87A4
:10AFB0007155058B631D072403C507001547E37D05
:10AFC000A7FC03C737001305F0057D171377F70FAC
:10AFD000E364E5FC03C35700E30003FC83C8670098
:10AFE000E38C08FA03C77700494579171377F70F01
:10AFF000E364E5FA03C7A70011481305F7FF1375CB
:10B00000F50FE36BA8F803CE97000D481305FEFF7C
:10B010001375F50FE362A8F803C8B70063090800C9
:10B0200065181378F80F1305600DE36705F703C57E
:10B03000C700794879151375F50FE36FA8F403C8B5
:10B04000D7000D457D181378F80FE36705F503D891
:10B050000701930E40175118420813580801E3EDF9
:10B060000EF303C8E7007D181378F80FE36605F3C5
:10B0700003C827017D181378F80FE36F05F103C8A3
:10B080008700C54E75181378F80FE3E70EF103D863
:10B090006701856E938EBEE06D1842081358080153
:10B0A000E3EC0EEF03D847016D184208135808016E
:10B0B000E3E40EEF03D8870179184208135808011A
:10B0C000E36C05ED03C8A7017D181378F80FE3655D
:10B0D00005ED03C5B7011D487D151375F50FE36D2B
:10B0E000A8EA03C5D701714879151375F50FE36513
:10B0F000A8EA03D5E7011308E00F7D154205418159
:10B10000E36CA8E803C50702494879151375F50FE4
:10B11000E364A8E8C85301C937C8340059151308B7
:10B1200058BFE36BA8E603A8870237C534001305B0
:10B1300055BF5918E36205E717B5FF1F232EC5C891
:10B1400003C6050117B5FF1F232AF5C80545E3759A
:10B15000C5E403D82501D04933760603E31E06E291
:10B1600003C61501E30A06E217B6FF1F2324B6C67D
:10B1700083C5270001466387A50003C61700F14574
:10B180003306B60283C707039305C00272971A07F6
:10B190001307C70516031A9796084697B387B70291
:10B1A00041553E973297420741836362E806177321
:10B1B000FFFFE702C3F2368597800000E780406C0E
:10B1C00097000100E780C04B2A8497A00000E78029
:10B1D000205E2A9497F00000E780002A2A94979036
:10B1E0000000E78040852A9497F0FFFFE780E06F3A
:10B1F0002A9497400000E78000972A9497700000F7
:10B20000E78040A022951773FFFF670083EF8280DD
:10B210001773FFFFE702A3EC4111A307A10097A05A
:10B220000000E78040C99305F100170500001305F1
:10B23000E5B597F0FFFFE780802F014541011773C7
:10B24000FFFF670003EC1773FFFFE702C3E617B4C5
:10B25000FF1F1304A4DB03288400795993681800A6
:10B2600097B4FF1F23A814DB13781800631008029B
:10B27000BA84BE89368B328A2E89AA8A97F0FFFF5C
:10B28000E780E0A77D15269519E531594A851773A2
:10B29000FFFF6700C3E597F0FFFFE78040A67D153D
:10B2A0002695A167E353F5FE97B7FF1F9387070D18
:10B2B00098433E8C814B01CB014597F00000E7801D
:10B2C000C047933B15004A85DA865686D28597900B
:10B2D0000000E78060512A8911CD1C44F99B17B703
:10B2E000FF1F2329F7D283270C00CDD3E3800BFA6D
:10B2F000829769BF268597B7FF1F23AB07D097F0CA
:10B30000FFFFE780809C4146CE8517B5FF1F1305E0
:10B3100065D997300100E780605A97D00000E78038
:10B32000E09C0325040B97D00000E780A0A0054512
:10B3300097D00000E780A0A7054597000000E780B0
:10B3400060EDA9B797B7FF1F938747CC9C47858BC4
:10B35000EDC71773FFFFE70283D817B5FF1F13056B
:10B36000A5D297B7FF1F23A307CA97B7FF1F23A133
:10B3700007CA97B7FF1F23AF07C897200100E780D0
:10B38000C08497500000E78080F997100100E780A3
:10B39000405097100100E780405697B7FF1F9387F2
:10B3A00067C59C4391C7054597800000E780E0236F
:10B3B00097B7FF1F9387C7AD9C4399C741657D151C
:10B3C00097700000E780E0A597F00000E7808041DB
:10B3D00097D00000E780209397B7FF1F938707D887
:10B3E0009C43139717016356070097F00000E7800E
:10B3F000A0B097B7FF1F23A707CA97B7FF1F23A5C2
:10B4000007CA97B7FF1F23A307CA97B7FF1F23A138
:10B4100007CA97000000E780008C97000000E780D3
:10B42000A07597F0FFFFE780401897F00000E780D5
:10B43000E0D91773FFFF6700C3CC828097B7FF1F67
:10B440009387C7BC8843828097B7FF1F938707BC49
:10B45000C8438280B7E7B0009387075063E1A70233
:10B4600097B7FF1F938787BAD843FD576367E500F7
:10B4700097B7FF1F23AEA7B881473E858280B95793
:10B48000EDBF1773FFFFE70283C597800000E780D9
:10B49000607597800000E780C0771773FFFF670033
:10B4A00043C61773FFFFE702E3C12A849304140223
:10B4B00001112E85B289A685214636C63A89973074
:10B4C0000100E780403D0DE9B24638082686CE856A
:10B4D0001305940497500000E780604121462C0832
:10B4E0004A8597300100E780003B13351500056160
:10B4F0001773FFFF670043C00145D5BF1773FFFFF8
:10B50000E702E3BD9305450617B5FF1F1305458DFB
:10B5100097100100E78020691773FFFF670063BE83
:10B520001773FFFFE702A3BB41112EC697F0FFFF81
:10B53000E780C017B24588C141011773FFFF67005C
:10B5400043BC1773FFFFE702E3B7AA842E849780FA
:10B550000000E780006CAA898545228597000000DD
:10B56000E780E07D83C7E4011389940899E3138998
:10B570000403CE85228597000000E780407C2146A9
:10B5800093051902228597000000E780607897B73D
:10B59000FF1F9387A7A78C43228597100000E780A1
:10B5A000C082214693858402228597000000E780AF
:10B5B00020761773FFFF670023B41773FFFFE702BE
:10B5C00083AF397197F00000E780E0B4930540063F
:10B5D00061E997800000E78000606302051497B777
:10B5E000FF1F83C7A78113B7170097B6FF1F2387D5
:10B5F000E680014499CFC16417B9FF1F130909A15F
:10B600009309400EFD1497000000E78020836342F9
:10B61000A40A97F0FFFFE78060094169B729090094
:10B62000096AFD7A2A8B81447D199389F97B130A73
:10B630000A71938A8AC797000000E780208063D749
:10B64000A4041304400EB387840217B7FF1F130727
:10B65000E79B0324070B3E948357C4016382270BA7
:10B6600018403307EB4063EAE9008347440085074D
:10B67000B3874703D6976365F708014681450945B7
:10B6800097F0FFFFE780C04AAA8B29E597400000AA
:10B69000E780808385476317F50689659385057183
:10B6A00017A5FF1F1305C57397100100E780A04F72
:10B6B00095A0B30734030327090BBA9703D7C70133
:10B6C0006308970003C75700A38207002382E7009F
:10B6D000050415BF9305C500228597000000E7808B
:10B6E00080E65E85228697650100938525D697F0D2
:10B6F000FFFFE780404F5E8597100000E780608A7B
:10B70000850415BF97B7FF1F938747909C478D838C
:10B71000858BC1F721611773FFFF6700439D0146C9
:10B720008545094502D002D202D402D697F0FFFF28
:10B73000E7800040AA8479DD97F00000E780E09C74
:10B740001389C4002A8481454A8597000000E78058
:10B75000005F0C4041464A8597000000E780405B4F
:10B76000832944006385090C4E8502D802DA02DC85
:10B7700002DE97300100E780E0382ACE141005463B
:10B780002C0808184ECC97500000E780E00A13758B
:10B79000F50F51ED8355840093E525004A85970008
:10B7A0000000E780E05E11460C104A85970000001B
:10B7B000E78000560146976501009385A5C9268557
:10B7C00097F0FFFFE7802042268597000000E78082
:10B7D000407D5C40A1D3014685450D4597F0FFFFB4
:10B7E000E7800035AA841DD548401389C4009730EE
:10B7F0000100E78020312AC64A8597000000E780D3
:10B80000404C3246636FC5004C404A8597000000AB
:10B81000E780005001468145268597F0FFFFE780CD
:10B82000803C268597000000E780A077E5B583552A
:10B830008400ADB71773FFFFE702638A97A7FF1F66
:10B840009387C77C9C471DC193E7870017A5FF1FFF
:10B850001305055917A7FF1F232EF77A971001002C
:10B86000E78040321773FFFF6700A389DD9B17A7AE
:10B87000FF1F2321F77A97300000E780E0647DF115
:10B8800017A5FF1F1305C55597100100E780E0338A
:10B89000D1BF1773FFFFE70203824169AA892E8A8D
:10B8A000B28A368BBA8B814417ACFF1F130C0C760F
:10B8B000930C400E7D1997F0FFFFE780205863C47A
:10B8C000A40001443DA03384940383270C0B3E94D1
:10B8D0008357C401638627055A87D6865286CE854C
:10B8E0001305040397000000E780E0BB01C9238033
:10B8F0000B0022851763FFFF6700637F8347F40116
:10B9000085C35A87D6865286CE851305940897003C
:10B910000000E78040B909C585472380FB00D1BFFF
:10B92000850451BF835745006380071E1763FFFFDF
:10B93000E702437901112A8497000000E780C04D97
:10B9400009C985476309F50605611763FFFF6700AD
:10B95000A37A97E00000E780007C7DF583574400E0
:10B960004947ED9BE392E7FEC14522859700000021
:10B97000E7804033AA84228597000000E780204FAB
:10B980000357440002CE91472A89631AF7002285A3
:10B9900097000000E780A0513C082ACC3ECE97E0FB
:10B9A0000000E78080765C55C5D374084A86A6857A
:10B9B0000545829751BF03574400D147E3F6E7F8A6
:10B9C000032A0400C169014997AAFF1F938A0A64E8
:10B9D000130B400EFD1997F0FFFFE7802046634FE1
:10B9E000A90E2285032A040097000000E780C042C8
:10B9F000A1452A89228597000000E780A02AAA8411
:10BA0000228597000000E780804A14402A86AA8990
:10BA100078082685CA8597000000E780C0E7AA84D9
:10BA200005D503C7F40189476315F7008347C101B2
:10BA300081DF5546D2851385640097300100E78089
:10BA4000E0E7014597800000E780C01901C583D772
:10BA5000C401A5E797A7FF1F9387475B9C479355B2
:10BA60001900858913D73700058B01CF8983858B12
:10BA70006399B70001452EC697000000E780C0DB40
:10BA8000B2454E8597800000E780601F0346C101E4
:10BA90002A8493751900268597900000E780E03985
:10BAA00035C1268597800000E780E018268511C003
:10BAB000014597800000E780004C97300000E78048
:10BAC000A0408547E312F5E883C754001307F00F41
:10BAD000E38CE7E68507A382F400BDB5B3046903F0
:10BAE00083A70A0BBE9483D7C401638B37015546E5
:10BAF000D2851385640097300100E780C0D955DDF9
:10BB00000509D1BD5DD86DB782801763FFFFE702DD
:10BB1000635B97800000E780000C05C1C1640144AD
:10BB200017A9FF1F1309894E9309400EFD1497F0C2
:10BB3000FFFFE780A030634EA40017A5FF1F130589
:10BB4000252A97100100E780E0031763FFFF6700D5
:10BB5000A35A330534038327090B3E958357C50148
:10BB6000638897002312050097800000E780A00CEF
:10BB7000050475BF97A7FF1F938747499C478D838F
:10BB8000858B8DE31763FFFFE702635517A5FF1F42
:10BB90001305052597100100E78020031763FFFFB9
:10BBA0006700235682801763FFFFE7024353970520
:10BBB00000009385C5A017A5FF1F130565229710E8
:10BBC0000100E78020EE1763FFFF670083531763D0
:10BBD000FFFFE702C3508841B7E70400BC5B0505DF
:10BBE00042054181829709C585472300F500050577
:10BBF0001763FFFF6700E35083C7F5FF2E858507B6
:10BC0000A38FF5FE828083C7F5FFFD1793F7F70F2B
:10BC1000A38FF5FE99EF1763FFFFE702434CB7E7E9
:10BC20000400BC571385F5FF82971763FFFF670079
:10BC3000434D82801C41035745008D8FBA951CC12E
:10BC40002312B5003E85828093D78500A20514415A
:10BC5000DD8D835745001387E6FF18C1890723123E
:10BC6000F50013D685004111238FB6FEA38FC6FEC3
:10BC70004101828018419307F7FF1CC1835745009B
:10BC800085072312F500A30FB7FE82808357450076
:10BC90008D8F2312F5001C41BE950CC12E8582802C
:10BCA000AA8703D7470008410D8FAA952392E70082
:10BCB0008CC38280184108453305A7408280835792
:10BCC0004500035765001D8F1C4108453385A7407B
:10BCD0003305A74082801763FFFFE702434041110D
:10BCE0002EC62A8497000000E780A0FDB24563734A
:10BCF000B50001A0835744000840BE952312B4004C
:10BD00003E9541011763FFFF6700A33F1763FFFFE5
:10BD1000E702E33C41112E84B28532C69700000051
:10BD2000E780A0FB3246A28597300100E78000B98A
:10BD300041011763FFFF6700C33C1763FFFFE70282
:10BD4000033A2E84854597000000E78000F9230020
:10BD500085001763FFFF6700C33A1763FFFFE70221
:10BD6000033841112317B100894597000000E7808F
:10BD7000C0F68347E1002300F5008347F100A300EC
:10BD8000F50041011763FFFF6700A3371763FFFF4B
:10BD9000E702E33493D78500A2054111DD8D231717
:10BDA000B100894597000000E78020F38347E10058
:10BDB0002300F5008347F100A300F500410117635C
:10BDC000FFFF670003341763FFFFE7024331139758
:10BDD000850193D78501C166938606F0D98F13D765
:10BDE0008500758FD98FA2053707FF00F98D4111A6
:10BDF000DD8D2EC6914597000000E78000EE6C00B7
:10BE0000114697300100E78060AB41011763FFFFE7
:10BE10006700232F1763FFFFE702632C1C41854552
:10BE200003C4070097000000E78080E622851763BF
:10BE3000FFFF6700032D1763FFFFE702432A1C4142
:10BE40004111894503C7070083C717002307E10095
:10BE5000A307F10097000000E78080E30355E100AD
:10BE600041011763FFFF6700C3291763FFFFE70264
:10BE700003271C414111894503C7070083C71700E9
:10BE80002307E100A307F10097000000E78040E0EE
:10BE90008357E100410113D58700A2075D8D42055C
:10BEA00041811763FFFF6700C3251763FFFFE702A8
:10BEB00003230C4141112A84114668009730010088
:10BEC000E780C09F9145228597000000E78040DC15
:10BED000B247C166938606F01397870113D5870191
:10BEE000598D13D78700758F598DA2073707FF002B
:10BEF000F98F5D8D41011763FFFF670083201C45AB
:10BF0000BE950CC18280AE87944391E6584101EF03
:10BF10000CC15CC1828003C7570013671700A3825E
:10BF2000E700B687D5B70CC3EDB7AA87084119CD8E
:10BF30001841D44398C36313D500D8C32A87034656
:10BF400057009376160081E62320070082809443F1
:10BF500081CA8C4203A847008CC363930601CCC3FB
:10BF6000799A14C3A302C7003687D1BF1C45DC47AA
:10BF70001D8DB777DBB6938777DB09853305F5022F
:10BF8000420541818280F147B385F50248452E95EF
:10BF900082808347450085072302F500828017636E
:10BFA000FFFFE702C3132A8409E41763FFFF67005A
:10BFB000431583474400F5DBFD1793F7F70F230282
:10BFC000F400E5F71C4403D7270005072391E70099
:10BFD000DC4399C3228582974C4889CD834754001E
:10BFE000898B99E71C4422859C479C439C478297F8
:10BFF000232A04000040232004007DB71763FFFFBD
:10C00000E702E30D8357250041112EC681EB014461
:10C01000228541011763FFFF6700A30E0357050048
:10C020008147F146E305F7FEB385D7024045850712
:10C030002E948345440008C4F5F5B247AA8481E7ED
:10C04000232A040009A81C456C0022859C439C43BC
:10C05000829748C84DDD85472312F400B24723205C
:10C060000400231804002319F4005C485CC483D73F
:10C070002400FD172391F40061BF1763FFFFE7025F
:10C08000030697A7FF1F9387A7D78843232605009A
:10C0900023240500410597100100E78000B31763D2
:10C0A000FFFF670003061763FFFFE702430317A4C0
:10C0B000FF1F1304E4D41C40411199CF9C47230077
:10C0C000B5002AC65CC197000000E78040FB1C4019
:10C0D000DC4399C33245829741011763FFFF670034
:10C0E00043020347450029E3584DAA877D551DCFDC
:10C0F0001763FFFFE702A3FE1CC3DC4797A6FF1FE1
:10C1000023A0E6D0F156130507012390D700970529
:10C1100000009385050297100100E780A098014573
:10C120001763FFFF6700E3FD7D5582808280176300
:10C13000FFFFE702C3FA01116146814528009760BD
:10C14000FFFFE780C0FC97A7FF1F938767CB9C4347
:10C1500028009305F00FDC473EC697000000E780FB
:10C16000C0F405611763FFFF6700A3F997A7FF1FDE
:10C17000938707C99C43D847A1679387C702631E6B
:10C18000F70A397106DE22DC26DA80004AD84ED65C
:10C1900052D456D23285B28497000000E780C0C7DF
:10C1A000AA89268597000000E78020C92318A4FCEF
:10C1B000268597000000E78040C82319A4FC268547
:10C1C00097000000E78060C783D744000A8A231ADB
:10C1D000A4FC858393F7F70F230EF4FC8607BD07B5
:10C1E00093F7073F3301F1408A8A01498347C4FD31
:10C1F0006367F902CE85130584FC232C54FD970058
:10C200000000E78080EA5281130104FCF25062547E
:10C21000D2544259B259225A925A216182802685BB
:10C2200097000000E78060C193171900D6970509B1
:10C230002390A7001379F90F55BF828097A7FF1F9E
:10C24000938707BC9C43D847A1679387A702631ACB
:10C25000F70A397106DE22DC26DA80004AD84ED68B
:10C2600052D456D23285B28497000000E780C0BA1B
:10C27000AA89268597000000E78020BCFD57231877
:10C28000A4FC26852319F4FC97000000E780E0BA9F
:10C2900083D744000A8A231AA4FC858393F7F70FF7
:10C2A000230EF4FC8607BD0793F7073F3301F140E7
:10C2B0008A8A01498347C4FD6367F902CE85130565
:10C2C00084FC232C54FD97000000E78000DE52819F
:10C2D000130104FCF2506254D2544259B259225A0A
:10C2E000925A21618280268597000000E780E0B4A1
:10C2F00093171900D69705092390A7001379F90F12
:10C3000055BF828097A7FF1F938787AF9C43D8476D
:10C31000A16789076310F70A397106DE22DC26DA85
:10C3200080004AD84ED652D456D2328532899700F0
:10C330000000E78060AEAA894A8597000000E78088
:10C34000C0AF835749000A8A2318A4FC858393F75A
:10C35000F70F230CF4FC8607BD0793F7073F330163
:10C36000F1408A8A8144834784FD63E7F402CE85E5
:10C37000130584FC232A54FD97000000E780E0D2D7
:10C380005281130104FCF2506254D2544259B25902
:10C39000225A925A216182804A8597000000E780E4
:10C3A000C0A993971400D69785042390A70093F40F
:10C3B000F40F55BF828097A7FF1F938767A49C4304
:10C3C000D847A1679387E704631EF70A397106DE31
:10C3D00022DC26DA80004AD84ED652D456D2328594
:10C3E000B28497000000E78020A3AA8926859700E1
:10C3F0000000E78080A42318A4FC26859700000095
:10C40000E780A0A3231AA4FC268597000000E780FC
:10C41000C0A283D744000A8A2319A4FC858393F71A
:10C42000F70F230EF4FC8607BD0793F7073F330190
:10C43000F1408A8A01498347C4FD6367F902CE85CA
:10C44000130584FC232C54FD97000000E780E0C511
:10C450005281130104FCF2506254D2544259B25931
:10C46000225A925A21618280268597000000E78037
:10C47000C09C93171900D69705092390A70013793C
:10C48000F90F55BF828097A7FF1F938767979C433B
:10C49000D847A1679387C704631AF70A397106DE84
:10C4A00022DC26DA80004AD84ED652D456D23285C3
:10C4B000B28497000000E7802096AA89268597001D
:10C4C0000000E7808097FD572318A4FC2685231AD7
:10C4D000F4FC97000000E780409683D744000A8A66
:10C4E0002319A4FC858393F7F70F230EF4FC86072A
:10C4F000BD0793F7073F3301F1408A8A014983471B
:10C50000C4FD6367F902CE85130584FC232C54FD1A
:10C5100097000000E78060B95281130104FCF250DB
:10C520006254D2544259B259225A925A216182809D
:10C53000268597000000E780409093171900D69752
:10C5400005092390A7001379F90F55BF828097A79B
:10C55000FF1F9387E78A9C43D847A167DD076317CE
:10C56000F7041763FFFFE70283B7797132853284DE
:10C5700097000000E780408A2AC6228597000000C5
:10C58000E780A08B2311A102228597000000E7809D
:10C59000A088B2452300A102280897000000E78088
:10C5A000C0B045611763FFFF6700A3B5828097A7FE
:10C5B000FF1F9387E7849C43D847A167938787042D
:10C5C0006317F7041763FFFFE70263B179713285E0
:10C5D000328497000000E78020842AC622859700D5
:10C5E0000000E78080852311A102228597000000CA
:10C5F000E7808082B2452300A1022808970000004E
:10C60000E780A0AA45611763FFFF670083AF8280C0
:10C610009797FF1F9387C77E9C43D847A16793874F
:10C62000A7046312F7021763FFFFE70243AB011190
:10C630002800814597000000E78020A70561176367
:10C64000FFFF670003AC82809797FF1F9387477BAC
:10C650009C43D847A167938757026319F702176372
:10C66000FFFFE702C3A70111328597F0FFFFE780C4
:10C67000A07A2308A1008145280097000000E780E8
:10C68000C0A205611763FFFF6700A3A78280979789
:10C69000FF1F9387E7769C43D847A1679387E702FC
:10C6A000631BF7041763FFFFE70263A301113285E1
:10C6B000328497F0FFFFE7804078AA84228597F0C4
:10C6C000FFFFE7808077854709E9228597F0FFFF24
:10C6D000E78080744205B337A00028008145231805
:10C6E00091003ECA97000000E780209C0561176317
:10C6F000FFFF670003A182809797FF1F9387477012
:10C700009C43D84799476313F7081763FFFFE70275
:10C71000039D79713285328497F0FFFFE780C06F07
:10C720002AC6228597F0FFFFE78020712310A1021F
:10C73000228597F0FFFFE780206E2301A10222856A
:10C7400097F0FFFFE780406DA301A102228597F0DB
:10C75000FFFFE780606C2302A102228597F0FFFFB4
:10C76000E780806B2313A102228597F0FFFFE7800B
:10C77000A06AB2452314A102280897000000E780B0
:10C78000C09245611763FFFF6700A3978280979768
:10C79000FF1F9387E7669C43D847A1679387C7032A
:10C7A0006313F7081763FFFFE7026393797132851C
:10C7B000328497F0FFFFE78020662AC6228597F033
:10C7C000FFFFE78080672310A102228597F0FFFF1B
:10C7D000E780A0662311A102228597F0FFFFE78082
:10C7E000A0632302A102228597F0FFFFE780C062C9
:10C7F000A302A102228597F0FFFFE780E0612303F7
:10C80000A102228597F0FFFFE7800061B245A303F4
:10C81000A102280897000000E7802089456117637E
:10C82000FFFF6700038E82801763FFFFE702238B01
:10C8300001112A8497F0FFFFE780005EAA84228519
:10C8400097F0FFFFE780605F228597F0FFFFE780AA
:10C85000C05E035744008D4763F7E700228597F0D9
:10C86000FFFFE780805D228597F0FFFFE780E05CB7
:10C870002800A68597000000E780208305611763E4
:10C88000FFFF670003889797FF1F938767579C43B5
:10C89000D847A167FD07631FF7001763FFFFE70293
:10C8A0000384328597000000E78040F81763FFFF9C
:10C8B0006700238582809797FF1F938767549C4367
:10C8C000D847A167E5076315F7081763FFFFE7027D
:10C8D000038179713285328497F0FFFFE780C0537E
:10C8E0002AC6228597F0FFFFE7802055228597F022
:10C8F000FFFFE78080542310A102228597F0FFFFFD
:10C90000E780A053520551812311A1022285230201
:10C91000010297F0FFFFE7802050A302A1022285C9
:10C9200097F0FFFFE780404F2303A102228597F095
:10C93000FFFFE780604EB245A303A102280897F0ED
:10C94000FFFFE780807645611753FFFF6700637B39
:10C9500082809797FF1F9387A74A9C43D847A16778
:10C960009387E703631FF7001753FFFFE70223775F
:10C97000328597000000E78060EB1753FFFF6700E8
:10C98000437882809797FF1F938787479C43D847B8
:10C99000A16793874704631EF7021753FFFFE7025F
:10C9A000037479713285328497F0FFFFE780C046C7
:10C9B0002AC6228597F0FFFFE7802048B245280865
:10C9C00097F0FFFFE780606E45611753FFFF670038
:10C9D000437382809797FF1F938787429C43D84772
:10C9E000A167938787026310F7041753FFFFE702DD
:10C9F000036F79713285328497F0FFFFE780C04181
:10CA00002AC6228597F0FFFFE7800041B245230048
:10CA1000A102280897F0FFFFE780206945611753BE
:10CA2000FFFF6700036E82801753FFFFE702236B4F
:10CA3000011197F0FFFFE780203EAA85280097F0BC
:10CA4000FFFFE780806605611753FFFF6700636B98
:10CA50009797FF1F9387C73A9C43D847A167D10791
:10CA6000631FF7001753FFFFE702636732859700E4
:10CA70000000E780A0FB1753FFFF670083688280F8
:10CA80009797FF1F9387C7379C43D847A167C50770
:10CA9000631FF7001753FFFFE702636432859700B7
:10CAA0000000E780A0F81753FFFF670083658280CE
:10CAB0009797FF1F9387C7349C43D847A167B9074F
:10CAC000631FF7001753FFFFE7026361328597008A
:10CAD0000000E780A0F51753FFFF670083628280A4
:10CAE0009797FF1F9387C7319C43D847A167AD072E
:10CAF000631FF7001753FFFFE702635E328597005D
:10CB00000000E780A0F21753FFFF6700835F828079
:10CB10009797FF1F9387C72E9C43D8478947631871
:10CB2000F7021753FFFFE702835B0111328532C81A
:10CB300097F0FFFFE780402EAA85280097F0FFFFBF
:10CB4000E780A05605611753FFFF6700835B828073
:10CB50009797FF1F9387C72A9C43D847A1678D07E4
:10CB60006311F7041753FFFFE70263570111328582
:10CB7000328497F0FFFFE780202A13066100AA8421
:10CB80004C00228597300000E780C0232800A6854E
:10CB900097F0FFFFE780605105611753FFFF6700C3
:10CBA000435682809797FF1F9387C7259C4381CF69
:10CBB000DC4391CB1753FFFFE70263528297175371
:10CBC000FFFF6700035482801753FFFFE7022351E2
:10CBD00079713C08AE843ED2A165B7070A002A8469
:10CBE0003ED448103C08DD053ED636C432C63AC2B3
:10CBF00097D0FFFFE780402C12474810BA8597F086
:10CC0000FFFFE780C01332464810B28597F0FFFF60
:10CC1000E780E014A2464810B68597F0FFFFE78052
:10CC20000012501001478146A685228597D0FFFF4C
:10CC3000E780E04D45611753FFFF6700834C1753B2
:10CC4000FFFFE702C34901117C000329C501AE843F
:10CC50003ECAA165B70707002A843ECC48087C007D
:10CC6000C5053ECE97D0FFFFE78000258345D9005C
:10CC7000480897F0FFFFE780800C50080147814685
:10CC8000A685228597D0FFFFE7806048056117538E
:10CC9000FFFF670003471753FFFFE702434483C7C3
:10CCA000950093F7F707A384F50097000000E7804D
:10CCB00040F91753FFFF6700C3441753FFFFE70214
:10CCC000034279713C08AE843ED2A165B7070900E2
:10CCD0002A843ED448103C08938545043ED632C68B
:10CCE00036C497D0FFFFE780201DA2464810B685C6
:10CCF00097F0FFFFE780A00432464810B28597F016
:10CD0000FFFFE780C005501001478146A6852285B8
:10CD100097D0FFFFE780A03F45611753FFFF6700F3
:10CD2000433E1753FFFFE702833B83C79500411142
:10CD30002A8493F7F707A384F50032852EC697F06F
:10CD4000FFFFE780800F85672AC46370F502977044
:10CD50000000E78020E92246B24509ED11478146EF
:10CD6000228597000000E78060E641011753FFFF2E
:10CD70006700233901478346F501DDB71753FFFFED
:10CD8000E702433401113C003ECAB7070A003ECC1B
:10CD90003C003ECE83C79500AA89328593F7F707FA
:10CDA000A384F5002E8497F0FFFFE78000098567D4
:10CDB000637DF504A165AA8493858504480897D00E
:10CDC000FFFFE780600F268597700000E78080E115
:10CDD0002A8929E19145480897F0FFFFE78020F66E
:10CDE000A685480897F0FFFFE78060F7CA854808E6
:10CDF00097F0FFFFE780A0F4014781465008A28525
:10CE00004E8597D0FFFFE780803005611753FFFF05
:10CE10006700832E8145480897F0FFFFE78020F2E6
:10CE20000349090275BF1753FFFFE702A329797170
:10CE30001C103ECAB7070F003ECC404D1C10AA8400
:10CE4000AE894808994532C636893ECE97D0FFFF55
:10CE5000E780800632464808B28597F0FFFFE780FA
:10CE600000EE630C0902A545480897F0FFFFE78034
:10CE7000C0E62546CA8597200100E78020A4500817
:10CE800001478146CE85268597D0FFFFE780202881
:10CE900045611753FFFF670023268355C4024808E6
:10CEA00097F0FFFFE780A0EB0355E402814505C53D
:10CEB000854785456301F502C167FD179305F00FAE
:10CEC000630BF5007D1597700000E780208E9305B9
:10CED000150093F5F50F480897F0FFFFE78020E66F
:10CEE00083450403480897F0FFFFE78040E583454A
:10CEF0001403480897F0FFFFE78060E4835524039C
:10CF0000480897F0FFFFE78080E583554403480811
:10CF100097F0FFFFE780A0E49DB71753FFFFE702FC
:10CF2000031C83C795008146014693F7F707A38446
:10CF3000F50097000000E78040EF1753FFFF670000
:10CF4000431C1753FFFFE702831979713E841C10BD
:10CF50003ECA2E89B7070F00A1653ECCFD051C1007
:10CF6000AA84480842C03AC23ECE36C432C697D0E0
:10CF7000FFFFE78060F432464808B28597F0FFFF74
:10CF8000E780E0DBA2464808B68597F0FFFFE78020
:10CF900000DD12474808BA8597F0FFFFE78020DCE4
:10CFA0000248630C08029145480897F0FFFFE780AC
:10CFB000C0D21146A28597200100E780209050083A
:10CFC00001478146CA85268597D0FFFFE780201458
:10CFD00045611753FFFF6700C3128945480897F062
:10CFE000FFFFE78080CF834704002300F5008347DD
:10CFF0001400A300F500E1B71753FFFFE702830C0D
:10D0000083C7950001112A8A93F7F707A384F500D7
:10D010003285AE8432C697F0FFFFE78000E23246E9
:10D020002A89328597F0FFFFE78000DF8567637309
:10D03000F902AA894A8597700000E780A0BA2A847D
:10D0400019ED114781464A86A68552859700000052
:10D05000E780C0B705611753FFFF6700E3099387B7
:10D06000E9FF93F7F70F0547E366F7FE8347F501FE
:10D0700095EB8947E380F9FE8346F4015285014729
:10D080004A86A68597000000E78040B4A167D907CB
:10D0900048083ECC230A010002CE97000000E7803A
:10D0A000A0B04DBF639EE7008947639EF9009307D8
:10D0B0001020231FF50097700000E780C0B76DBFF8
:10D0C0000947E39BE7FA8D47E398F9FA22859770C1
:10D0D0000000E78080DF9797FF1F9387A7F19C43AD
:10D0E00099E79797FF1F9387A7DA9C4399C703D5C2
:10D0F000040097800000E780A0CE231F0400228553
:10D100005DBF1753FFFFE70283FD01113C003ECADC
:10D11000B7070B003ECC3C003ECE83C795002A8962
:10D12000328593F7F707A384F500AE8497F0FFFFED
:10D13000E780A0D093170501C187635AF006A16567
:10D140002A849385E502480897D0FFFFE780C0D680
:10D15000A285480897F0FFFFE78060C09797FF1F00
:10D16000938707D39C43A9EB01449375F40F4808B8
:10D1700097F0FFFFE780A0BC9355844093F5F50F2F
:10D18000480897F0FFFFE78080BB9355044193F573
:10D19000F50F480897F0FFFFE78060BA0147814626
:10D1A0005008A6854A8597D0FFFFE78040F60561C5
:10D1B0001753FFFF6700E3F4416585460546A285E6
:10D1C0007D1597500000E78060BD59DD510597003F
:10D1D0000100E780808F130440063344850271B755
:10D1E0001753FFFFE702A3EF0111B70706003EC682
:10D1F00083C7950021642A8993F7F707A384F50074
:10D20000AE8428009305A4040AC40AC897D0FFFF7F
:10D21000E78080CA300001478146A6854A8597D0BD
:10D22000FFFFE780C0EE97E0FFFFE780E011130407
:10D230009404480822CC230A010002CE9700000083
:10D24000E780809605611753FFFF670083EB175354
:10D25000FFFFE70223E7C1642A8901449799FF1F72
:10D260009389C9DA130A8002FD1497E0FFFFE78073
:10D27000E0BD6347A40001451753FFFF6700C3E704
:10D28000B307440303A7C90ABA9703D70700630685
:10D29000970083D72700638427010504F9B7054564
:10D2A000E1BF1753FFFFE702E3E12A8A2E8999C104
:10D2B00023A0050081498144979AFF1F938ACAB42D
:10D2C000614B97E0FFFFE780A0BE63C7A4004E85D7
:10D2D0001753FFFF670043E23384640383A70A0008
:10D2E0003E948357040099E76304090023208900D2
:10D2F0008504C1BF4146D285130544009710010043
:10D30000E780605975F5A289E5B71753FFFFE7027B
:10D3100063DB39717C083ED4B7070A003ED67C082F
:10D320003ED883C795002A8A328593F7F707A384EE
:10D33000F5002E8932C697F0FFFFE78000B08567C1
:10D340006373F5083246AA84328597F0FFFFE780C1
:10D35000A0AC8547AA8963E8A706A16593858504E3
:10D36000281097D0FFFFE78020B526859770000032
:10D37000E78040872A8429ED9145281097F0FFFF28
:10D38000E780E09BA685281097F0FFFFE780209DAF
:10D39000CE85281097F0FFFFE780609A014781460D
:10D3A0003010CA85528597D0FFFFE78040D6A1672D
:10D3B0009387770448183EDC230A010202DE97F0C7
:10D3C000FFFFE780607E21611753FFFF6700C3D234
:10D3D0008145281097F0FFFFE7806096A68528100A
:10D3E00097F0FFFFE780A0979797FF1F9387C7F8F5
:10D3F0009C4381CB22856389090097D00000E78098
:10D4000040248345040271B797D00000E780C02212
:10D41000CDBF1753FFFFE702E3CA83C79500411151
:10D42000AA8993F7F707A384F5003285AE84328A80
:10D4300097F0FFFFE78060A08567637FF5022A8988
:10D4400097600000E780007A2A84914631C58347BF
:10D45000F50105476387E70291C70D476366F70447
:10D46000AD461DA89305050303250A004146971004
:10D470000100E78040420DE941011753FFFF6700BB
:10D48000A3C79305950803250A004146971001009C
:10D49000E7806040814669F54A86A6854E859700FB
:10D4A0000000E780C081C9BF83250A0013059408E6
:10D4B00097700000E780A02919C1C146F1BF979776
:10D4C000FF1F938727B39C4399E79797FF1F938785
:10D4D000279C9C4399C7228597800000E780208A7B
:10D4E00069FD8547A30FF400228597B00000E7800F
:10D4F0006084228597600000E780E0734E85814656
:10D500004A86A68597F0FFFFE780607BA167938737
:10D51000570448003EC42302010002C697F0FFFFF3
:10D52000E780806891BF1753FFFFE702C3B883C746
:10D5300095004111AA8993F7F707A384F500328576
:10D540002E89B28A97F0FFFFE780208F856763748A
:10D55000F50EAA8497600000E780C0682A840DED6C
:10D56000416B014A979BFF1F938B4BAA130C400EF4
:10D570007D1B19A833048A0383A70B0B3E948357A2
:10D58000C40163836705050A97E0FFFFE780008B0E
:10D59000E342AAFE95460DA08357C5016396970204
:10D5A0009305050303A50A00414697100100E78093
:10D5B000802E994611E181462686CA854E8597F0D0
:10D5C000FFFFE780C06F85A883A50A001305040349
:10D5D00097700000E780A017C14679FD2285231EC1
:10D5E000940097A00000E780E07422859760000017
:10D5F000E78060649797FF1F938707D89C43A9C370
:10D6000023000402228597D00000E78040F04E8579
:10D6100081462686CA8597F0FFFFE780406AA167AA
:10D620009387070448003EC42302010002C697F016
:10D63000FFFFE780605741011753FFFF670023ABEF
:10D6400089472300F402E1B7397106DE22DC4AD8AB
:10D65000800052D456D25AD026DA4ED65ECE2E8ACA
:10D6600032892A8B97D0FFFFE780407A0605710543
:10D6700041998A8A3301A140232224FC231404FC0B
:10D6800097D0FFFFE780807883479A00060535052D
:10D6900093F7F7072315A4FCA304FA004A85232671
:10D6A00024FC97E0FFFFE780407993170501C187CD
:10D6B0006340F0025681130104FCF2506254D254CC
:10D6C0004259B259225A925A025BF24B216182802E
:10D6D000AA844A8597E0FFFFE7802076AA894A85D9
:10D6E00097E0FFFFE7806075A1659385C5022A89F1
:10D6F000130544FC97C0FFFFE780007C268597C098
:10D70000FFFFE7804070854511C94A86CE8597C0E6
:10D71000FFFFE780C069AA8B21E98945130544FC16
:10D7200097E0FFFFE780A061A685130544FC97E022
:10D73000FFFFE780C062CE85130544FC97E0FFFF42
:10D74000E780E061CA85130544FC97E0FFFFE780AE
:10D75000006101478146130644FCD2855A8597D063
:10D76000FFFFE780C09AB9B78145130544FC97E0F5
:10D77000FFFFE780C05CA685130544FC97E0FFFF30
:10D78000E780E05DCE85130544FC97E0FFFFE7806E
:10D79000005DCA85130544FC97E0FFFFE780205C2D
:10D7A000814497D0FFFFE7806066E3D4A4FA83A7A3
:10D7B0000B0113971400BA9783D5070099C5130579
:10D7C00044FC97E0FFFFE78080598504D9BF797159
:10D7D00006D622D44AD000184ECE52CC56CA26D2F3
:10D7E0005AC8AE893289AA8A97D0FFFFE7800062C3
:10D7F0000605690541990A8A3301A140232A24FCC0
:10D80000231C04FC97D0FFFFE780406083C799008A
:10D8100006052D0593F7F707231DA4FCA384F90043
:10D820004A85232E24FC97E0FFFFE78000619317D1
:10D830000501C187634FF0005281130104FDB2500E
:10D84000225492540259F249624AD24A424B4561EB
:10D850008280AA844A8597E0FFFFE780005EA16589
:10D860009385A5022A89130544FD97C0FFFFE78031
:10D87000A064268597C0FFFFE780E058854509C969
:10D88000CA8597C0FFFFE78080552A8B29E189452B
:10D89000130544FD97E0FFFFE780604AA685130566
:10D8A00044FD97E0FFFFE780804BCA85130544FDE8
:10D8B00097E0FFFFE780A04A01478146130644FD39
:10D8C000CE85568597D0FFFFE7806084B5B7814548
:10D8D000130544FD97E0FFFFE7806046A68513052A
:10D8E00044FD97E0FFFFE7808047CA85130544FDAC
:10D8F00097E0FFFFE780A046814497D0FFFFE780D5
:10D90000E050E3DBA4FA83270B0113971400BA97C6
:10D9100083D5070099C5130544FD97E0FFFFE78015
:10D9200000448504D9BF1743FFFFE702437B8347C9
:10D930004500404DD5EFFD575DC48346940009472F
:10D940006363D70A0346B400854663EEC6088306C0
:10D95000E40063CA06085C45F9562390D700978710
:10D96000FF1F83C7A74A99E3A304E4009787FF1F1B
:10D97000938707529C4381E78947A306F400979752
:10D98000FF1F9387679F9C4381E789472306F40025
:10D990009705000093854506AA841305040197F0B6
:10D9A0000000E7802010FD57231AF40281471CDC99
:10D9B00001489787FF1F23A787449787FF1F9387F7
:10D9C000A744232E040304C0804397D0FFFFE780C1
:10D9D000204E61463306C502814522859740FFFFF0
:10D9E000E780E07281473E851743FFFF6700637160
:10D9F000FD57D5BF1743FFFFE702636E2A84035527
:10DA0000450297600000E780E01D19E5231E040031
:10DA10001743FFFF6700E36E8357E401F5DB9305CF
:10DA200004FF174501001305A5DC97E00000E7801F
:10DA3000E014F9BF1743FFFFE702636A2E89A1656F
:10DA400041119385E5032A8436C432C6BE843AC2A6
:10DA500097C0FFFFE780404612472285BA8597E0CE
:10DA6000FFFFE780C02D32462285B28597E0FFFF99
:10DA7000E780E02EA2462285B68597E0FFFFE7808B
:10DA8000002E630309029145228597E0FFFFE7809E
:10DA9000C0241146A68597100100E78020E24101CD
:10DAA0001743FFFF6700E3658945228597E0FFFF85
:10DAB000E780A02283C704002300F50083C7140079
:10DAC000A300F500E9BF1743FFFFE702436183C7E7
:10DAD0009500444D054793F7F707A384F5001C42D2
:10DAE000411183C707006367F7062E842A89B1C0F6
:10DAF00003C7D400630FF7021787FF1F13074739C7
:10DB0000184305C3A386F40097A00000E780404AAD
:10DB100083C7D40099E741657D1597400000E780F1
:10DB2000403083D72403918B89C797E00000E780BA
:10DB3000C0134A85A28597F0FFFFE7808010A16798
:10DB4000C10748003EC42302010002C697F0FFFF50
:10DB5000E780800541011743FFFF6700835A1743A1
:10DB6000FFFFE702C35703D745008D47AA84411141
:10DB70002E8432892E8563E3E70297E0FFFFE7807A
:10DB8000C02BAA8523000900268597C0FFFFE780E8
:10DB9000002541011743FFFF6700A35697E0FFFFF1
:10DBA000E780A0292AC6228597E0FFFFE780E028CA
:10DBB000B24585472A862300F900268597C0FFFFD6
:10DBC000E780E01EF9B7397106DE22DC26DA800034
:10DBD0004ED652D456D24AD85AD05ECEAE89B284EE
:10DBE000AA8A97D0FFFFE78060210605130525026A
:10DBF00041990A8A3301A140232224FC231404FC06
:10DC000097D0FFFFE780801F83C7990006054D0569
:10DC100093F7F7072315A4FCA384F9002685232690
:10DC200024FC97E0FFFFE780402193170501C1879F
:10DC30006340F0025281130104FCF2506254D2544A
:10DC40004259B259225A925A025BF24B21618280A8
:10DC5000AA8B03AB040097C0FFFFE780C01A51E511
:10DC600083D7440001498544F11793B71700A301F6
:10DC7000F4FC834734FCA165C9C79385E50413050B
:10DC800044FC97C0FFFFE7802023A685130544FCD2
:10DC900097E0FFFFE780A00ADE85130544FC97E0CC
:10DCA000FFFFE780C00B834734FC114691E3094630
:10DCB000DA85130544FC97E0FFFFE78060058144A7
:10DCC000630A0900416B7D1B97D0FFFFE7800013BB
:10DCD00063CCA40201478146130644FCCE855685D9
:10DCE00097C0FFFFE780A042B1B7A685130634FCBA
:10DCF00097000000E780E0E6933415002A89860447
:10DD00008DBF9385C504A5BF8327C9001397140051
:10DD1000BA9783D5070063886501130544FC97E033
:10DD2000FFFFE780C003850445B71743FFFFE70205
:10DD3000833879711C103EC4B7070F003EC61C1013
:10DD40003EC883C79500AA8A328593F7F707A38454
:10DD5000F500AE89328497E0FFFFE780000E93174D
:10DD60000501C187635AF0062A8A228597E0FFFFE2
:10DD7000E780A00C2A895285032B040097C0FFFF7F
:10DD8000E780600839ED8357440081440544F1176A
:10DD900093B71700A303F10083457100DA87228748
:10DDA000CA865286280097000000E780E0C8014735
:10DDB00081463000CE85568597C0FFFFE78020352D
:10DDC000A1679387D70348083ECC230A810026CE5B
:10DDD00097F0FFFFE78040DD45611743FFFF6700D5
:10DDE0000331A2851306710097000000E78060D719
:10DDF000AA84094455D13544E30055FB4A8597F080
:10DE0000FFFFE78000450D4441D9014497D0FFFF53
:10DE1000E780C0FE634DA400C16B0144FD1B97D099
:10DE2000FFFFE780A0FD634EA4001544B5B7DC44B6
:10DE300013171400BA9783D70700638327030504D9
:10DE4000F1B7D84493171400BA9703D70700631BA0
:10DE5000770123902701268597A00000E78080DBCB
:10DE600001441DBF050465BF1743FFFFE70283257B
:10DE700083C7950041112A8A93F7F707A384F50019
:10DE800032852E89328497E0FFFFE78000FB9317ED
:10DE90000501C1876353F006AA89228597E0FFFF39
:10DEA000E780A0F92311A1004E85832A040097C0C2
:10DEB000FFFFE78040F539E583574400854401447E
:10DEC000F11793B71700A300F1000348110003579F
:10DED0002100D6875285CE862686CA8597F0FFFF19
:10DEE000E7806006A167F10748003EC42302910065
:10DEF00022C697F0FFFFE78020CB41011743FFFFC9
:10DF00006700831FA2851306110097000000E780B9
:10DF100040C52A84894455D9835721001167854417
:10DF2000BA97C2071167C1831307F7EFE36FF7F8DA
:10DF30009787FF1F9387070C9C4381CB854513056B
:10DF4000210097500000E78020758355210022852D
:10DF5000814497C0FFFFE780A0E125D92310050089
:10DF6000228597A00000E78040CD85B71743FFFFCB
:10DF7000E702631483C7950041112A8B93F7F707D3
:10DF8000A384F50032852E8A328497E0FFFFE78074
:10DF9000C0EA93170501C1876351F006AA8A22855A
:10DFA00097E0FFFFE78060E92A895685832B04000C
:10DFB00097C0FFFFE78020E531E5835744008144A7
:10DFC0000544F11793B71700A301F100034831008E
:10DFD000DE875A854A87D6862286D28597F0FFFF4C
:10DFE000E78060F6A167ED0748003EC42302810088
:10DFF00026C697F0FFFFE78020BB41011743FFFFD4
:10E000006700E30EA2851306310097000000E78049
:10E0100040B5AA8409445DD99167CA97C2071167C0
:10E02000C1831307F7EF0544E362F7FACA8597C087
:10E03000FFFFE780E0D3014451F9814997D0FFFF0A
:10E04000E780C0DC63DBA900984893971900BA9772
:10E0500003D7070005EF2390270197D0FFFFE78044
:10E06000E0DA1544E384A9F6268597A00000E7804E
:10E07000C0BC9787FF1F9387E7F79C430144B9D73C
:10E080004A8597500000E780C05889B785097DB759
:10E090001743FFFFE702030379713E847C083EC803
:10E0A0002E8AB7071400A1653ECAE5057C08AA8937
:10E0B000080836C4428932C6BA8AC6843ECC97C0A4
:10E0C000FFFFE78060DFCA85080897E0FFFFE78071
:10E0D00000C732460808B28597E0FFFFE78020C8F6
:10E0E000A246630A09049D45080897E0FFFFE78000
:10E0F000C0BE1D4681459740FFFFE7804001638910
:10E100000A089145080897E0FFFFE78000BD114627
:10E11000A68597000100E780607A100801478146D4
:10E12000D2854E8597C0FFFFE78060FE45611743AB
:10E13000FFFF670063FCB685080897E0FFFFE780F4
:10E1400000C21C400808D8439355C70185891207AF
:10E150005183B205D98D97E0FFFFE78040C01C4096
:10E16000080883C5870097E0FFFFE78040BD1C409B
:10E17000080883C5A70097E0FFFFE78040BC1C406C
:10E18000080883C5970097E0FFFFE78040BB85BF85
:10E190008945080897E0FFFFE78020B483C70400A3
:10E1A0002300F50083C71400A300F500BDB7174393
:10E1B000FFFFE70223F183C795004111AA8993F776
:10E1C000F707A384F5003285AE84328497E0FFFF21
:10E1D000E780A0C693170501C187635DF0042A8913
:10E1E000032A040097C0FFFFE780E0C119E98357C5
:10E1F00044000548F11793B71700A307F1008146C3
:10E2000031A81306F100A28597000000E780609511
:10E210001DC51C459DC783D6470001480347F10033
:10E2200093078500D2884A86A6854E859700000010
:10E23000E78040E641011743FFFF6700E3EB094831
:10E240007DBF1D486DBF1743FFFFE702A3E7657160
:10E250005C083EC4B7077B013EC65C083EC883C766
:10E2600095002A8A328593F7F707A384F500AE89D3
:10E2700097E0FFFFE78040BA8357E100E1C7894597
:10E28000280097C0FFFFE78020C38145280097E062
:10E29000FFFFE780C0AA97C0FFFFE78000C997870C
:10E2A000FF1F9387670D9C431784FF1F034404B629
:10E2B000AA843334800099C3136424009787FF1F16
:10E2C000938707BD9C4399C3136444009787FF1F3E
:10E2D000938747D29C4399C31364840083D5040079
:10E2E0002800014997E0FFFFE78060A783D524005D
:10E2F000280097E0FFFFE78080A683D54400280030
:10E3000097E0FFFFE780A0A597D0FFFFE78000AB75
:10E3100093150501C181280097E0FFFFE78020A445
:10E32000A285280097E0FFFFE78060A39C4463601C
:10E33000F902014781463000CE85528597C0FFFF24
:10E34000E780E0DC59611743FFFF6700E3DADC4454
:10E350001314490028003E9497E0FFFFE780609681
:10E36000834744000347540089070607BA97860786
:10E37000E36AF5FC835524002800814A97E0FFFFFB
:10E38000E780E09D83454400280097E0FFFFE78099
:10E39000009B83455400280097E0FFFFE780209A08
:10E3A0008347440063C9FA00814A8347540063C12C
:10E3B000FA020509A5BF1C4413975A002800BA9712
:10E3C00083D50700850A97E0FFFFE7804099C9BF22
:10E3D000032BC40093975A0028003E9B83552B00C3
:10E3E000850A97E0FFFFE780809783550B002800A0
:10E3F00097E0FFFFE780A0964DBF1743FFFFE702BE
:10E4000003CE5C4993E717005CC997A00000E78042
:10E4100020B61743FFFF6700C3CE1743FFFFE70295
:10E4200003CC2E84814597F0FFFFE780C0E705C548
:10E4300083570500FD172310F50009C483572500F5
:10E440002310F40097000000E78060FB01451743AC
:10E45000FFFF670003CB31457DD823100400C5BF03
:10E460001743FFFFE70203C683C7950041112A8ABD
:10E4700093F7F707A384F50032852E89328497E05D
:10E48000FFFFE780809B93170501C1876356F00665
:10E49000AA89C145228597E0FFFFE780A0802A8BEB
:10E4A0004E85832A040097C0FFFFE780C09531E9BD
:10E4B00083574400231101000544F11793B7170057
:10E4C000A300F10081440348110003572100D687BF
:10E4D0005285CE862286CA8597F0FFFFE780A0A6E8
:10E4E000A1679387170248003EC42302810026C615
:10E4F00097E0FFFFE780406B41011743FFFF670094
:10E50000A3BF13061100A28597F0FFFFE7806065A7
:10E51000AA8409E523110100094475B79305210078
:10E520005A8597000000E78080EF835721002A84F6
:10E53000D9DB9787FF1F9387E7AB9C4381CB85454A
:10E540001305210097500000E78000158355210036
:10E550002685314497C0FFFFE78080812DD52310A9
:10E560000500268597900000E780206D0144A1BF3B
:10E570001743FFFFE702A3B641112E896C00AA845E
:10E5800002C697F0FFFFE78000D20DC103570500D8
:10E5900005072310E50097000000E78040E681476B
:10E5A0003E8541011743FFFF6700A3B532479547FA
:10E5B00065DBCA85268597300000E780400DC1479E
:10E5C000E34005FE3244854741462310F40083575B
:10E5D0000900A685130544002311F40097000100EB
:10E5E000E780C02D228545BF1743FFFFE70283ADBB
:10E5F00083C795004111AA8A93F7F707A384F50012
:10E600003285AE89328497E0FFFFE780008393175D
:10E610000501C1876356F0062A8AC145228597D035
:10E62000FFFFE7802068AA845285032B040097B07F
:10E63000FFFFE780407D31E983574400231101004B
:10E640008544F11793B71700A300F1000144034874
:10E65000110003572100DA875685D2862686CE859B
:10E6600097F0FFFFE780208EA1679387070248009D
:10E670003EC42302910022C697E0FFFFE780C0520C
:10E6800041011743FFFF670023A7A285130611006E
:10E6900097F0FFFFE780E04C2A8409E52311010091
:10E6A000894475B726859305210097000000E7800F
:10E6B00060ECAA8449FD83552100228597B0FFFFB5
:10E6C000E780006B49F5014997C0FFFFE7800074C0
:10E6D000635DA900184893171900BA9703D707007C
:10E6E0000DEF035721002390E70097C0FFFFE7805D
:10E6F000E071630625039787FF1F9387A78F9C43CD
:10E7000099C70355210097500000E78080F02285CB
:10E7100097900000E78060521DBF050975B79544CA
:10E720003DB705C19307F00F630FF500C547630CB4
:10E73000F5009307F5FF05453315F50042054181C6
:10E7400082800145828041657D158280B9E9174349
:10E75000FFFFE702C39803450603328497000000D9
:10E76000E78060FC9305803EB305B502C205C18118
:10E7700081CD0357E402854763F8E70013050401E0
:10E7800097E00000E78020428357E40241677D174D
:10E790006385E700FD172317F4021743FFFF6700A7
:10E7A000439682801743FFFFE702E390004283C74E
:10E7B0009500444D0349140093F7F707A384F5002F
:10E7C00083470400220911673369F900A167B34741
:10E7D000F90041112A8BAE8A63ECE70E83472400CF
:10E7E0001307C00EB91793F7F70F6373F7100347BA
:10E7F0003400C14763EEE70E834744001307E00788
:10E8000093C707086371F70C83498400834774003A
:10E81000A209B3E9F900856763F7F90A034A6400BE
:10E82000834754004E85220A336AFA00975000004D
:10E83000E780403B61C123962403834B3400137A65
:10E84000FA00239A34032388740323994403938999
:10E850000401631C090023A60402239804024E85C8
:10E8600097E00000E78060363DA0034924004A8518
:10E8700097000000E78020EB2397A4028347440021
:10E880004E85A388F402E38D0BFCE30B09FC97E0B3
:10E890000000E780202F97900000E78000738146FA
:10E8A0000146D6855A8597E0FFFFE7800058A167AB
:10E8B000938797033EC423020100480002C697E0F5
:10E8C000FFFFE780602E41011743FFFF67002382AF
:10E8D0008544A2862686D6855A8597E0FFFFE78085
:10E8E000C054A167938797033EC423029100F1B7F8
:10E8F000BD44C5B79144F1BF1733FFFFE702837CE6
:10E9000001111C08404D3EC2B7070F003EC41C0851
:10E910003EC62A89AE8997C0FFFFE78000D7585CC2
:10E920001C5C6346B70E6394E50063E2A70E338573
:10E93000A740B3B7A700B305B7401306803E814692
:10E940009D8D97000100E78080B793140501C18079
:10E95000A1659385C503480097B0FFFFE780C055C8
:10E960008145480097D0FFFFE780603D8355040450
:10E97000480097D0FFFFE780803E8355240448007D
:10E9800097D0FFFFE780A03D814589CCC167FD1787
:10E990009305F00F6388F400268597500000E78008
:10E9A000E0E0AA85480097D0FFFFE7804039035593
:10E9B0004404814501CDC167FD179305F00F63073E
:10E9C000F50097500000E78060DEAA85480097D0E8
:10E9D000FFFFE780C03683456404480097D0FFFFFF
:10E9E000E780E03583457404480097D0FFFFE78057
:10E9F0000035500001478146CE854A8597B0FFFF1C
:10EA0000E780E07005611733FFFF6700E36E814424
:10EA100081B71733FFFFE702836C83C7950093F735
:10EA2000F707A384F50097000000E78020ED173377
:10EA3000FFFF6700036D1733FFFFE702A36883C77B
:10EA400095004111404D93F7F707A384F5002A8AFA
:10EA50003285B284AE8997D0FFFFE780003E2A8BD3
:10EA6000268597D0FFFFE780403D2A89268597D0ED
:10EA7000FFFFE780603A93170B0163CA0702E17753
:10EA8000CA97C207C183116763E3E70293070910BE
:10EA9000C207C1831307B00F637BF7009317090107
:10EAA000C187AA8A634AF000C54763FE5701410146
:10EAB0001733FFFF6700436497B0FFFFE78020250F
:10EAC000E31725FFD5B763080B02630609028144EB
:10EAD00063890A02B7077F00231064052311240508
:10EAE0007CC0568597000000E780E0C39304803E19
:10EAF000B304950239A0B7077F00232004047CC02B
:10EB000081440355240497E00000E780A0A3A1C43A
:10EB100097C0FFFFE78060B7269593D7F44133375E
:10EB20009500AE97BA9708DC5CDCCE8552859700DD
:10EB30000000E780A0DC99E023220404A16793870A
:10EB4000B70348003EC42302010002C697E0FFFF5E
:10EB5000E7808005A9BF814701481CDC232E040300
:10EB6000E9B71733FFFFE702835797C0FFFFE7803E
:10EB70002034E1473305F502914597500000E780C6
:10EB800000C5E55711C59777FF1F23AFA72681471B
:10EB90003E851733FFFF6700C35685471777FF1F72
:10EBA0002306F72682801733FFFFE7024353977748
:10EBB000FF1F9387272580433DC08357040463903C
:10EBC000A70683572404639CB7043689B28497C090
:10EBD000FFFFE78080AB5C5C63C3B7046395B7005D
:10EBE0001C5C63EEA7028347640463F3F400A6870A
:10EBF0002303F4048347740463F39700A687A303F5
:10EC0000F4048357440441677D176385E700850753
:10EC10002312F4043C4481C7CA85268582971733A2
:10EC2000FFFF6700034E9777FF1F9387A71D9C4345
:10EC3000014599C303C5870082801733FFFFE702B0
:10EC4000034A0111B70707003EC683C79500584D18
:10EC50000AC493F7F7070AC8A384F5002A89AE848B
:10EC600011CB1C4283C707002304F70097900000D4
:10EC7000E7800034216493055402280097B0FFFF19
:10EC8000E780802397000000E78020FAAA8528000B
:10EC900097D0FFFFE780A00A300001478146A68594
:10ECA0004A8597B0FFFFE780804613044402480876
:10ECB00022CC230A010002CE97E0FFFFE780C0EEDE
:10ECC00005611733FFFF6700C3431733FFFFE702F8
:10ECD000034101117C003ECAB70707003ECC7C000F
:10ECE0003ECE83C795002E84AA8493F7F707A384AA
:10ECF000F500A16593855502480897B0FFFFE780AE
:10ED0000A01B97000000E78040F2AA85480897D032
:10ED1000FFFFE780C002500801478146A285268593
:10ED200097B0FFFFE780A03E05611733FFFF670044
:10ED3000433D9777FF1F9387E70C9C43094599C391
:10ED400003C5970082809777FF1F9387A70B9C438B
:10ED5000094599C303C5D70082809777FF1F938722
:10ED6000670A9C43014599C303C5A70082801733F6
:10ED7000FFFFE70223350111B70708003EC683C72E
:10ED80009500404D0AC493F7F7070AC8A384F5001D
:10ED90002A89AE8429C41442854703C7060063E06C
:10EDA000E70A83479400094681496380C702B30795
:10EDB000F740A304E400B339F00083C7160023052D
:10EDC000F40097900000E780A01E03572403058BF2
:10EDD00019C76386090097D00000E78000E9216425
:10EDE00093058402280097B0FFFFE780E00C9700AE
:10EDF0000000E78040F4AA85280097D0FFFFE78055
:10EE000000F497000000E78080F5AA85280097D0DD
:10EE1000FFFFE780C0F2014781463000A6854A85A2
:10EE200097B0FFFFE780A02E13047402480822CC9D
:10EE3000230A010002CE97E0FFFFE780E0D60561DC
:10EE40001733FFFF6700432B1733FFFFE702232928
:10EE500001117C003ECAB70708003ECC7C003ECEC4
:10EE600083C795002E84AA8493F7F707A384F5003F
:10EE7000A16593858502480897B0FFFFE780C0032E
:10EE800097000000E78020EBAA85480897D0FFFF95
:10EE9000E780E0EA97000000E78060ECAA85480878
:10EEA00097D0FFFFE780A0E9500801478146A2857F
:10EEB000268597B0FFFFE780802505611733FFFFA8
:10EEC000670023249777FF1F9387C7F39C4301456F
:10EED00099C303C5B70082801733FFFFE7022320E1
:10EEE0000111B70707003EC683C79500404D0AC40D
:10EEF00093F7F7070AC8A384F5002A89AE8405C8EA
:10EF00001C42054783C707006368F7060347B40040
:10EF1000630FF700A305F40097900000E780400915
:10EF20008347B400B9CF97D0FFFFE78040BE21648C
:10EF30009305B400280097B0FFFFE780E0F7970043
:10EF40000000E78060F8AA85280097D0FFFFE780DF
:10EF500000DF014781463000A6854A8597B0FFFF54
:10EF6000E780E01A2904480822CC230A010002CED7
:10EF700097E0FFFFE78040C305611733FFFF67009D
:10EF8000431897D0FFFFE78020BF55B71733FFFF27
:10EF9000E702E31401117C003ECAB70707003ECC2C
:10EFA0007C003ECE83C795002E84AA8493F7F70792
:10EFB000A384F500A165AD05480897B0FFFFE78081
:10EFC000A0EF97000000E78020F0AA85480897D0BE
:10EFD000FFFFE780C0D6500801478146A2852685FD
:10EFE00097B0FFFFE780A01205611733FFFF6700AE
:10EFF00043119777FF1F9387E7E09C43094599C327
:10F0000003C5C70082801733FFFFE702430D0111DC
:10F010007C00AE843ECAA165B70707002A843ECCB7
:10F02000D1057C0048083ECE97B0FFFFE780C0E8DE
:10F0300097000000E78020FCAA85480897D0FFFFD2
:10F04000E780E0CF500801478146A685228597B02A
:10F05000FFFFE780C00B05611733FFFF6700630AFE
:10F060001733FFFFE702A30783C7950093F7F7075E
:10F07000A384F50097000000E78020F91733FFFF15
:10F08000670023081733FFFFE702C30383C7950018
:10F090000329C501411193F7F707A384F5001C422A
:10F0A00083C90700854763E637079777FF1F938774
:10F0B000A72C9C432E84AA8485CF97000000E7806C
:10F0C00080F389476306F502630409028347C90098
:10F0D000638037032306390197900000E78040EDF5
:10F0E00083572903898B89C797D00000E780E0B751
:10F0F0002685A28597000000E78020F1A167CD0753
:10F1000048003EC42302010002C697E0FFFFE780EB
:10F11000A0A941011733FFFF670003FE9777FF1F88
:10F12000938747CE9C431D4599C303C5E700828062
:10F130001733FFFFE702A3FA0111B70707003EC626
:10F1400083C79500584D0AC493F7F7070AC8A384EC
:10F15000F5002A89AE8415C71C4283C70700939621
:10F160008701E18663C4060685466381D706834628
:10F17000E7006388F6002307F70097900000E78018
:10F1800020E321649305E400280097B0FFFFE780A7
:10F19000A0D297000000E780A0F8AA85280097D0A9
:10F1A000FFFFE780C0B9014781463000A6854A8548
:10F1B00097B0FFFFE780A0F53504480822CC230A6A
:10F1C000010002CE97E0FFFFE780009E0561173344
:10F1D000FFFF670003F31733FFFFE70243F001115E
:10F1E0007C003ECAB70707003ECC7C003ECE83C7FA
:10F1F00095002E84AA8493F7F707A384F500A165F0
:10F20000B905480897B0FFFFE78000CB97000000E2
:10F21000E78000F1AA85480897D0FFFFE78020B279
:10F22000500801478146A285268597B0FFFFE780F9
:10F2300000EE05611733FFFF6700A3EC1733FFFFF4
:10F24000E70243E8AA8401441779FF1F1309C9BBE9
:10F25000E14997C0FFFFE780A0C56344A4000145D2
:10F2600019A833053403832709003E9583572500E9
:10F270006397970011051733FFFF6700E3E7050465
:10F28000C9BF032E8500630A0E121773FF1F1303F5
:10F2900063D603230300631503002943639006121A
:10F2A00003234E01631503001D43639907101733B1
:10F2B000FFFFE70243E0C689428A3E89BA8AB684E4
:10F2C000328BAE8B2A84B5E103554E0019E501431C
:10F2D0001A851733FFFF670083E1A167A98F1167C4
:10F2E00063FBE70097000000E78080F5814597F019
:10F2F000FFFFE780C0120844B70700E05841F98FCC
:10F3000018455CC1B707001FF98F1CC55C4991C740
:10F31000610597E00000E780408BE38A09FA2285C7
:10F3200097900000E78060C65DB7328597C0000007
:10F33000E78040430D4349DD1C44116703D5470076
:10F34000A167A98F63FBE70097000000E78040EF0B
:10F35000814597F0FFFFE780800C0323840093161C
:10F360004B01D1828347B300035663008588FD8B30
:10F37000A305F300FD777D8E558EFD76FD16B20454
:10F38000F18E83274301C58E231273012313D3000B
:10F390002304530123052301A3044301BDDF228578
:10F3A00097B0FFFFE78080C9AA850844B5D1610501
:10F3B00097D00000E780207F8DB71D431A8582809B
:10F3C0001733FFFFE70203D00569AA84AE89328AAA
:10F3D0000144FD5A7D1997C0FFFFE78020A26347D3
:10F3E000A40001451733FFFF670003D1D8449317EA
:10F3F0001400BA9703D70700631F37032390570100
:10F4000063070A00268597900000E780A0809C444F
:10F410009DC383D76700B3F72701639E3701D28866
:10F42000014881470147814601468145268597006D
:10F430000000E78040E5050479BF1733FFFFE702CE
:10F4400063C879711C103EC4B7070F003EC61C107C
:10F450003EC883C79500AA8A328593F7F707A3842D
:10F46000F5002E89328497D0FFFFE780009D931727
:10F470000501C187635AF006AA89228597D0FFFF4C
:10F48000E780A09B2A8A4E85032B040097B0FFFFDC
:10F49000E780609739ED8357440081440544F117B4
:10F4A00093B71700A303F10083457100DA87228721
:10F4B000D2864E86280097E0FFFFE780E05701479D
:10F4C00081463000CA85568597B0FFFFE78020C48B
:10F4D000A1679387F70348083ECC230A810026CE14
:10F4E00097D0FFFFE780406C45611733FFFF67004F
:10F4F000A3C0A2851306710097E0FFFFE780606656
:10F50000AA84094455D1528597E0FFFFE78060D473
:10F510000D4459D90546D285268597000000E7801D
:10F5200060EA2A8451B71733FFFFE70243BB8355D4
:10F5300007000346270041112A842E8532C62EC4B7
:10F5400097E0FFFFE780E0D001C93246A24522855F
:10F5500097000000E78000E741011733FFFF6700D5
:10F5600043BA1733FFFFE70203B583C79500411184
:10F57000AA8A93F7F707A384F5003285AE8932840F
:10F5800097D0FFFFE780608B93170501C187635712
:10F59000F00AC1452A8A228597C0FFFFE780807064
:10F5A0002A8D228597D0FFFFE78020892A8922852E
:10F5B00097D0FFFFE7804086930705F893F7F70F92
:10F5C0001307E007AA8B637BF706228597D0FFFF1E
:10F5D000E78080842A8C228597D0FFFFE780C08354
:10F5E000AA8C5285032B040097B0FFFFE780A0810F
:10F5F00039E983574400231101008144F11793B77F
:10F600001700A300F10005440347110083562100B1
:10F61000938784005685DA8822885286CE8597F0B3
:10F62000FFFFE78020A7A167E90748003EC4230247
:10F63000810026C697D0FFFFE780005741011733AE
:10F64000FFFF6700C3AA13061100A28597E0FFFF22
:10F65000E7802051AA8409E52311010009446DB710
:10F66000930521006A8597F0FFFFE780A0F02A84C8
:10F6700041FD835521009356C90013164901854861
:10F680006688E2875E87858A51822685970000001A
:10F69000E78060BF2A848DBF1733FFFFE702A3A175
:10F6A00083C7950041112A8B93F7F707A384F500D0
:10F6B0003285AE89328497C0FFFFE78000789317C8
:10F6C0000501C1876352F00A2A8A228597C0FFFF8D
:10F6D000E780A076AA8A228597C0FFFFE780E075C1
:10F6E0002A89228597C0FFFFE7800073930705F8FA
:10F6F00093F7F70F1307E0072A8C6377F706228545
:10F7000097C0FFFFE7804071AA8C228597C0FFFF5A
:10F71000E78080702A8D5285832B040097A0FFFF1D
:10F72000E780606E39E58357440085440144F11752
:10F7300093B71700A301F10003473100930784003A
:10F740005A85DE882688D6865286CE8597F0FFFFBA
:10F75000E78040948D4748003EC42302910022C6B2
:10F7600097D0FFFFE780404441011733FFFF670058
:10F770000398A2851306310097E0FFFFE780603E03
:10F780002A84894455D99356C900131649018548DE
:10F790006A88E6876287858A5182D685970000004D
:10F7A000E78060AEAA8449BF1733FFFFE702839169
:10F7B0002A8981440144617A916A177BFF1F130BE8
:10F7C0006B8397B0FFFFE780606463C7A400228566
:10F7D0001733FFFF670043928327090093991400B2
:10F7E000CE9703D507003307450142074183636481
:10F7F000570305C103270B0019C785453E85974070
:10F800000000E78060E9832709000504CE97239074
:10F81000070085047DB797000000E78060A283277A
:10F8200009000504CE972390070065D5814597F020
:10F83000FFFFE780C0BEF1BF1733FFFFE7028388F9
:10F8400083C7950041112A8A93F7F707A384F5002F
:10F8500032852E89328497C0FFFFE780005E9317C0
:10F860000501C187635AF004AA89832A040097A07E
:10F87000FFFFE780405931E5835744008544014448
:10F88000F11793B71700A301F10003483100D687A1
:10F8900052850147CE862686CA8597D0FFFFE7802E
:10F8A000806AA167F50748003EC42302910022C682
:10F8B00097D0FFFFE780402F41011733FFFF67001C
:10F8C000A383A2851306310097E0FFFFE78060293C
:10F8D0002A8489445DD99767FF1F9387A7719C434A
:10F8E00081CF044997B0FFFFE7804052AA85268563
:10F8F00097400000E78040DA1305040197000000FC
:10F90000E780C0EA228597800000E78000338144C9
:10F91000ADBF1723FFFFE702037A83C795004111AC
:10F92000AA8A93F7F707A384F5003285AE8932845B
:10F930002311010097C0FFFFE780205093170501B6
:10F94000C1876354F0062A8AC145228597C0FFFF0C
:10F95000E7804035AA8B5285032B040097A0FFFF58
:10F96000E780604A21E98357440085440144F11748
:10F9700093B71700A300F1000348110003572100BB
:10F98000DA875685D2862686CE8597D0FFFFE78018
:10F99000805BA1679387270248003EC42302910041
:10F9A00022C697D0FFFFE780202041011723FFFFE9
:10F9B0006700E373A2851306110097E0FFFFE7805D
:10F9C000401A2A8489444DD99767FF1F938787621D
:10F9D00098433E8901CF044997B0FFFFE780004379
:10F9E000AA85268597400000E78000CB1305040117
:10F9F00097000000E78080DB97B0FFFFE7800041C1
:10FA000095443DD9930521005E8597F0FFFFE7807F
:10FA100060B6AA8435F11C48035721002285239043
:10FA2000E70097800000E780402183270900A9D7DD
:10FA30000355210097400000E780A0BD35BF172384
:10FA4000FFFFE702436783C795004111AA8A93F736
:10FA5000F707A384F5003285AE89328497C0FFFF93
:10FA6000E780A03D93170501C1876351F0062A8AFC
:10FA7000228597C0FFFFE780403C2A895285032BEF
:10FA8000040097A0FFFFE780003831E5835744006A
:10FA900085440144F11793B71700A301F10003480F
:10FAA0003100DA8756854A87D2862686CE8597D05A
:10FAB000FFFFE7804049A167F90748003EC42302E1
:10FAC000910022C697D0FFFFE780000E4101172367
:10FAD000FFFF6700C361A2851306310097E0FFFFB7
:10FAE000E78020082A8489445DD99167CA97C207B4
:10FAF0001167C1831307F7EF8544E362F7FA97674D
:10FB0000FF1F9387274F9843BE8B01CF044997B0BF
:10FB1000FFFFE780A02FAA85268597400000E78099
:10FB2000A0B71305040197000000E78020C897B034
:10FB3000FFFFE780A02D95443DD11C4822858144DC
:10FB40002390270197800000E780200F83A70B00F8
:10FB5000B9D74A8597400000E780A0AB89B7172343
:10FB6000FFFFE702C3572A844105B28497000000D3
:10FB7000E780C0C311C5228597800000E780E00BB5
:10FB800081460146A685228597800000E780C04E09
:10FB90001C4C89C7DC4799C3228582971723FFFF36
:10FBA000670023569767FF1F9387C7259C4301452E
:10FBB00099C31385070182809767FF1F9387872466
:10FBC000884382801723FFFFE70263519317C60023
:10FBD000DD8DC2054111C1812A8432C697C0FFFF65
:10FBE000E780E0173246228511829375F60F97C0A1
:10FBF000FFFFE780C01441011723FFFF6700635038
:10FC00001723FFFFE702034C79713C083ED2B70788
:10FC10000C003ED43C083ED683C79500AE842A89AA
:10FC200093F7F707A384F500A16593853504481081
:10FC300097A0FFFFE7804028C165FD150144176AC2
:10FC4000FF1F130AAA3C930A400EAE892E8B2EC6C4
:10FC500097B0FFFFE780801E4205931704014181A2
:10FC6000C183B24563E9A702C167FD176387F50049
:10FC7000481097C0FFFFE780800E50100147814673
:10FC8000A6854A8597A0FFFFE78060484561172356
:10FC9000FFFF670063463307540383270A0BBA97B5
:10FCA00003D6C701630A3601638A350148109700FD
:10FCB0000000E78060F1DA85050451BFB285EDBF31
:10FCC0001723FFFFE702233F79717C083EC8B7077F
:10FCD00011003ECA7C083ECC83C79500AA893285B4
:10FCE00093F7F707A384F5002E8997C0FFFFE780FD
:10FCF000C01485676378F504A165AA84890508089E
:10FD000097A0FFFFE780401B268597400000E78013
:10FD100060ED133415000A04A285080897C0FFFFA0
:10FD2000E780E001A685080897C0FFFFE780200371
:10FD300025CC014781461008CA854E8597A0FFFF54
:10FD4000E780E03C45611723FFFF6700433AB307B4
:10FD500054030327CA0ABA9703D70700631C970006
:10FD600003D6270063806505080897000000E78038
:10FD7000A0E5DE8505042EC697B0FFFFE780000DE5
:10FD80004205931704014181C183B245E3E1A7FC19
:10FD9000C167FD17E38FF5F8080897C0FFFFE780FC
:10FDA00000FC41BFB285F9B7C165FD150144176A72
:10FDB000FF1F130AAA25930A80022E8BAE8B65BF04
:10FDC0001723FFFFE702A33118418347170083463B
:10FDD0000700A207D58FD207D1832390F500834770
:10FDE0002700034717008D45A207D98F9183231061
:10FDF000F60097C0FFFFE780A0E91723FFFF670029
:10FE000043301723FFFFE702E32BC1640144176966
:10FE1000FF1F1309A91F93098002FD1497B0FFFF6C
:10FE2000E780C0026347A40001451723FFFF670076
:10FE3000A32C330534038327C90A3E958357050055
:10FE4000E38597FE0504D9BF1723FFFFE702832749
:10FE50002A8AAE89B284B68A97400000E78080D8AB
:10FE600019E591473E851723FFFF6700E3282A899C
:10FE70004E8597C00000E780E08E2A84638E0A04D6
:10FE80008D476DD103570500C547E31D47FD034767
:10FE9000F9018546AD47E317D7FC8347450081CF7D
:10FEA0004146A6855D0597F00000E780C09E81472A
:10FEB00055D9AD4745BF130965012302E500CA8541
:10FEC000268597100000E780606231C1A547E38B6B
:10FED0000AF82302040079B705C183570500E392AD
:10FEE00047F94146A685190597F00000E780A09ADA
:10FEF00081472DD99947BDB74E8597000000E7800F
:10FF000080F02A84954739DD130955004DBF4146DD
:10FF1000A68523104401231134011305190097F01D
:10FF20000000E780A099228597800000E780A0EA82
:10FF300081470DBF1723FFFFE702631A79717C0029
:10FF40003ECCB7070A003ECE7C003ED083C795006A
:10FF5000B2842E8493F7F707A384F5001306A1005B
:10FF60002A892C00268597000000E780A0E5A1657E
:10FF700028088D0597A0FFFFE78000F49040835587
:10FF8000A10003558100854697000000E78000EC42
:10FF9000AA84AA85280897C0FFFFE78040DA0356A5
:10FFA000A10083558100280897000000E780C0C1A8
:10FFB000300801478146A2854A8597A0FFFFE78068
:10FFC0000015854748103ED42302910202D697D0EF
:10FFD000FFFFE78060BD45611723FFFF67006312E5
:10FFE0001723FFFFE702A30F79717C003ECCB70710
:10FFF0000A003ECE7C003ED083C79500B2842E849A
:020000040001F9
:1000000093F7F707A384F5001306A1002A892C00B3
:10001000268597000000E780E0DAA16528088D05B5
:1000200097A0FFFFE78040E990408355A10003556A
:100030008100814697000000E78040E1AA84AA85FC
:10004000280897C0FFFFE78080CF0356A1008355A3
:100050008100280897000000E78000B730080147BA
:100060008146A2854A8597A0FFFFE780400A481095
:100070002302910202D402D697D0FFFFE780C0B2DC
:1000800045611723FFFF6700C3071723FFFFE70240
:10009000030597000000E78060DB1723FFFF670080
:1000A00043069767FF1F938727D6884382801723CD
:1000B000FFFFE702C302835725004111AE842A8463
:1000C0002307B10017F5FFFF130525466C00231623
:1000D000F10097A0FFFFE780804591C422859780BB
:1000E0000000E780E0D6FD572310F400130620023D
:1000F0008145130554009720FFFFE780400141012F
:100100001723FFFF6700E3FF1723FFFFE70283FBCF
:1001100079717C003ECCB7070A003ECE7C003ED011
:1001200083C79500AA89AE8493F7F7073285A38425
:10013000F5001306A1002C0097000000E78080C89E
:1001400003558100114497400000E780A0A915C520
:100150000355A100014497B00000E780A06011CDD5
:10016000035705008357810045446318F700854510
:1001700097000000E780E0F301442169930539000E
:10018000280897A0FFFFE78020D3A285280897C002
:10019000FFFFE780C0BA0356A100835581002808FD
:1001A00097000000E78040A2300801478146A685FD
:1001B0004E8597A0FFFFE78080F548104AD42302C0
:1001C000810202D697D0FFFFE780009E456117238A
:1001D000FFFF670063F21723FFFFE702A3EE9767B5
:1001E000FF1F938727C22A8488432E8915C503578A
:1001F00045038357C4016311F70223260502231820
:100200000502410597D00000E780209C63060900A5
:1002100097800000E78060DB81449769FF1F938926
:10022000E9DE130A800297B0FFFFE78020C263C4B3
:10023000A4049767FF1F9387A7C59C4399C70355DD
:10024000C40197200000E780C0BD63070900228534
:1002500097800000E780C0A01306400E81452285EC
:100260009720FFFFE780A0EAFD57231EF400172325
:10027000FFFF670063E83385440383A7C90A3E95FF
:10028000035705008357C4016317F700CA85970019
:100290000000E78000E2850479B71723FFFFE7023B
:1002A00063E283C795004111AA8993F7F707A384F6
:1002B000F5003285AE8497C0FFFFE78000B8856700
:1002C0006378F5042A8997400000E780A0910144F3
:1002D00001CD83D704003144638827018545970009
:1002E0000000E78080EF01444E85A2864A86A685FD
:1002F00097D0FFFFE780A09CA16793871704480071
:100300003EC42302810002C697D0FFFFE780C08968
:1003100041011723FFFF670023DE1723FFFFE702DA
:1003200063DA9767FF1F9387E7AD804329C40145D0
:1003300097C00000E780002181470148C1641CDCB0
:10034000232E0403232004041769FF1F130909CC7B
:1003500001449309400EFD1497B0FFFFE78000AE03
:10036000634FA400814517F5FFFF1305857F97A014
:10037000FFFFE780C01B1723FFFF6700E3D73305AC
:1003800034038327090B3E958357C5016387970084
:10039000854597000000E78040E4050475BF93574A
:1003A000050113D78700A380F50093170501C183CA
:1003B000A1832380E5002381F500A381A50082802D
:1003C0001723FFFFE702A3D12300050083C7150011
:1003D000A300F50083C725002301F50083C735007E
:1003E000A301F50083C745002302F50083C755002C
:1003F000A302F50083C7650093059500A3030500DC
:100400002303F50023040500328597000000E780F0
:1004100040F91723FFFF6700C3CE1723FFFFE70252
:1004200063CA4111E9540DCD85CD93F9C5FF2E84E2
:100430002A89AA84338AA900B7EA040063189A02B9
:100440000D88854411CCB7E704009C5F82972AC6CB
:1004500022866C003305390197E00000E7800046F2
:10046000268541011723FFFF670003C983A78A037D
:100470009104829793170501C183A183A38EF4FE93
:1004800093570501238FF4FEA183238EA4FEA38F2F
:10049000F4FE6DB763E6D5021723FFFFE70223C41E
:1004A000B28741113686BE8536C697E00000E780E8
:1004B000E040B246410136851723FFFF670063C461
:1004C000814636858280838705001387F5003D05C8
:1004D000FD8793F77708834607007D158606B58F5D
:1004E000A300F5006307B7007D17834717009D83BE
:1004F000DDB782801723FFFFE70263BEB7E7040082
:1005000083A7070932872A863A8582971335150013
:100510001723FFFF6700E3BE15C181478DC1172375
:10052000FFFFE702C3BB414697E00000E7800039C8
:1005300085473E851723FFFF6700A3BC81473E85A3
:1005400082801DCD1723FFFFE70263B94146814535
:100550002A849720FFFFE78080BB41468145130531
:1005600004039720FFFFE78080BA0147C167232279
:10057000040438C87CC805451723FFFF670063B82B
:100580000145828081473DCDB5CD1723FFFFE702AE
:1005900003B5B2842E891306800581452A849720ED
:1005A000FFFFE780C0B6CA8524C4268597000000F7
:1005B000E780C0F64146814522859720FFFFE7800E
:1005C00000B53044A285228597000000E780C0F284
:1005D00093040401A285268597000000E780E0EEE1
:1005E000A6851305040297000000E78000EE22852F
:1005F00097000000E78020F585473E851723FFFF21
:10060000670023B03E8582801723FFFFE70283AB9C
:100610004111E9540DCD85CD93F9C5FF2E842A896A
:10062000AA84338AA900B7EA0400639844030D88BA
:10063000814411CCB7E704009C5F82972AC62286CA
:100640006C003305390197E00000E78020272685FC
:1006500041011723FFFF670023AA83A78A039104A0
:10066000829793170501C183A183A38EF4FE93574C
:100670000501238FF4FEA183238EA4FEA38FF4FE35
:100680006DB765CD1723FFFFE702C3A3B28411E660
:1006900005451723FFFF670023A62A842E890145FD
:1006A000EDD93C487848B3E6E700E5D69386F7FFF6
:1006B000B3B7F6007D17032A4404BA9734C87CC840
:1006C00063050A06C14913050A03B3894941229506
:1006D000637D3601B2862E86A68597000000E780EE
:1006E000A0DB7C40BE9464C065B7CE862E86CE85E6
:1006F00097000000E78040DAC114D2944E9923227B
:100700000404A2879306040103C7070003C6070376
:100710008507318FA38FE7FEE398F6FE3044A2856C
:10072000228597000000E78020DD2699C149330625
:10073000994063EC9900A9DCA686A68513050403FD
:1007400097000000E78040D579BF8147B306F400E9
:100750003307F6000347070083C5060085072D8F82
:100760002380E600E39437FF3044A285228597007A
:100770000000E78060D8C1145DBF014582800DC1D3
:100780001723FFFFE702A3951306800581459720F5
:10079000FFFFE780C09705451723FFFF67006396BB
:1007A00001458280814749C5C1C51723FFFFE70284
:1007B0000393FC4141462E84AA846399C70413869F
:1007C0000501A2878146C14503C7070003C507038A
:1007D0008507298F3305D600034505008506298F37
:1007E000A38FE7FEE392B6FE3044A28526859700EC
:1007F0000000E78060D0228597000000E78060F865
:1008000085473E851723FFFF6700A38F13850703E6
:100810001D8E814522959720FFFFE780408F7C4009
:10082000130700F813060402A2972388E70251BFBA
:100830003E8582801723FFFFE702638A6D712E8455
:10084000B284AA8590102800368997000000E780BE
:10085000A0D309EDD55725A050400C4028009700A3
:100860000000E78040E27DD5FD142104F5F42C0062
:100870004A8597000000E78020F3814761DD3E85CF
:1008800051611723FFFF6700C3871723FFFFE702AC
:10089000038541112EC432C62C0005469700000086
:1008A000E78080F941011723FFFF67008385172345
:1008B000FFFFE702C38201112A842EC602C802CAC2
:1008C00002CC02CE97E00000E780C023B2462A8621
:1008D000A285080897000000E78060FB1375F50FFC
:1008E00005611723FFFF6700C3811713FFFFE702AE
:1008F000037F7971B2872A8421462308B10013054A
:100900001101BE853AC436C697E00000E78000FBBF
:10091000B24693059101368597000000E78060A8F4
:100920002285141035460C0897000000E78020F659
:100930002A84224701E921460C103A8597E00000FD
:10094000E780C0F7228545611713FFFF6700637BCF
:100950001713FFFFE702A3787171AE84AA850A8599
:10096000328497000000E78060BB11C90A86A68523
:10097000228597000000E78020B8814711E1C54734
:100980003E854D611713FFFF6700A3771713FFFF25
:10099000E702E3711D712A8AB289BE843546854714
:1009A000130511012E8CB68A3A8BC28C468D230812
:1009B000F10097E00000E78060F010100C0852850D
:1009C000231F010097000000E780C0F82A843DED56
:1009D000A1476313FD089307900591E0E54735466D
:1009E000E2851305110113990A012308F100135937
:1009F000090197E00000E78060EC135789009397A6
:100A00008A00D98F90080C085285231FF1009700A7
:100A10000000E78020F42A8415E9A1E49387FA0016
:100A200091831379F9003EC6631309004149668B2F
:100A30008144C14B854DB247639F970C6A868C00F9
:100A400033855C0197E00000E78040E7228525615F
:100A50001713FFFF6700636993079004C9F0A54768
:100A6000BDBF834701050947C14B2308F1008347F8
:100A70001105A58FA308F10093872400814463E149
:100A8000FB04014714083386E6008C08B386E400B3
:100A9000BA95DA9683C6060083C505000507AD8EB4
:100AA0002300D600E390E7FE4147639CE7049008EB
:100AB0000C08528597000000E780C0E925D181A08D
:100AC000B3069B00BA871008B305F60090083E965F
:100AD00003C506000346060085078506298E238088
:100AE000C500E39277FF998F90080C085285BE9459
:100AF00097000000E78000E68947014749D12A8432
:100B0000B1B790083E96034606001408BE962380AF
:100B1000C600850759BFB24785046387971481478C
:100B20001808B306F70098083E973386F900034784
:100B30000700034606008507318F2380E600E39116
:100B400077FF90080C08528597000000E78080E04E
:100B50005DF53546E285130511012308B10197E0E3
:100B60000000E780A0D51397040141839397840088
:100B70002183D98F10180C085285231FF10097008C
:100B80000000E78020DD25FD814710183387F9003C
:100B90003E960347070003460600B306FB008507A1
:100BA000318F2380E600E39277FF65A81808B3062B
:100BB000F70098083E973386F9000347070003467D
:100BC00006008507318F2380E600E3E127FFCA870F
:100BD000639E770990080C08528597000000E78013
:100BE00060D711FD81479800B306F70090081810F0
:100BF0003E973E9603470700034606008507318F60
:100C00002380E600E39177FF3546E2851305110165
:100C10002308B10197E00000E78040CA1397040160
:100C20004183939784002183D98F10180C08528533
:100C3000231FF10097000000E780C0D1E31105EC0D
:100C4000814710183387F9003E9603470700034693
:100C50000600B306FB008507318F2380E600E3E240
:100C600027FFC109410BC1BB814785B79408BE96D8
:100C700083C6060018083E972300D700850789BF62
:100C8000638006321713FFFFE702634259712A841B
:100C9000BE89B28B85473546130511022E8B468CD3
:100CA0004289BA8A368A2300F10297E00000E78081
:100CB000E0C010180C1022852317010297000000D5
:100CC000E78040C963180512A147631FFC0693071C
:100CD000900563930900E5473546DA85130511024F
:100CE00093140A012300F102C18097E00000E7801D
:100CF000E0BC93178A0013D78400D98F90080C109A
:100D000022852317F10297000000E780A0C47DE14F
:100D1000639209049307FA00BD88918391E0C1446E
:100D2000C207C183DE8C814A3EC6414DB24763E2B1
:100D3000FA0E6286B3854B01881097E00000E780C9
:100D400080B54DC93D557DA093079004E39609F801
:100D5000A54759B7834701050947C14C2300F10254
:100D600083471105B3C7F900A300F1029387290057
:100D7000814963E1FC04814618103306D7008C08D2
:100D80003387D900B69556970347070083C50500FA
:100D900085062D8F2300E600E390D7FE4147639040
:100DA000E70690080C10228597000000E78080BAC3
:100DB00035D189A0B3863A01BA871010B305F60081
:100DC00090083E9603C50600034606008507850683
:100DD000298E2380C500E39297FF3387EC4090086B
:100DE0000C102285BA9997000000E780A0B68947C9
:100DF000014741D165611713FFFF6700032F90087A
:100E00003E96034606001410BE962380C600850752
:100E100079B7B247850A93990A01939D8A0093D9BD
:100E200009016391570F85473546DA85130511028D
:100E30002300F10293D9890097E00000E78000A821
:100E4000B3ED3D0190000C1022852317B1039700EC
:100E50000000E78020B059FD8147A68963EA970624
:100E600026860C084A8597E00000E78020A5814788
:100E70001810B306F700100898083E973E960347EF
:100E80000700034606008507318F2380E600E3E173
:100E900097FE639FA90590080C102285970000001B
:100EA000E78040AB21F981479810B306F70090081E
:100EB00018183E973E96034707000346060085072D
:100EC000318F2380E600E391A7FF4109C10CB9BD32
:100ED00018089000B306F7003E963387FC000347DE
:100EE0000700034606008507318F2380E600B5B76B
:100EF00098084E97034707001C10CE972380E70001
:100F0000850941BF85473546DA851305110223005F
:100F1000F10293D9890097E00000E780209AB3EDB1
:100F20003D0190000C1022852317B10397000000AB
:100F3000E78040A2E31005EC814718089000B30653
:100F4000F7003E963387FC00034707000346060080
:100F50008507318F2380E600E391A7FF41460C0807
:100F60004A8597E00000E780609581471810B30636
:100F7000F700100898083E973E960347070003467F
:100F800006008507318F2380E600E391A7FF9008D4
:100F90000C10228597000000E780C09B1DD599BDED
:100FA0007D5582801713FFFFE702631301112A8426
:100FB0002E8593055100328902C002C202C402C6C6
:100FC0009304740097F0FFFFE780A03D1D46A685BF
:100FD0001305910097E00000E780408E10088A8595
:100FE0004A8597000000E780E09619ED930714000A
:100FF000180883C607000346070085070507B18E5A
:10100000A38FD7FEE397F4FE05611713FFFF670078
:10101000430F1713FFFFE702E30A2E848C414111AF
:10102000AA89838715003289914463D30700A144BC
:101030009757FF1F938747349C43A1C7C1CA8D4769
:101040002310F10083C725004A852301F10083C7DF
:101050003500A301F10083C745002302F10083C7D7
:101060005500A302F10083C7650093059100A30317
:1010700001002303F1002304010097F0FFFFE78044
:1010800040320C404A860A8597F0FFFFE7808033A4
:101090000328040083564400A6881D0881470147A1
:1010A000E51642868A854E8597000000E780408ECF
:1010B0002A8919E5A685228597B0FFFFE780E0C160
:1010C0004A8541011713FFFF670003034A860A851B
:1010D00097F0FFFFE780002F6DB71713FFFFE702C0
:1010E00063FE2E848C414111AA89838715003289C1
:1010F000914463D30700A1449757FF1F9387C727E5
:101100009C43A1C7C1C68D472310F10083C72500AA
:101110004A852301F10083C73500A301F10083C78D
:1011200045002302F10083C75500A302F10083C7E5
:10113000650093059100A30301002303F10023043C
:10114000010097F0FFFFE780C0250C404A860A8522
:1011500097F0FFFFE7800027835644000328040030
:101160008A85858EC2061D08C1822312D400A688F6
:1011700081470147E51642864E8597000000E780CB
:1011800060B041011713FFFF670003F74A860A8525
:1011900097F0FFFFE78000234DBF1713FFFFE70223
:1011A00003F4B335B000011185052A891315F60142
:1011B000336515012308B1009305110136843AC641
:1011C00032C03EC442C297F0FFFFE780801DA247B5
:1011D0001248425593D68700230BF10093059101E5
:1011E00093578800A30AD100A30BF100230C01013F
:1011F00097F0FFFFE780E01A324702460328040019
:10120000B337E000835644009207914411C2A144D1
:101210004A85A68842860C0897F0FFFFE780407752
:101220002A8919E5A685228597B0FFFFE780E0AA05
:101230004A8505611713FFFF6700A3EC1713FFFF33
:10124000E70243E801113EC68647B335B000850585
:10125000AA891315F6015D8D2308B10093051101CC
:1012600036843A89B28442C446C297F0FFFFE780D1
:10127000401322489248164593578800A30AF1006C
:101280009305910193D78800230B0101A30BF10073
:10129000230C110197F0FFFFE780A01032471040A8
:1012A00083564400B337E0009207032809009148B1
:1012B00091C0A1480C084E8597000000E780809CF3
:1012C000AA8401E9835544004A8597B0FFFFE7806F
:1012D000C0A0268505611713FFFF6700E3E1AA950B
:1012E0009307F00F17070100130707546317B500A2
:1012F00013C5F7FF1375F50F828005058346F5FFCB
:10130000B58FBA9783C70700D5B703574500144177
:101310009307F00F17060100130606513697420790
:101320004183139506014181631BE500AD8FB297A0
:1013300003C50700130515F31335150082808506D4
:1013400003C5F6FFA98FB29783C70700D9BF17134C
:10135000FFFFE702C3D8B28736842E86BA86AA85F5
:101360003E85BA8497F0FFFFE7806052634F050027
:10137000228597D00000E780E0782A86A686A2859D
:10138000268597F0FFFFE78080501713FFFF670067
:1013900043D71713FFFFE702E3D25D712A8BAE8AB2
:1013A000170501001305C5452C00B284368ABA8999
:1013B0003E8997F0FFFFE780C04F2A845DE134103B
:1013C0004146DA85280097F0FFFFE780404C2A84E9
:1013D00049E98547A303F100A6C2930771002408D9
:1013E000BEC4A68685470D462C18281002DC02DEF6
:1013F000D6C0BEC697F0FFFFE78000442A8435E1DF
:1014000083477102A6860D4693F7F7072300FA007B
:10141000C1473EDE2C188947281026DCA303F100C3
:1014200097F0FFFFE78040412A8405ED4146A685FD
:101430004E8597D00000E78060488D47A6860D4610
:101440002C182810A303F10097F0FFFFE780C03E9F
:101450002A8401E94146A6854A8597D00000E780A5
:10146000E045228561611713FFFF6700E3C817138A
:10147000FFFFE702C3C697F700009387A7A1984331
:1014800083C7470079712A89AE84170501001305C7
:10149000A5370C083AC42306F10097F0FFFFE78058
:1014A00040412A8405ED14104146CA85080897F08A
:1014B000FFFFE780C03D2A8415E1140815462C0083
:1014C000081097F0FFFFE780803C2A8401E921465D
:1014D0002C08268597D00000E780403E2285456194
:1014E0001713FFFF6700E3C11713FFFFE70223BFD6
:1014F00097F700009387079A9C477971AA842E84F6
:10150000170501001305C5300C083EC697F0FFFF14
:10151000E780203A0DE914104146A685080897F0A7
:10152000FFFFE780C03605E1140811466C00081083
:1015300097F0FFFFE780A03519E58347F10193F7A6
:10154000F7032300F40045611713FFFF670063BB37
:101550001713FFFFE702A3B83688A1488147014768
:10156000E54697F0FFFFE780A0421713FFFF6700F3
:1015700043B91713FFFFE70283B63688A1488147B6
:101580000147E54697F0FFFFE780C06F1713FFFFA5
:10159000670023B71713FFFFE70263B401112A8422
:1015A0002E850C0832C697F0FFFFE780803009EDEA
:1015B000324797060100938626241008C1452285EC
:1015C00097000000E780E0D805611713FFFF670070
:1015D00043B31713FFFFE70283B04111C1472EC089
:1015E00032C48A8509463EC23EC697F0FFFFE780B7
:1015F000A02441011713FFFF6700A3B01713FFFFDB
:10160000E702E3AD4111AE8613061009AA850A85EB
:1016100002C002C202C402C697F0FFFFE780202783
:1016200041011713FFFF6700C3AD1713FFFFE70268
:1016300003AB3287970601009386061E2E8693051C
:10164000000297000000E780C0D01713FFFF67007B
:1016500043AB1713FFFFE70283A87971C1472ACC78
:101660002ED032D42C080D4628003ECE3ED23ED697
:1016700002C402C602C802CA97F0FFFFE780C01B7F
:1016800045611713FFFF6700C3A71713FFFFE702AA
:1016900003A50111AA842E8417050100130545181E
:1016A0008A8597F0FFFFE780C02015E514084146C2
:1016B000A6850A8597F0FFFFE780601D09ED834747
:1016C000E1010347F101A207D98FCA07C9836177F6
:1016D000D98F2310F40005611713FFFF670063A281
:1016E00015CD1713FFFFE702839F9747FF1F9387CF
:1016F000277690439745FF1F9385C5751745FF1FB4
:101700001305057197D00000E78000C51745FF1F3E
:10171000130505701713FFFF6700A39E1745FF1FF2
:101720001305056F82808DCD1713FFFFE702239B02
:101730009747FF1F9387C771944301112E840A8630
:101740009745FF1F9385057197D00000E78040C63D
:101750000A850294014505611713FFFF6700639A2C
:101760007D5582801713FFFFE702639797D0000033
:10177000E78080D19747FF1F23ACA76C17F5FFFFC9
:101780001305E5C997B00000E780C0741713FFFF89
:10179000670023971747FF1F1307C76D931715009F
:1017A00008433E95FD572310F50082801713FFFF75
:1017B000E702E3922A84084009E51713FFFF670058
:1017C00043941C4158401CC06313E5005CC0834730
:1017D000550023200500F99BA302F50097A0FFFF09
:1017E000E780207CC9BF1713FFFFE702A38D97474F
:1017F000FF1F9387276A98432A8411CB83473500BC
:1018000093F7070289C70355050089450297130519
:10181000440197B00000E780403B83550400035526
:10182000E40097300000E780A00C485819C597A045
:10183000FFFFE7800077232A040213058403970043
:101840000000E780E0F68144B1499790FFFFE78010
:10185000206A63CBA402834734002320040493F757
:1018600027FCA301F40000489790FFFFE780406940
:1018700013161500814522859710FFFFE780208908
:101880001713FFFF67004387B3873403032904035B
:1018900085043E994A8597000000E78060F12304A3
:1018A000090065B78347350093F7070299E30145BF
:1018B00082808357E500E39CB7FEC167FD1763167E
:1018C000F60005458280054599A81713FFFFE7023A
:1018D000038193170601C187B2842A8401496359A1
:1018E000F002835705009DCB01456367F600034571
:1018F00084003E953325A6001375F50F0DA01C48F6
:1019000013171900BA9783D70700E38E97FA0509D2
:101910009790FFFFE780C05EE343A9FE01451703F0
:10192000FFFF6700037E1703FFFFE702A379AE897D
:10193000AA849790FFFFE78060522A8497D0FFFF28
:10194000E780A02EAA8601471306840197050000B0
:10195000938585E41745FF1F130505529790FFFFF8
:10196000E780E0182A8925C98C441304C500228524
:101970009E0593F5050897A0FFFFE780403CCC400B
:1019800083877400E18163DD070493E50508228500
:1019900097A0FFFFE780A03A0D469385440022857B
:1019A00097A0FFFFE780C03683D50400228597A06B
:1019B000FFFFE780E03D83D52400228597A0FFFF4D
:1019C000E780003D03D6490083A50900228597A042
:1019D000FFFFE780E0334A851703FFFF6700C3710D
:1019E00093F5F5076DB71703FFFFE702436F01118A
:1019F0002A84328532C697A0FFFFE780E0279780D0
:101A0000FFFFE780C030835704001747FF1F13070D
:101A1000E75F3246231BF100930700F8A30DF100A6
:101A20001C471843231AA1008983858BB307F7400D
:101A3000B28548083ECE231C0100230D010097000B
:101A40000000E78080EE05611703FFFF6700636B0E
:101A50001703FFFFE7020367004101453DC49304FC
:101A6000C40026853289AE8997A0FFFFE780C02495
:101A700095452A8A2685035B040197A0FFFFE7802E
:101A80002021268597A0FFFFE780603E8D45AA8A2A
:101A9000268597A0FFFFE780A01F268597A0FFFF60
:101AA000E780E03C5C48420A135A0A01D2975CC4C2
:101AB00023186401814763983A0146054D81330636
:101AC00025419337160013F5F70F1703FFFF670043
:101AD000A3621703FFFFE702035E89692A8BAE8BBF
:101AE000328AB68A81440144314CFD199790FFFF38
:101AF000E780004063CDA4009790FFFFE78040425D
:101B0000018D33B5AA001703FFFF6700435E3389D9
:101B1000840383270B003E9963170A0083478900DB
:101B200085043E94E1B703560A00DE854A8533F604
:101B3000C90097000000E780E0F16DD10545E1B7ED
:101B40001703FFFFE702A35901112A847C00035504
:101B5000E5003ECAB70707003ECC7C003ECE97208A
:101B60000000E78020082A898545480897A0FFFFE4
:101B7000E78020399945480897A0FFFFE780E015E6
:101B8000AA844A8597200000E780A0082380A4004B
:101B90009747FF1F938787479C434166130606F0CC
:101BA0009396870113D78701558F93D68700F18EBF
:101BB000558FA207B706FF00F58FD98F11462C006D
:101BC000138514003EC497D00000E78020CF500852
:101BD000A38204008945228597000000E780E0E0A9
:101BE00019C9AA851305840397A0FFFFE780E03198
:101BF0003C4085073CC005611703FFFF6700635049
:101C00001703FFFFE702A34D9790FFFFE7804031E6
:101C10002A8405049790FFFFE780802F3305A402F4
:101C2000F14791453305F50297200000E78020BA7F
:101C300011E565551703FFFF6700A34C9747FF1F8A
:101C400023A2A7249790FFFFE780802D2A84050414
:101C50009790FFFFE780C02B3305A4028945060556
:101C600097200000E780A0B669D59747FF1F23A300
:101C7000A7209790FFFFE780A02A2A840504979069
:101C8000FFFFE780E0283304A4029747FF1F239556
:101C9000871E9790FFFFE780A0282A849790FFFF78
:101CA000E7800027930714003385A7029747FF1F9B
:101CB0002395A71C97F700009387477A1747FF1FC4
:101CC0002320F71C0145BDB71703FFFFE702833F41
:101CD000AA842E8901449749FF1F93892933130A47
:101CE00080069790FFFFE780A0226347A40001458C
:101CF0001703FFFF670043403305440383A709022E
:101D00004A86A6853E9597000000E780E0B919E174
:101D10000504C1BF0545E9BF1703FFFFE702A3396B
:101D2000AA8A2E8BB28B368C3A8A8144014481492F
:101D3000974CFF1F938C8C2D130D80069790FFFFFF
:101D4000E780001D63C9A40011E085494E85170393
:101D5000FFFF6700C3393389A40383A70C025E86A3
:101D6000D6853E994A8597000000E780E0B31DC103
:101D70009790FFFFE780C01A0544636D4501D28646
:101D80006286DA851305090397000000E780A0D476
:101D900011C1854985045DB71703FFFFE702833250
:101DA000C16441112A8901449749FF1F938909267B
:101DB000130A8006FD1436C632C42EC29790FFFF68
:101DC000E780001592452246B2466348A4000145CB
:101DD00041011703FFFF670023323305440383A744
:101DE00009023E9509C683473500C18B9DC791C640
:101DF0008347350093F707028DC363069900835725
:101E0000E500639C27010357050001CB63E7E5006C
:101E100083478500BA97E3CDF5FA050469BF170338
:101E2000FFFFE702232AC1642A8901449749FF1F63
:101E30009389C91D130A8006FD149790FFFFE78060
:101E4000200D6346A4001703FFFF6700E32A330554
:101E5000440383A709023E958357E500638A9700F0
:101E6000630499006396270197000000E780E097DC
:101E70000504E1B71703FFFFE702632389692A8A94
:101E8000AE8A328BB68B8144174CFF1F130C0C1893
:101E9000930C8006314DFD199790FFFFE7804007B6
:101EA00063C6A4001703FFFF67002324338994034C
:101EB00083270C028355CA015A863E994A859700AA
:101EC0000000E780609E31C1814D15A03384AD03D1
:101ED0008327090303D60B00D68533F6C9003E9449
:101EE000228597000000E780E0B609E9850D97900C
:101EF000FFFFE780E0FFE3CBADFC01A82285970060
:101F00000000E780E08A23040400850471B717030A
:101F1000FFFFE702431A4169AA8A014A174BFF1FD4
:101F2000130BCB0E7D19C14B054C9790FFFFE7803B
:101F300020FE6346AA001703FFFF6700431B9309B7
:101F40008006B3073A0383290B02BE9983D7E900C1
:101F5000638E270163842A01639A570103A48903CE
:101F600001E84E8597000000E780C0BD050A75BFF7
:101F700083570401639977099304C400268597A0C9
:101F8000FFFFE78060D385452A8D2685835C0401A9
:101F900097A0FFFFE780C0CF268597A0FFFFE780CF
:101FA000A0E762056185635905048D45268597A0E4
:101FB000FFFFE780E0CD8945268597A0FFFFE780FA
:101FC00020CD8945268597A0FFFFE78060CC854519
:101FD000268597A0FFFFE780E0CC834705000947EF
:101FE00093F7F707639AE7009945268597A0FFFFC7
:101FF000E78040CBA30285014848337D2D0123189B
:1020000094016A9548C40040A1BF1703FFFFE7028F
:10201000030D37E404008327041D82979747FF1FB1
:1020200083C7C7EB1715FF1F13054550A300F50025
:102030008327441C82978327841C81461306F00F54
:102040008145014582971703FFFF6700830B174700
:10205000FF1F1307A7D818439745FF1F83C505E83F
:102060009747FF1F938707E6834687030346970337
:102070006397D5009747FF1F2382C7E6828083C5F9
:1020800087010347A7036317B6009747FF1F2387FE
:10209000E7E4828003C687016317C7009747FF1FE5
:1020A000238ED7E2828083C687011307500263190B
:1020B000D700930760021747FF1F2301F7E28280D2
:1020C00083C68701130660026315D600930770026A
:1020D000DDB783C7870155BF9747FF1F938787DE0B
:1020E000D44B0947638DE6081703FFFFE70223FF80
:1020F0001749FF1F130949DA3E8483470900918B72
:102100009DCFB7E4040083A7041D829783A7441CD6
:102110001745FF1F1305C5D8829783A7841C8146E6
:102120001746FF1F0346C6D981450145829721C541
:1021300083470900ED9B1747FF1F230FF7D4834701
:10214000040093F7F70F85CB91471747FF1F23250F
:10215000F7D897000000E78080EB97000000E78049
:1021600040EFB7E70400BC4F414691451745FF1FBC
:102170000345C5D582971703FFFF670083F8828068
:102180001703FFFFE702A3F58D4741116306F5042E
:10219000C5476308F50285476310F5029747FF1F9F
:1021A0002380A7D4B7E70400BC4B93050010174564
:1021B000FF1F0345A5D1829741011703FFFF670069
:1021C00043F485471747FF1F230CF7D0B7E70400F8
:1021D000BC4B93050020E1BF9747FF1F938787CE35
:1021E000D44B1147638DE600B7E7040083A7071DB2
:1021F0008297B7E70400BC4B930500044DBF054927
:102200001747FF1F232A27CD83C7070032C62E8416
:1022100093F7F70FD5D3B7E4040083A7041D7D140B
:102220001374F40F8297E37689FCB245994703C68D
:102230001500E3F0C7FCFC4409061745FF1F130512
:1022400065CA8297BC48930500081745FF1F0345E0
:10225000E5C7829779BF1703FFFFE70243E81747F7
:10226000FF1F130727C64047184B1C409746FF1F08
:1022700023A0F6C66316E4001747FF1F232CF7C4FC
:10228000130584FE9790FFFFE78060A6035564FF67
:102290009780FFFFE780E06E97A0FFFFE78060D0A8
:1022A0001703FFFF6700E3E51703FFFFE70223E3E0
:1022B0009747FF1F938707C1D84BDC4789C7970013
:1022C0000000E78080F985471747FF1F2326F7C0E6
:1022D0009747FF1F938787B09C43930500021745DC
:1022E000FF1F0345A5BE83C787031747FF1F2307AB
:1022F000F7BEB7E70400BC4B82971703FFFF6700E8
:1023000043E09747FF1F23A1A7BC82801703FFFF6D
:10231000E70243DB37E404007C4CA1451745FF1F6F
:102320000345C5BA82977C48A1451745FF1F034561
:10233000E5B99744FF1F9384E4B88297DC4489EBA6
:1023400097000000E78080D91703FFFF6700C3DA1A
:1023500003D567FF9780FFFFE780A062AA896DD150
:10236000D84891476310F7027C4C91451745FF1FF1
:102370000345C5B582977C4891451745FF1F034526
:10238000E5B4829703A9490103D409018947B7E954
:1023900004001747FF1F2321F7B483A7091D210459
:1023A0004204829783C784011715FF1F1305051880
:1023B00061191717FF1FA30BF71683A7491C41804C
:1023C00082979747FF1F238D07B083A7C91C8146BB
:1023D00009469375F40F4A85829711E99747FF1FC5
:1023E00083C747C089C79710FF1FE780A080B7E762
:1023F0000400BC4F2146A1451745FF1F034505AD0D
:10240000829799B71703FFFFE70263CD93F7052083
:1024100001112E8481CF97000000E78020E9134549
:10242000042005611703FFFF6700A3CD93F7051094
:10243000A9CF9744FF1F9384E4A8DC4897000000CD
:10244000E78020C11747FF1F13074799184383C729
:102450008401034787036318F700DC4489C79700AA
:102460000000E78080DF85471747FF1F2326F7A678
:10247000B7E70400BC4B930500021745FF1F034557
:10248000E5A482971345041069BF93F70508BDC7FB
:102490009747FF1F83C717A5E91719469745FF1FE1
:1024A000938565A41305D10093F4F70F1749FF1F17
:1024B000034949A397C00000E78040409397040177
:1024C000C1831747FF1F130767A2231DF100231CB9
:1024D000F1009747FF1F9387E79E3ACE3ACAD84349
:1024E0002306010009CBDC439315890154080D46EE
:1024F000E185680082971345040825B793F7250006
:10250000A5C39747FF1F9387E79BD84B894763066F
:10251000F7029747FF1F83C7279813F7270011EF8C
:10252000918B99CFB7E70400BC4F1306000A894589
:102530001745FF1F03458599829713452400D5B59C
:102540009747FF1F938787899C4383C78703174754
:10255000FF1F2305F79897000000E78060DBF1BFBD
:1025600093F7050281CB97000000E78060DA1345FE
:10257000040245BD93F7850081CB97000000E780FA
:10258000E0D21345840071BD93F7150081CB97000D
:102590000000E780A0B41345140061B593F745002F
:1025A00081CB97000000E78060B31345440095BDE0
:1025B00093F7050495C39747FF1F83C7A79091CB57
:1025C00097000000E780A0A491471747FF1F23252D
:1025D000F79013450404B1B593F705010145E38273
:1025E00007E49747FF1F9387E78DD84B9147631008
:1025F000F7049747FF1F9387278A9C4313D7270029
:102600008583D98F858B91E7B7E7040083A7071DE2
:102610008297B7E70400FC4F91451745FF1F03451C
:10262000E58A829785471747FF1F2327F78A1345B7
:102630000401C5BB9747FF1F2386A79A8280170313
:10264000FFFFE702C3A99747FF1F23A30788974708
:10265000FF1F23A1078885471734FF1F1304047841
:102660001747FF1F232AF7861C4083C78703174796
:10267000FF1F2305F7869790FFFFE780A08F29C5EE
:102680009717FF1F23A8A7EA1C4017050000130592
:10269000A5D783C787031747FF1F2301F7841717A1
:1026A000FF1FA305F7E89747FF1FA38D0780B7E734
:1026B000040083A7070882979747FF1F2388A780F6
:1026C0001703FFFF6700E3A3B7C7898E938767ED02
:1026D0001717FF1F2320F7E645BF1737FF1F0347D4
:1026E000677E795555E79737FF1F9387A77D03C707
:1026F000170005079736FF1FA386E67C03C7170060
:102700008D463377D7029736FF1FA38DE67A83C6AF
:1027100017001737FF1F1307676C184393F6F60F60
:10272000A9EE834787031737FF1F2309F77A8547E9
:102730001737FF1F2308F7789737FF1F9387C77551
:102740009C430145998BA9E71703FFFFE7022399F3
:1027500037E404007C48C1451735FF1F0345057762
:1027600082973C4885451735FF1F0345257682979C
:1027700001451703FFFF6700C39883C7170085460D
:102780006395F6008347970379BF8347A70361BF2B
:1027900082809737FF1F83C7E772A1CF1703FFFF20
:1027A000E702E39337E404009737FF1F238C077099
:1027B0007C4885451735FF1F0345457182977C4C42
:1027C00091451735FF1F0345657082977C489145F9
:1027D0001735FF1F0345856F82973C48C145173564
:1027E000FF1F0345A56E829701451703FFFF670092
:1027F0004391795582801703FFFFE702438E2A84B5
:10280000035565FF9780FFFFE780A0179737FF1FED
:102810009387476BD847BE841DEF9790FFFFE780F3
:1028200080779C48232004009DEB9737FF1F23A34C
:10283000876A9737FF1F23AD8768B7E70400BC4B53
:1028400089451735FF1F03456568829701451703C2
:10285000FFFF6700038B630A8700184375BF80C3BF
:102860009737FF1F23A88766C9BF7955CDB71703D0
:10287000FFFFE702C3869737FF1F9387E7768843FA
:102880002326050023240500510597A00000E780BA
:10289000C0331703FFFF6700C3861703FFFFE7027C
:1028A00003841734FF1F130424741C40411199CF73
:1028B0009C472302B5002AC61CC197000000E78090
:1028C00040FB1C409C4B99C3324582974101170342
:1028D000FFFF670003831703FFFFE70243804111F7
:1028E000444D328532842EC69790FFFFE780C05258
:1028F0002AC422859790FFFFE780205403A8440054
:10290000630C0800B245835744001840224683D523
:102910004500AA8626850298410117F3FEFF67004D
:10292000437E17F3FEFFE702837B404D1DC808C0BE
:1029300097050000938565031305440197A00000E7
:10294000E78040169737FF1F9387076A9C4301452E
:1029500089E79737FF1F23A9876817F3FEFF6700F2
:10296000437A7D55DDBF17F3FEFFE7024377011180
:1029700068009305F00F02C602C802CA02CC02CE5C
:1029800097000000E780A0F1056117F3FEFF6700E4
:1029900043779737FF1F938727659C43D847A167E5
:1029A0009D076319F70217F3FEFFE7024373011156
:1029B00032859790FFFFE7802046230AA1008145DA
:1029C000680097000000E78080ED056117F3FEFFC7
:1029D0006700237382809737FF1F9387E7609C43CC
:1029E000D847A167938777036319F70217F3FEFFB0
:1029F000E702E36E011132859790FFFFE780C04147
:102A0000230AA1008145680097000000E78020E9C3
:102A1000056117F3FEFF6700C36E82809737FF1FC3
:102A20009387875C9C43D84795476316F70417F351
:102A3000FEFFE702C36A0111328532849790FFFFDF
:102A4000E780803D230AA10022859790FFFFE78061
:102A5000C03E83574400231BA10081453ECC1C404F
:102A600068003ECE97000000E78060E3056117F341
:102A7000FEFF670003698280930785FF8DC383276C
:102A8000C5FF91CFDC4B81CF17F3FEFFE702236533
:102A9000032585FF829717F3FEFF67008366828018
:102AA00017F3FEFFE702A3632A8432859790FFFFA6
:102AB000E7808036BD4763EBA70018449377F500A5
:102AC0000345B70041995D8DA305A70017F3FEFFED
:102AD0006700236317F3FEFFE702636001117C00C8
:102AE0003ECAB70707003ECC7C003ECE5C4DA9C76E
:102AF0002A8413858700AE8497A00000E780E0FC5D
:102B0000A1652A899D0548089770FFFFE780C03AB4
:102B10009305803EB345B902480893F5F50F9790A9
:102B2000FFFFE780C021014781465008A685228526
:102B30009770FFFFE780A05D056117F3FEFF670058
:102B4000435C17F3FEFFE702835997000000E7801C
:102B5000A0F817F3FEFF6700C35A17F3FEFFE70262
:102B6000035801117C00AE843ECAA165B707070077
:102B70002A843ECC48087C00938575033ECE97702E
:102B8000FFFFE78060331C44480883C5B700BD8958
:102B90009790FFFFE780A01A500801478146A6855D
:102BA00022859770FFFFE7808056056117F3FEFFCF
:102BB0006700235517F3FEFFE70263522A84AE84B1
:102BC00097000000E78000EEA685228597000000B0
:102BD000E780E0F817F3FEFF6700A35217F3FEFF4C
:102BE000E702E34F97000000E78060F717F3FEFF6E
:102BF0006700235117F3FEFFE702634E0329C50167
